:100000000C946B090C949C090C949C090C949C090D
:100010000C949C090C949C090C949C090C949C09CC
:100020000C949C090C949C090C949C090C949C09BC
:100030000C949C090C94B20F0C949C090C949C0990
:100040000C949C090C949C090C949C090C949C099C
:100050000C949C090C949C090C949C090C94B40E6F
:100060000C949C090C943D910C9413910C949C0954
:100070000C949C090C949C090C949C090C949C096C
:100080000C949C090C949C090C949C090C949C095C
:100090000C949C090C949C090C949C090C94D5100C
:1000A0000C949C090C949C090C949C090C949C093C
:1000B0000C949C090C949C090C949C090C949C092C
:1000C0000C949C090C949C090C949C090C949C091C
:1000D0000C949C090C949C090C94DD900C94B390A6
:1000E0000C949C090C943A0A0C94E10C0C940E0D9F
:1000F0000C94340A0C94C3280C94F8210C945F0AD5
:100100000C941D270C94467F0C949E090C948A2E07
:100110000C94BB240C94D88D0C94EF220C942B0FD0
:100120000C94640A0C94C81A0C9413820C94F12356
:100130000C94440A0C94800C0C94D4960C943425A2
:100140000C94D50C0C9475230C9482250C94EC0C17
:100150000C94560A0C941F0A0C9408240C94E40C7A
:100160000C949A0C0C946D250C944E270C9427211A
:100170000C94B1210C945F7F0C94B2090C94E98229
:100180000C94300C0C94F51A0C94C0090C94DF2ECE
:100190000C94D51C0C940B0D0C944C0A0C94807789
:1001A0000C94B40B0C94C0210C94040D0C94310AE3
:1001B0000C946C210C94557F0C94B00C0C94480A50
:1001C0000C94880B0C94187F0C94F00C0C946338EE
:1001D0000C94B0230C948F230C94BB0C0C9420191A
:1001E0000C94960C0C94AD0B0C9416950C94100C6E
:1001F0000C94520A0C94C5260C94D10C0C943E0A13
:100200000C94890B0C94E10B0C948B0B0C94E3264F
:100210000C94250A0C942D0A0C94290A0C94C41CE5
:100220000C94C1180C948A0B0C9442210C94192341
:100230000C94600A0C94D0220C94CC090C94297E66
:100240000C94B7180C9412250C949A0B0C94C7209C
:100250000C9419290C945A0A0C94DF0C0C94F40C8D
:100260000C94EE280C9493280C949C820C94197F87
:100270004E414E494E495459494E46CDCCCC3D0A8B
:10028000D7233C17B7D13877CC2B329595E6241F6E
:10029000B14F0A000020410000C84200401C462027
:1002A000BCBE4CCA1B0E5AAEC59D7400407A10F3FA
:1002B0005A00A0724E18090010A5D4E80000E87694
:1002C00048170000E40B54020000CA9A3B000000EB
:1002D000E1F505000080969800000040420F000004
:1002E00000A08601000000102700000000E80300C5
:1002F0000000006400000000000A0000000000018F
:1003000000000000002C76D888DC674F0823DFC18E
:10031000DFAE59E1B1B796E5E3E453C63AE6519949
:100320007696E8E6C28426EB898C9B62ED407C6F72
:10033000FCEFBC9C9F40F2BAA56FA5F490055A2A29
:10034000F75C936B6CF9676DC11BFCE0E40D47FE35
:10035000F520E6B500D0ED902E030094357705002A
:1003600080841E080000204E0A000000C80C3333B1
:1003700033330F986E12831141EF8D2114893BE6C0
:100380005516CFFEE6DB18D1844B381BF77C1D9049
:100390001DA4BBE424203284725E228100C9F124B2
:1003A000ECA1E53D27436F6E74656E742D54797032
:1003B000653A20746578742F68746D6C0D0A0D0AA7
:1003C0003C68313E45504943204641494C3C2F68EA
:1003D000313E00485454502F312E302034303020DC
:1003E00042616420526571756573740D0A00416342
:1003F000636573732D436F6E74726F6C2D416C6CFB
:100400006F772D4F726967696E3A202A0D0A436F24
:100410006E74656E742D547970653A200053657260
:100420007665723A205765626475696E6F2F312E5A
:10043000370D0A00485454502F312E3020323030BE
:10044000204F4B0D0A00506F7374206661696C6514
:100450006400436F6E6E656374696F6E3A20636CFF
:100460006F73650D0A00436F6E6E656374696F6E1E
:100470003A20636C6F73650D0A436F6E74656E741A
:100480002D547970653A206170706C69636174698C
:100490006F6E2F782D7777772D666F726D2D757251
:1004A0006C656E636F646564002D2D2D2D2D2D57A9
:1004B00065624B6974466F726D426F756E646172EE
:1004C000796A673271564955533874654F41624EA7
:1004D000332D2D00436F6E74656E742D54797065E5
:1004E0003A206170706C69636174696F6E2F6F631D
:1004F0007465742D73747265616D00436F6E7465FD
:100500006E742D446973706F736974696F6E3A20ED
:10051000666F726D2D646174613B206E616D653D27
:100520002266696C65223B2066696C656E616D654B
:100530003D22002D2D2D2D2D2D5765624B697446C2
:100540006F726D426F756E646172796A673271564F
:100550004955533874654F41624E3300436F6E7492
:10056000656E742D4C656E6774683A2000436F6E3B
:1005700074656E742D547970653A206D756C74696C
:10058000706172742F666F726D2D646174613B20AF
:10059000626F756E646172793D2D2D2D2D576562E8
:1005A0004B6974466F726D426F756E646172796AE1
:1005B000673271564955533874654F41624E330066
:1005C000436F6E6E656374696F6E3A20636C6F7310
:1005D0006500504F53542055706C6F616420466124
:1005E000696C65643A2000234E6F2073656E736FEB
:1005F0007220666F722074656D7020262068756D9C
:10060000696469747921004E6F2053656E736F724F
:10061000210020666F722074656D70202620687539
:100620006D696469747921002353656E736F72205C
:100630004572726F72200053656E736F722045723F
:10064000726F7221002357726F6E672073656E732D
:100650006F7220666F722074656D70202620687539
:100660006D6964697479210057726F6E67205365F4
:100670006E736F7221004320483D00543D002020DE
:10068000202020202020202020202020202000208A
:10069000202020202020202020202020202020007A
:1006A000202020202020202020202020202020204A
:1006B000002020202020202020202020202020205A
:1006C000002020202020202020202020202020204A
:1006D0000054696D657374616D702075706C6F6125
:1006E00064206661696C65640053657474696E6743
:1006F00020636C6F636B2074696D65002365727293
:100700006F72202D200049502061646472657373FC
:100710003A2000496E76616C696420534D207374F1
:100720006570732070657220616E676C653D005363
:100730004D2073746570732070657220616E676CF4
:10074000653D003C703E54696D653A20003C2F6861
:10075000333E0A003C62723E4254206E616D653D3C
:10076000003C62723E506174683D003C68333E5309
:10077000797374656D3A2056657273696F6E3D00CA
:10078000506172616D657465727320726573657412
:1007900020646F6E6521002F6F652F736D6C696724
:1007A0006874706F2F73332F00234C616D70207647
:1007B0006F6C74616765207061726974793A2000AA
:1007C000235461626C6520616E676C652064697298
:1007D000656374696F6E3A20002343757272656EAB
:1007E0007420534D20697320230023534D3A5461E4
:1007F000626C652073746570732070657220616E21
:10080000676C653D0023534D3A506F6C6172697A95
:1008100065722073746570732070657220616E67F5
:100820006C653D002344485450494E3D00234448E4
:10083000543D00236E65743D424C4500236E657443
:100840003D5769466900236E65743D425400236636
:10085000747020757365726E616D653A003A00239D
:10086000486F7374207365727665722049502061F9
:100870006E6420506F72743A002354696D65207362
:1008800065727665722049503A002352656C617931
:1008900020646576696365733A002352656C6179FB
:1008A00020737461747573206C6162656C733A2097
:1008B000002352656C6179207374617465733A002A
:1008C0002352656C61792070696E733A00234E6F14
:1008D0002E206F6620636F6E74726F6C2072656C71
:1008E0006179733D00234E6F2E206F662072656C18
:1008F0006179733D0046696E64696E672057694689
:1009000069204950004E45543D426C7565746F6FC7
:100910007468204C45004E45543D426C7565746FBB
:100920006F7468004E45543D576946690053442032
:100930006F70656E206661696C004E65772064613A
:10094000746120636F6C6C656374696F6E2073747F
:1009500061727465640053484F57533D00484947DE
:1009600048004C4F57004E4557002343757272653F
:100970006E742073657474696E67733A00534554DE
:100980000053797374656D207265736574206174AA
:1009900020005245534554005052494E5450415244
:1009A00000524541445344005341564553443D0091
:1009B00023445320546865726D6F6D6574657220B1
:1009C00063616C6962726174656420666F72202372
:1009D0000044535400496E76616C696420616E670F
:1009E0006C6520666F7220004D323D004E3D004D1B
:1009F000323D004E3D002073746570732070657247
:100A000020616E676C653D005350413D005453506A
:100A1000413D00505350413D005350413D00207333
:100A2000746570732070657220616E676C653D003F
:100A300046313030300046353030004631303030CD
:100A400000414E474D0054414E47430050414E47F0
:100A50004300414E4743005461626C654000506F53
:100A60006C6172697A65724000414E474D3D005499
:100A7000414E474D3D0050414E474D3D00414E4790
:100A80004D3D00414E47533D005233300054414EDE
:100A900047533D0050414E47533D00414E47533D63
:100AA000005200414E474C453D0054413D005041ED
:100AB0003D00413D00414E474C453D005461626C54
:100AC0006520536574203000235475726E74616222
:100AD0006C6520536574203000523330004633304B
:100AE00000506F6C6172697A6572205365742030B2
:100AF0000023506F6C6172697A65722053657420AF
:100B00003000505A45524F3D00540050005A455253
:100B10004F005461626C652053657420300023548B
:100B200075726E7461626C6520536574203000507C
:100B30006F6C6172697A657220536574203000238E
:100B4000506F6C6172697A65722053657420300051
:100B500053455400505A45524F3D005A45524F009C
:100B600053504545443D005053504545443D005485
:100B700053504545443D0053504545443D004D3D8F
:100B8000004D4F544F523D004D3D004D4F544F527C
:100B90003D00534D3D00535445503D004453544E89
:100BA0003D005256484947483D0052564C4F573D2C
:100BB000004C4F5746414E54494D453D004849472A
:100BC000484D4F544F523D004C4F574D4F544F528C
:100BD0003D004849474854454D503D004C4F5754FF
:100BE000454D503D0054454D50433D007361766581
:100BF00053443D004E45543D0057694669204950D5
:100C00003A0049504144440041542B0050494E3D64
:100C10000042543D004C43443D00534554434C4F27
:100C2000434B00234C6F67676572204E616D653AD8
:100C300020004C4F474745520056455253494F4EAE
:100C4000002344657669636520737461747573204D
:100C500075706C6F6164656421005553544154553F
:100C600053005265626F6F74696E672E2E2E0052AC
:100C700045424F4F540053657276657220506F7233
:100C80007420757064617465640053504F52543D14
:100C90000049502075706461746564005349503D8B
:100CA000002354696D652053657276657220495042
:100CB000207570646174656400545349503D00525E
:100CC000454C41593F0052454C4159200043524543
:100CD0004C41590044485450494E3D00524E414DFC
:100CE000453D004E523D005052494E54004E554E27
:100CF0004348554B3D004155544F53544152543D88
:100D00000074696D6520696E74657276616C3D0072
:100D100054494D453D0054494D455354414D503D76
:100D20000054494D455354414D500053484F574985
:100D300050005445535452454C4159004348454393
:100D40004B433D00434845434B543D004453543DC1
:100D5000004C5041524954593D0046414E3D004FD0
:100D600056454E3D004448543D0050573D005553B4
:100D700045523D00504154483D007C3C3E5E2B3D79
:100D80003F2F5B5D3B2C2A225C00000020002300EB
:100D9000260029002C002F00320000010000030172
:100DA0000601090100000A0B02090C0D0E080703D9
:100DB000040100000000000000000000000000002E
:100DC0000000000000000000000000000000000023
:100DD00012111000000000000000000000000000E0
:100DE000000000000000000000003C703E4C616DFF
:100DF0007020616E64204D6F746F7220447269764A
:100E000065727320537461747573EFBC9A3C2F70D4
:100E10003E003C21646F63747970652068746D6C6A
:100E20003E3C68746D6C3E3C686561643E3C6D653B
:100E3000746120636861727365743D227574662DF8
:100E400038223E3C7469746C653E4F6E6C696E6509
:100E5000206578706572696D656E74202D20506F05
:100E60006C6172697A6174696F6E2065666665632C
:100E70007473206F66206C696768743C2F746974A2
:100E80006C653E3C2F686561643E3C626F64793EF0
:100E90003C68313E4F6E6C696E6520657870657296
:100EA000696D656E74202D20506F6C6172697A6176
:100EB00074696F6E2065666665637473206F662063
:100EC0006C696768743C2F68313E003C68343E436F
:100ED0006F70797269676874284329323032302D17
:100EE000323032322E50726F662E205945554E47A1
:100EF00020596175205975656E3C2F68343E3C2F32
:100F0000626F64793E3C2F68746D6C3E003C6831C2
:100F10003E43616E6E6F74206765742073656E73F7
:100F20006F722072656164696E6773213C2F68314E
:100F30003E0023776562736572766572206265672D
:100F4000696E730053657474696E6720495000536D
:100F5000657474696E6720446576696365204950DD
:100F6000202E2E2E00506F6C6172697A65722053AC
:100F7000657420300023506F6C6172697A6572204D
:100F800053657474696E6720302E2E2E005465737D
:100F900074204C616D70732F46616E7300657272C0
:100FA0006F72206F70656E696E672066696C653A56
:100FB00020004C616D70204D6F746F720023546976
:100FC0006D65202020202020446174652020202091
:100FD000205365636F6E647320506F6C6172697A21
:100FE0006572205461626C652054286F4329204843
:100FF000282529202000696E69742E20646F6E6593
:101000002E00534420696E69742E206661696C65F8
:10101000642100696E69742E206661696C656421C3
:101020000053657474696E672049502063616D00D8
:101030002323204F452057656C636F6D6520232364
:1010400000496E697469616C697A696E67205344FE
:1010500020636172642E2E2E0053797374656D20A7
:101060007374617274696E672E2E2E0075706C6FCA
:10107000616420627920465450206661696C656421
:10108000210075706C6F6164206279204654502095
:101090004F4B210053797374656D207265737461D1
:1010A0007274656421002053797374656D207265D4
:1010B000737461727465642100234E6574776F7276
:1010C0006B206D61696E7461696E65642061742066
:1010D000002323436F6D6D616E6440000A00446518
:1010E0007669636520737461747573206174200080
:1010F00000002200250028002B002E0031003400C3
:1011000002010000050108010B010000210024007C
:1011100027002A002D0030003300010100000401E7
:1011200007010A01010210202008081020401020A9
:10113000408002010201080402010102040810209B
:101140004080804020100804020180040201804099
:101150002010080402010804020101020408102002
:1011600040800102040810204080050505050705A0
:1011700008080808020202020A0A08080404040413
:10118000010101010101010103030303030303033F
:10119000040707070C0C0C0C0C0C0C0C02020202CE
:1011A00006060606060606060B0B0B0B0B0B0B0BB7
:1011B000417070656E64206D6561732E2000536907
:1011C0006E676C65206D6561732E200053617665D6
:1011D000206D65617375726520746F3A0020202060
:1011E000202020202020202020202020200000005F
:1011F000010001001010020001000100B000000019
:101200001600000028000000100000002000000070
:1012100001000100000000000000000000000000CC
:1012200000000000000000000000000000000000BE
:10123000FF000000FFFF0000FFFF0000FFFF0000B5
:10124000CFBF0000C7BF0000C3BF0000C1BF000088
:10125000C0BF000000000000C0BF0000C1BF000010
:10126000C3BF0000C7BF0000CFBF0000FFFF0000EA
:10127000FFFF000000000000000000000000000070
:10128000000000000000000000000000000000005E
:10129000000000000000000000000000000000004E
:1012A000000000000000000000000000000000003E
:1012B00000000000557365722D6167656E743A20F9
:1012C0002A0D0A446973616C6C6F773A202F0D0AFE
:1012D0000000D496169511241FBECFEFD1E2DEBFD9
:1012E000CDBF00E00CBF18E0A0E0B2E0ECE3F3E714
:1012F00001E00BBF02C007900D92A03AB107D9F7E9
:1013000024E1A0EAB8E001C01D92AC32B207E1F7D7
:1013100019E0CAE6D9E000E006C021970109802F54
:10132000FE010E94A5B6C936D10780E00807A9F7DB
:101330000E9491990C948CB90C940000FC01918D41
:10134000828D981761F0A28DAE0FBF2FB11D5D96F3
:101350008C91928D9F5F9F73928F90E008958FEF95
:101360009FEF0895FC01918D828D981731F0828D49
:10137000E80FF11D858D90E008958FEF9FEF0895A0
:10138000FC01918D228D892F90E0805C9F4F821B04
:1013900091098F73992708958FE59FE7892B49F06D
:1013A00080E090E0892B29F00E945F7F81110E94EC
:1013B000000080E090E0892B49F080E090E0892BEC
:1013C00029F00E94000081110E94000080E090E05E
:1013D000892B49F080E090E0892B29F00E940000E1
:1013E00081110E94000085E59FE7892B49F080E08C
:1013F00090E0892B29F00E94557F81110C94000008
:1014000008958150823108F05AC0E82FF0E0882713
:10141000E35FF54F8F4F0C94A5B62D0A310A1F0AD2
:10142000250A290A5F0A340A3A0A3E0A440A480A87
:101430004C0A520A560A5F0A5A0A600A640A8091E4
:1014400080008F77809380000895809180008F7D49
:10145000F9CF80918000877FF5CF84B58F7784BDE9
:10146000089584B58F7DFBCF8091B0008F778093F6
:10147000B00008958091B0008F7DF9CF80919000E9
:101480008F77809390000895809190008F7DF9CFA1
:1014900080919000877FF5CF8091A0008F77809317
:1014A000A00008958091A0008F7DF9CF8091A000C9
:1014B000877FF5CF809120018F7780932001089559
:1014C000809120018F7DF9CF80912001877FF5CF1A
:1014D0004F925F926F927F928F929F92AF92BF9244
:1014E000CF92DF92EF92FF920F931F93CF93DF93F0
:1014F0004B015C018091B20B9091B30BA091B40BA6
:10150000B091B50B88159905AA05BB0509F4C6C0AD
:101510008CE3C82ED12CE12CF12CC501A70196013A
:101520000E940FB56093B60BCA01B901A7019601DD
:101530000E940FB56093B70BC501B40120E13EE0F6
:1015400040E050E00E940FB5CA01B90128E130E047
:1015500040E050E00E940FB56093B80BC501B401A4
:1015600020E831E541E050E00E940FB569017A01C1
:10157000CA01B9016C5F7F4F8F4F9F4F27E030E06A
:1015800040E050E00E940FB56F5F6093B90B412CB3
:10159000512C320140E004E610E0C0E9D1E0242FF4
:1015A00030E02E54384FF901E370FF273097F9F4FB
:1015B000C901B8010E9491B6892B31F4C901BE015D
:1015C0000E9491B6892B99F48EE691E0A0E0B0E0FC
:1015D000480E591E6A1E7B1ED301C201AA27BB27D3
:1015E000C816D906EA06FB0638F04F5FD8CF8DE65D
:1015F00091E0A0E0B0E0ECCF4093BC0BC90164E601
:1016000070E00E9491B6EC01C90160E971E00E94AE
:1016100091B6309721F42097D9F40097C9F04DE6A0
:1016200051E060E070E0441A550A660A770AC4186F
:10163000D508E608F708A5E2B3E020E0213069F418
:101640003097E9F5209711F40097C9F54DE106C0F0
:101650004EE651E060E070E0E6CF4C9150E070E083
:1016600060E031E0320FC416D506E606F70640F01A
:10167000C41AD50AE60AF70A1196232F3C30F1F670
:101680002F5F2093BB0BC394C092BA0B8092B20B16
:101690009092B30BA092B40BB092B50BDF91CF91A7
:1016A0001F910F91FF90EF90DF90CF90BF90AF9080
:1016B0009F908F907F906F905F904F9008954CE136
:1016C000CDCF2091BE0A260F3327331F213231059B
:1016D000ECF42091890EFC0190E080E0243069F068
:1016E00082E00895A091BE0A2191AC014256554F67
:1016F000A40FB52FB11D2C930196861798F38091F6
:10170000BE0A680F6093BE0A80E0089581E00895E4
:10171000089508950895E091430C8091420CE817D4
:1017200030F4F0E0E358F54F808190E008958FEFBA
:101730009FEF08959091430C8091420C2FEF3FEF63
:10174000981748F4E92FF0E0E358F54F208130E096
:101750009F5F9093430CC90108958091420C909132
:10176000430C891B990B0895CF92DF92EF92FF9261
:101770000F931F93CF93DF937C01CB018A012091BC
:101780008F0E222389F0EB016B01C40ED51ECC1500
:10179000DD0569F06991D701ED91FC910190F0812F
:1017A000E02DC7011995F3CF642F0E94610BC8018A
:1017B000DF91CF911F910F91FF90EF90DF90CF902D
:1017C0000895CF93DF931F92CDB7DEB76983209141
:1017D0008F0E2223F9F02091B20E203258F021E032
:1017E00030E0FC013383228390E080E00F90DF91B2
:1017F000CF9108958091900EE82FF0E0EF56F14FD1
:10180000998190838F5F8093900E8093B20E81E0D8
:1018100090E0ECCF61E0CE0101960E94610BF7CF22
:10182000DC015996ED91FC913097B9F08389948948
:10183000A589B6894285538564857585841B950B7A
:10184000A60BB70B811520E89207A105B10538F06A
:101850008FEF9FE7A0E0B0E0089590E080E008956A
:10186000CF93DF931F92CDB7DEB76983DC01ED9193
:10187000FC910280F381E02D41E050E0BE016F5FFA
:101880007F4F19950F90DF91CF910895FC01208132
:101890002EBD9B012150310941F051810DB407FE4D
:1018A000FDCF4EB55EBD4193F5CF61507109860FF6
:1018B000971F0DB407FEFDCF2EB5FC0120830895C0
:1018C000E091480CF091490C90818091470C8095F3
:1018D0008923808308958EBD00000DB407FEFDCFDF
:1018E0008EB5089590E020914A0C233339F40C967C
:1018F000982F990F990F990F80E008954896F8CF87
:10190000CF93DF931F92CDB7DEB76983DC01ED91F2
:10191000FC910280F381E02D41E050E0BE016F5F59
:101920007F4F19950F90DF91CF910895FC01818D24
:10193000928D0895CF93DF931F92CDB7DEB7698361
:10194000DC01ED91FC910280F381E02D41E050E05B
:10195000BE016F5F7F4F19950F90DF91CF91089572
:10196000FC019485FB018485981303C081E09830C5
:1019700008F080E00895CF93DF931F92CDB7DEB7D4
:101980006983DC01ED91FC910280F381E02D41E05F
:1019900050E0BE016F5F7F4F19950F90DF91CF919F
:1019A0000895FC01768765870895DC01ED91FC912F
:1019B000068CF78DE02D199591E089270895862FE3
:1019C000089581E08627089521E0FC018485883010
:1019D00008F020E0822F0895FC0184859585089504
:1019E000FC0184899589089520E334E0FC0131836A
:1019F0002083FB014089518962897389FC014283FC
:101A00005383648375830895DC01ED91FC91048C0C
:101A1000F58DE02D199490E080E00895CF92DF924B
:101A2000EF92FF920F931F93CF93DF93CDB7DEB763
:101A3000AF970FB6F894DEBF0FBECDBF7C016A0131
:101A400000E314E01A8309831C861B8688EE93E06A
:101A5000A0E0B0E08D879E87AF87B88B8AEB93E0DC
:101A60009A878987188F0F8B198E1A8E1B8E1C8E62
:101A700088E089A31BA70AA71CA61DA61EA61FA651
:101A80008091451090914610A0914710B091481058
:101A90008EA39FA3A8A7B9A78B839C83AD83BE8386
:101AA00018861F82AE01465D5F4FCE0101960E94EF
:101AB000A78681309105B1F4D701ED91FC9104889E
:101AC000F589E02D1DA30CA38CA59DA5AEA5BFA5F2
:101AD0008EA39FA3A8A7B9A7A601BE016C5D7F4FE7
:101AE000C7011995AF960FB6F894DEBF0FBECDBFF4
:101AF000DF91CF911F910F91FF90EF90DF90CF90EA
:101B00000895FC01A48DA80FB92FB11DA35ABF4F92
:101B10002C91848D90E001968F739927848FA689EC
:101B2000B7892C93A089B1898C91837080648C9340
:101B3000938D848D981306C00288F389E02D8081EF
:101B40008F7D80830895CF93DF93282F30E0F901B4
:101B5000EC55F24F8491F901EC5DFE4ED491F90100
:101B6000E659FE4EC491CC23A1F081110E94010AD6
:101B7000EC2FF0E0EE0FFF1FE657F24FA591B49166
:101B8000EC91ED2381E090E009F480E0DF91CF91CA
:101B9000089580E090E0FACF1F93CF93DF93282F32
:101BA00030E0F901EC55F24F8491F901EC5DFE4E05
:101BB000D491F901E659FE4EC491CC23A9F0162F19
:101BC00081110E94010AEC2FF0E0EE0FFF1FE0519F
:101BD000FF4EA591B4918FB7F894EC91111108C004
:101BE000D095DE23DC938FBFDF91CF911F910895B5
:101BF000DE2BF8CFCF93DF9390E0FC01EC5DFE4E3F
:101C0000249186599E4EFC0184918823D1F090E066
:101C1000880F991FFC01E65FFE4EA591B491FC016F
:101C2000E051FF4EC591D49161110EC09FB7F89459
:101C30008C91E22FE0958E238C932881E223E88318
:101C40009FBFDF91CF9108958FB7F894EC91E22B6D
:101C5000EC938FBFF6CF3FB7F8948091D00B909163
:101C6000D10BA091D20BB091D30B26B5A89B05C088
:101C70002F3F19F00196A11DB11D3FBFBA2FA92F0B
:101C8000982F8827BC01CD01620F711D811D911D08
:101C900042E0660F771F881F991F4A95D1F7089574
:101CA0008F929F92AF92BF92CF92DF92EF92FF926C
:101CB0006B017C010E942B0E4B015C01C114D1040D
:101CC000E104F104B9F00E942B0E681979098A0920
:101CD0009B09683E73408105910580F321E0C21A9B
:101CE000D108E108F10888EE880E83E0981EA11C57
:101CF000B11CE4CFFF90EF90DF90CF90BF90AF90FA
:101D00009F908F9008952FB7F8946091CC0B7091AD
:101D1000CD0B8091CE0B9091CF0B2FBF0895609388
:101D2000C70B7093C80B8093C90B9093CA0B645D6B
:101D30007E4F8F4F9F4F6093C30B7093C40B809364
:101D4000C50B9093C60B82E090E09093C20B8093FA
:101D5000C10B0E94830E6093BD0B7093BE0B8093EA
:101D6000BF0B9093C00B08951F920F920FB60F9266
:101D700011242F933F938F939F93AF93BF938091A1
:101D8000CC0B9091CD0BA091CE0BB091CF0B30919D
:101D9000CB0B23E0230F2D3758F50196A11DB11D64
:101DA0002093CB0B8093CC0B9093CD0BA093CE0BB9
:101DB000B093CF0B8091D00B9091D10BA091D20B0F
:101DC000B091D30B0196A11DB11D8093D00B9093C0
:101DD000D10BA093D20BB093D30BBF91AF919F9136
:101DE0008F913F912F910F900FBE0F901F901895DC
:101DF00026E8230F0296A11DB11DD2CFFC0124813C
:101E000031E030938F0E2093B10E1092900E10920D
:101E1000B20E8385682B8EEE9FE00E94E10B81E07D
:101E20000C940C830F931F93CF938C01C62F0E94A9
:101E3000FE0E6C2F6460C8010E94FE0E6C2F6B7F3B
:101E4000C8010E94FE0E83EC90E00197F1F7CF915C
:101E50001F910F9108950F931F93CF938C01C62F5D
:101E6000607F61600E94120F80E1C89FB001112461
:101E70006160C8010E94120F81E090E0CF911F9134
:101E80000F910895CF92DF92EF92FF920F931F93DD
:101E90000E94830E8B019C01C090BD0BD090BE0BA5
:101EA000E090BF0BF090C00B6091C70B7091C80B16
:101EB0008091C90B9091CA0B0C191D092E093F097D
:101EC000083E134021053105E0F0DC01CB0101960D
:101ED000A11DB11D8093C70B9093C80BA093C90B94
:101EE000B093CA0BB701A60148515C4F6F4F7F4FAB
:101EF0004093BD0B5093BE0B6093BF0B7093C00B10
:101F0000C7CF1F910F91FF90EF90DF90CF90089572
:101F10000E94420F0E94680A8091BC0B90E08E5490
:101F2000984F08950E94420F0E94680A8091BB0B4F
:101F300090E008950E94420F0E94680A8091BA0BB7
:101F400090E008950E94420F0E94680A8091B70BAA
:101F500090E008950E94420F0E94680A8091B80B99
:101F600090E008951F920F920FB60F9211240BB6B6
:101F70000F922F933F934F935F936F937F938F9322
:101F80009F93AF93BF93EF93FF938091E20A0E94D8
:101F9000A30D2091E50A3091E60A2F5F3F4F309361
:101FA000E60A2093E50A9091E40A953618F096E047
:101FB0009093E10A9091E10A943009F46EC0F8F42C
:101FC000923031F1933009F44CC09091E30A992397
:101FD00019F0811171C02F9AFF91EF91BF91AF91CC
:101FE0009F918F917F916F915F914F913F912F9131
:101FF0000F900BBE0F900FBE0F901F90189595304D
:1020000009F457C0963009F791E09093B10B4FC097
:102010008111DBCF2091E50A3091E60A24363105A3
:1020200028F41092E60A1092E50ACFCF1092B10B75
:102030001092E40AE091E40A91E09E0F9093E40A82
:10204000F0E02091E50A3091E60AEE0FFF1FE9511A
:10205000F54F318320831092E60A1092E50A93E04F
:1020600019C0813009F0B1CFE091E40A91E09E0FF0
:102070009093E40AF0E02091E50A3091E60AEE0F31
:10208000FF1FE951F54F318320831092E60A109229
:10209000E50A94E09093E10A98CF882359F22091C1
:1020A000E50A3091E60A2536310508F48ECF95E031
:1020B000F1CF81118ACFB5CF2F988ECF1092890E94
:1020C00081E08093880E1092630E61E084E10E94AB
:1020D000CC0D61E085E10E94CC0DE9EBF0E0808160
:1020E0008E7F808380818D7F808388E48093B80099
:1020F00085E48093BC000895CF93DF9391E09093A3
:102100009D0A8823B9F0C091B800D091BA0080919F
:10211000BC008A7B8093BC0060E084E10E94CC0D0F
:1021200060E085E10E94CC0D0E945E10D093BA0061
:10213000C093B800DF91CF91089585ED8093BC00E6
:1021400080918B0E90918C0EA0918D0EB0918E0E81
:102150000796A11DB11D23E0B695A7959795879584
:102160002A95D1F72091BC0024FD03C01092890E5E
:10217000089540918B0E50918C0E60918D0E709150
:102180008E0E452B462B472B69F30097A105B10511
:1021900041F025E32A95F1F700000197A109B10963
:1021A000E1CF80918A0E0C947C101F920F920FB693
:1021B0000F9211240BB60F922F933F934F935F937F
:1021C0006F937F938F939F93AF93BF93EF93FF93FF
:1021D0008091B900887F803609F44DC008F040C076
:1021E000883209F4A9C028F5803109F49DC0C8F4EB
:1021F000882309F4FBC0883009F496C0FF91EF9161
:10220000BF91AF919F918F917F916F915F914F910E
:102210003F912F910F900BBE0F900FBE0F901F900C
:102220001895883109F488C0803241F78093870E71
:1022300014C0803409F49DC040F48033B9F388336E
:10224000E9F68093870E85ECB0C0803509F485C02F
:10225000883509F496C0883489F60E949D10CECF47
:10226000883909F48CC038F5883729F050F488365D
:1022700011F0803719F683E08093890E1092E00AFE
:1022800057C0883809F47BC0803919F0803809F0CC
:10229000B5CF8091E00A803208F071C0E091E00A89
:1022A00081E08E0F8093E00A8091BB00F0E0E05463
:1022B000F54F80833DC0803B39F0E0F4803A09F46B
:1022C00079C0883A09F09ACF84E08093890E109201
:1022D000BF0A1092BE0AE091400CF091410C199592
:1022E0008091BE0A81110FC081E08093BE0A1092D6
:1022F0009E0A09C0803C09F4A6CF883C09F4A3CF0C
:10230000883B09F07BCFE091BF0A81E08E0F80937C
:10231000BF0AF0E0E256F54F80818093BB009091B8
:10232000BF0A8091BE0A29C08091640E8093BB00D1
:1023300085EC8093BC0062CF9091860E8091850ED3
:10234000981758F5E091860E81E08E0F8093860EE7
:10235000F0E0EB59F14F8081E9CFE091860E81E00A
:102360008E0F8093860E8091BB00F0E0EB59F14F09
:1023700080839091860E8091850E9817C8F285E82B
:10238000D8CFE091860E81E08E0F8093860E8091EB
:10239000BB00F0E0EB59F14F80838091880E8111F2
:1023A0005CCF81E08093630E84EA8093BC0010923E
:1023B000890E24CF85EC8093BC001092890E809109
:1023C000E00A803230F4E091E00AF0E0E054F54FAA
:1023D00010826091E00A70E0E0913E0CF0913F0CB9
:1023E00080EC9AE019951092E00A08CF1092870EBF
:1023F00034CF61E0FC0184810C94CC0DCF93DF934A
:10240000EC018FEF8EBD2FEF8F819885AC014F5F70
:102410005F4F58874F838130924028F40DB407FEF8
:10242000FDCF2EBDF1CF0DB407FEFDCFCE010E9432
:10243000F9111E82DF91CF9108958EBD0DB407FE74
:10244000FDCF08958FEF0E941D128EB508958F92D3
:102450009F92AF92BF92FF920F931F93CF93DF9300
:10246000EC01F62E49015A018E81882319F0CE0124
:102470000E94FE1160E08C810E94CC0D8CE291E004
:102480000E94E1858F2D80640E941D1208E110E0FA
:10249000D501C401002E04C0B695A79597958795E0
:1024A0000A94D2F70E941D1208501109083F8FEFBD
:1024B000180771F785E9FF2021F088E0F8120DC0B8
:1024C00087E80E941D1210E00E9422128A8787FF6F
:1024D00006C01F3F21F01F5FF7CF8FEFF2CFDF91D4
:1024E000CF911F910F91FF90BF90AF909F908F90D1
:1024F0000895AF92BF92CF92DF92EF92FF920F9327
:102500001F93CF93DF93EC016901C801820F931FE2
:102510008130924050F58E81882379F088819981AD
:10252000AA81BB8184179507A607B70731F48F816D
:102530009885C816D90608F042C0488359836A8333
:102540007B838B85833039F089E0440F551F661FEC
:10255000771F8A95D1F79A01AB0161E1CE010E9404
:102560002712882389F083E08D83CE010E94F91120
:1025700080E0DF91CF911F910F91FF90EF90DF905E
:10258000CF90BF90AF9008950E94830E5B010E9490
:1025900022128A878F3F69F40E94830E6A197B0991
:1025A0006D327140A0F38FE08D83CE010E94F9114E
:1025B000DCCF8E3FB1F418861F8281E08E838FEFCF
:1025C0008EBD2FEF8F8198858C159D0560F40DB41D
:1025D00007FEFDCF2EBD8F819885019698878F834A
:1025E000F1CF8DE0E1CFC8010197F7012FEFAF01E7
:1025F0004E195F094817590738F40DB407FEFDCF8F
:102600003EB531932EBDF3CF0DB407FEFDCF2EB5F1
:10261000E80EF91EF70120838F819885080F191F96
:1026200018870F838985882319F00115124030F02F
:102630008E81882319F0CE010E94FE1181E099CF8E
:102640000F931F93CF93DF93EC01890182E1411532
:1026500051056105710599F08B85833039F089E06A
:10266000440F551F661F771F8A95D1F79A01AB015A
:1026700068E1CE010E942712882319F084E08D833F
:1026800038C08EEF8EBDF801C8019E5F0DB407FE05
:10269000FDCF20812EBD0DB407FEFDCF21812EBDC3
:1026A0003296E817F90791F70DB407FEFDCF8FEFCB
:1026B0000E941D128FEF0E941D120E9422128A8713
:1026C0008F71853089F488E592E00E94E185882346
:1026D000A9F020E030E0A9016DE0CE010E942712B0
:1026E000882371F084E1CBCF81E18D83CE010E94FC
:1026F000F911CE010E94F91180E00AC085E1BFCF37
:102700000E9422128111EECFCE010E94F91181E0C8
:10271000DF91CF911F910F9108958091780A8823BE
:10272000A9F1409144025091450260914602709196
:1027300047022FE53CE08091440C9091450C0E94AB
:102740002013811102C080E008954091790A5091D0
:102750007A0A60917B0A70917C0A411551056105E6
:10276000710591F02FE53CE08091440C9091450C6F
:102770000E942013882339F31092790A10927A0A62
:1027800010927B0A10927C0A1092780A81E00895D8
:102790008F929F92AF92BF92EF92FF920F931F93EF
:1027A000CF934B015C01C42F80914402909145026C
:1027B000A0914602B091470288159905AA05BB056C
:1027C00049F10E948D1381110BC080E0CF911F91C0
:1027D0000F91FF90EF90BF90AF909F908F900895D2
:1027E0008FE5E82E8CE0F82E00E012E030E020E0EB
:1027F000B501A4018091440C9091450C0E9479127E
:10280000882319F38092440290924502A0924602D6
:10281000B09247024091780A4C2B4093780A81E0AD
:10282000D5CF4F925F926F927F928F929F92AF928D
:10283000BF92CF92DF92EF92FF920F931F93CF93AD
:10284000DF93EC01423051056105710590F480E0A1
:10285000DF91CF911F910F91FF90EF90DF90CF907C
:10286000BF90AF909F908F907F906F905F904F90B0
:10287000089589859A85AB85BC850196A11DB11DFA
:1028800084179507A607B70710F3CB88DC88ED8877
:10289000FE888F89803109F042C0BB27A72F962F71
:1028A000852F480159012A013B01C80ED91EEA1E95
:1028B000FB1E8091440290914502A0914602B09186
:1028C0004702C816D906EA06FB0699F58F898031BA
:1028D000C1F5B301A201552766277727440F551F7D
:1028E000415A534FFA01918280828091780A816027
:1028F0008093780A8A89823080F08D819E81AF81B1
:10290000B8858C0D9D1DAE1DBF1D8093790A9093D7
:102910007A0AA0937B0AB0937C0A81E099CFDB010D
:10292000CA01E7E0B695A79597958795EA95D1F7FF
:10293000B8CF40E0C701B6010E94C8138111C6CFCD
:1029400086CFB301A2014F77552766277727440F1B
:10295000551F440F551F415A534FFA0180829182EF
:10296000A282B382C2CF8F929F92AF92BF92CF9238
:10297000DF92EF92FF920F931F93CF93DF93FC01AF
:1029800081859285A385B4850196A11DB11D84170B
:102990009507A607B70770F480E0DF91CF911F91EC
:1029A0000F91FF90EF90DF90CF90BF90AF909F90EE
:1029B0008F90089583889488A588B6888789803108
:1029C00089F5BB27A72F962F852FE9016A017B0187
:1029D0008F01BC01CD01680D791D8A1D9B1D809062
:1029E000440290904502A0904602B090470286169D
:1029F0009706A806B90601F5F8018789803111F517
:102A0000DD24EE24FF24F601EE0FFF1FE15AF34F01
:102A100080819181B0E0A0E088839983AA83BB8301
:102A200081E0BBCFDB01CA01C7E0B695A7959795BA
:102A30008795CA95D1F7C9CF40E00E94C81381118C
:102A4000DBCFAACFE894C7F8DD24EE24FF24F601FB
:102A5000EE0FFF1FEE0FFF1FE15AF34F80819181B0
:102A6000A281B381BF70D8CF4F925F926F927F9255
:102A7000AF92BF92CF92DF92EF92FF920F931F938C
:102A8000CF93DF9300D01F92CDB7DEB78C0149837F
:102A90005A836B837C835901C12CD12C7601412C44
:102AA00082E0582E612C712C49815A816B817C8186
:102AB0009E012F5F3F4FC8010E94B314882339F154
:102AC000F8018585A301920104C0220F331F441F22
:102AD000551F8A95D2F7DA01C901C80ED91EEA1E20
:102AE000FB1E49815A816B817C818789803111F17C
:102AF00088EF9FEFAFEFBFE0481759076A077B07E2
:102B000098F2F501C082D182E282F38281E00F90D7
:102B10000F900F900F90DF91CF911F910F91FF9029
:102B2000EF90DF90CF90BF90AF907F906F905F90CD
:102B30004F90089588EF9FEFA0E0B0E0DDCFCF92F7
:102B4000DF92EF92FF921F93CF93DF93EC0180E22D
:102B5000689FF0011124E15AF34F9385917161F060
:102B6000842F827449F080E0DF91CF911F91FF9014
:102B7000EF90DF90CF900895142F6A8B80914402DC
:102B800090914502A0914602B09147028E879F879F
:102B9000A88BB98BC488D588F12CE12C7601DD2473
:102BA000CC24CF8AD88EE98EFA8E828D938DB0E0B8
:102BB000A0E0AC01BD014C295D296E297F294F8B16
:102BC000588F698F7A8F83858871B1F4848D958D44
:102BD000A68DB78D8B8B9C8BAD8BBE8B81E08D834F
:102BE0001F701C831E821F82188619861A861B86F8
:102BF0001C861D8681E0B8CF803109F0B4CF9E01DC
:102C00002D5E3F4F8B8D9C8D0E943415882309F4D7
:102C1000AACF84E0E4CF8F929F92AF92BF92CF92DF
:102C2000DF92EF92FF920F931F93CF93DF93EC010C
:102C30008D8181110EC080E0DF91CF911F910F91A6
:102C4000FF90EF90DF90CF90BF90AF909F908F90CC
:102C500008950B891C892D893E89041715072607BD
:102C6000370748F34A015B01823031F48A869B863C
:102C7000AC86BD8681E0E0CF81149104A104B1044B
:102C800049F41E821F82188619861A861B861C86A6
:102C90001D86F0CF0A851B852C853D85EB8DFC8D2F
:102CA000858590E00996B901A80141505109610953
:102CB0007109082E04C076956795579547950A9433
:102CC000D2F775016401E1E0CE1AD108E108F108FC
:102CD00004C0F694E794D794C7948A95D2F7C416A3
:102CE000D506E606F70620F0012B022B032B11F583
:102CF0008F89988DA98DBA8D8E839F83A887B98778
:102D00008E010A5F1F4FC114D104E104F10409F4DC
:102D1000ADCF4E815F816885798598018B8D9C8DC3
:102D20000E94B31491E0C91AD108E108F108811199
:102D3000EACF81CFC41AD50AE60AF70AE1CF3F925B
:102D40004F925F926F927F928F929F92AF92BF92BB
:102D5000CF92DF92EF92FF920F931F93CF93DF9367
:102D6000CDB7DEB72C970FB6F894DEBF0FBECDBF40
:102D70005C01DC015B968D909C905C9716964D9063
:102D80005D906D907C901997411451046104710419
:102D900009F468C0BFEF4B1A5B0A6B0A7B0A312C3F
:102DA000F40181859285A385B4859C01AD012F5FD7
:102DB0003F4F4F4F5F4F29873A874B875C8773019F
:102DC00062011D821E821F821886F4018185928510
:102DD000A385B4852D813E814F81588528173907F9
:102DE0004A075B0708F056C089859A85AB85BC8584
:102DF0008C159D05AE05BF0550F482E0C82ED12C80
:102E0000E12CF12C92E0492E512C612C712C9E0169
:102E10002F5F3F4FB701A601C4010E94B31488235E
:102E2000C9F189819A81AB81BC81892B8A2B8B2B3B
:102E300009F1260137019FEF491A590A690A790AEF
:102E40002D813E814F8158852F5F3F4F4F4F5F4F00
:102E50002D833E834F8358873FEFC31AD30AE30A7B
:102E6000F30AB3CFF4014080518062807380332431
:102E7000339496CFC414D504E604F70409F70FEF92
:102E80001FEF2FEF3FE0B701A601C4010E9411140C
:102E9000811119C080E02C960FB6F894DEBF0FBEEA
:102EA000CDBFDF91CF911F910F91FF90EF90DF90F9
:102EB000CF90BF90AF909F908F907F906F905F90DA
:102EC0004F903F900895F501468157816085718547
:102ED000411551056105710539F097018601C4015D
:102EE0000E9411148823B1F2D5011696CD92DD927D
:102EF000ED92FC921997332051F0D701C60101964B
:102F0000A11DB11DF40180839183A283B383F501D8
:102F10008789908DA18DB28D892B8A2B8B2B39F4CB
:102F2000C78AD08EE18EF28E84818068848381E0AE
:102F3000B2CF2F923F924F925F926F927F928F9279
:102F40009F92AF92BF92CF92DF92EF92FF920F9338
:102F50001F93CF93DF93EC015B012A018D818111D7
:102F600015C08FEF9FEFDF91CF911F910F91FF90D1
:102F7000EF90DF90CF90BF90AF909F908F907F9019
:102F80006F905F904F903F902F9008958C8180FFBD
:102F9000E8CF0B891C892D893E894A855B856C8524
:102FA0007D85C201B0E0A0E068017901C41AD50AAC
:102FB000E60AF70AC816D906EA06FB0618F428013D
:102FC000441A550A42011E0126E0220E311C8114CA
:102FD000910409F4B3C04A855B856C857D856A01DF
:102FE00081E0D8228B8D9C8D8A019B01E9E036958A
:102FF000279517950795EA95D1F7ED81E230E1F530
:10300000FC01628D738D848D958D600F711F821F01
:10301000931F612C22E0722E6C187D088614970491
:1030200008F434012C8126FD04C06114F2E07F060F
:1030300071F40091440210914502209146023091B2
:103040004702061717072807390709F053C040E061
:103050000E94C813882309F484CFC601815A934F74
:10306000D5019C01260D371DFC012E173F0709F4E1
:1030700060C041914D93F9CFFC0174807A94702225
:10308000C114D10471F471100CC0452B462B472B91
:1030900039F58F89988DA98DBA8D8E839F83A887E6
:1030A000B987EB8DFC8D6E817F8188859985625013
:1030B000710981099109258504C0660F771F881F52
:1030C000991F2A95D2F70685178520893189600FC7
:1030D000711F821F931F670D711D811D911D99CF57
:1030E0004E815F816885798591010E94B3148111B9
:1030F000D8CF37CF750183019601AB01BC01809118
:10310000440C9091450C0E947912882309F429CF30
:10311000A60CB71C8A859B85AC85BD85860D971D41
:10312000A11DB11D8A879B87AC87BD87861897082C
:103130004ECF281B390BA20EB31EECCFC20113CF0A
:10314000CF93DF931F92CDB7DEB741E050E0BE01D1
:103150006F5F7F4F0E949917019731F4898190E04A
:103160000F90DF91CF9108958FEF9FEFF9CFFC0182
:10317000818D928D009711F00C94A0188FEF9FEF26
:1031800008950F931F93CF93DF93EC01898D9A8D50
:1031900010E000E0009799F00E94A0188C010F3F0A
:1031A000100769F0898D9A8DFC01428553856485ED
:1031B000758541505109610971090E940B16C801BA
:1031C000DF91CF911F910F910895CF93DF93EC0181
:1031D0008D81882329F18C8187FF1EC0CE010E943A
:1031E000FC85FC01892BE1F08D81823040F48B89D4
:1031F0009C89AD89BE89848F958FA68FB78F8F8963
:10320000988D938F828F8F89988DA98DBA8DB58B6C
:10321000A48B8C818F778C83DF91CF910C948D134D
:1032200080E0DF91CF910895CF93DF93EC010E946E
:10323000E518882311F01D8281E0DF91CF91089578
:10324000FC01818D928D009711F00C94E518089582
:103250003F924F925F926F927F928F929F92AF9226
:10326000BF92CF92DF92EF92FF920F931F93CF9373
:10327000DF9300D000D000D01F921F92CDB7DEB7F1
:103280007C01DC0115968C91811115C0FE013196EF
:10329000CE010C966F0130E23193E817F907E1F7A0
:1032A000DA0130E087E09D91B92E992329F19E3211
:1032B00039F48A3011F480E0D9C038E08AE0F3CFE5
:1032C000EAE7FDE04491442321F031969413FACFCC
:1032D000F2CF831780F34FED490F4E3560F74FE97A
:1032E000490F4A3118F440EEB42EB90EF601E30F3F
:1032F000F11DB0823F5FD7CF89818032E1F2322E5B
:103300008B01FB01838D948DD7015C969C938E93EA
:103310005B97168217821086118612861386148692
:103320001586F80182859385A485B58543895489DE
:103330006589768984179507A607B70708F04DC0F9
:1033400025E0B695A795979587952A95D1F7F82FFB
:10335000FF70AF2ED80115968C91823008F4ABCF58
:10336000C8010E94A01897FDA6CFF8018285938519
:10337000A485B5854F96A11DB11D82879387A4872B
:10338000B587F0E2AF9EB0011124615A734F611509
:10339000710509F490CFDB018C91882341F0853EC3
:1033A00009F057C0BB2029F0BB24B394BACFB110A9
:1033B0000EC0F701A28A8091440290914502A0912B
:1033C0004602B091470286879787A08BB18BDB01BD
:1033D0008C918111E9CFBB24B394832D827182310A
:1033E00009F069CFBB2009F459C0C7010E94FC85D0
:1033F000009709F460CF20E2FC0111922A95E9F7C9
:103400002BE0F601DC0101900D922A95E1F721E213
:1034100038E2DC0151963C932E93509740E058E0FF
:103420001F965C934E931E9753963C932E93529700
:1034300059963C932E93589757965C934E93569774
:103440000E948D13882309F436CF432DF70162893A
:103450000AC04BE050E0C6010E94DBB8892B09F09E
:1034600060CF432D6A2DC7010E949F152B960FB682
:10347000F894DEBF0FBECDBFDF91CF911F910F91AA
:10348000FF90EF90DF90CF90BF90AF909F908F9084
:103490007F906F905F904F903F900895F8018581E5
:1034A000823009F408CFC8010E949F16882309F4CE
:1034B00002CFD8015B96ED91FC915C9716968D90AA
:1034C0009D90AD90BC901997B2E08B1A9108A1081D
:1034D000B108858504C0880C991CAA1CBB1C8A9560
:1034E000D2F786859785A089B189880E991EAA1E74
:1034F000BB1E848124013501480E511C611C711CC6
:1035000084149504A604B70401F1E1E04E1A5108B1
:10351000610871080E948D13882309F4CCCEEFE571
:10352000FCE011928FE59EE08E179F07D1F7409245
:103530004402509245026092460270924702809186
:10354000780A81608093780ADBCFD8015B96ED9191
:10355000FC91258580E092E0A0E0B0E004C0880FF7
:10356000991FAA1FBB1F2A95D2F7F80143895489D6
:1035700065897689840F951FA61FB71F838B948B4F
:10358000A58BB68BD70152961C928FE59CE033CF6A
:103590001F93CF93DF93CDB7DEB76D970FB6F89437
:1035A000DEBF0FBECDBFAB011C821B8222E933E020
:1035B0003A8329831E8221E0BC01CE0101960E943C
:1035C000281911E081110CC010E0812F6D960FB603
:1035D000F894DEBF0FBECDBFDF91CF911F9108954C
:1035E000CE0101960E941419F0CFCF93DF93CDB78F
:1035F000DEB76D970FB6F894DEBF0FBECDBF442384
:1036000091F1AB01BC011C821B8282E993E09A8399
:1036100089831E8222E0CE0101960E942819811121
:103620000EC090E081E0911101C080E06D960FB670
:10363000F894DEBF0FBECDBFDF91CF910895CE01CC
:1036400001960E941586882361F3CE0101960E949F
:10365000FC85009731F325EEFC0120831E820E9439
:103660008D13982FDFCF81E0E1CF2F923F924F92C1
:103670005F926F927F928F929F92AF92BF92CF9202
:10368000DF92EF92FF920F931F93CF93DF9300D0BF
:103690001F92CDB7DEB78C015B011A01DC011596D4
:1036A0008C911597813009F0C8C014968C9181FFD8
:1036B000C4C082FDAEC06101D8011A964D915D91E2
:1036C0006D917C911D97C114D10409F429C15B96B9
:1036D0008D919C915C97FC0174802FEF270D2A013E
:1036E0003B0139E076946794579447943A95D1F723
:1036F000722E74207A01F1E0FF22711020C0E114D3
:10370000F104E9F416964D915D916D917C911997B4
:10371000411551056105710509F098C057968D91C5
:103720009D910D90BC91A02D0097A105B10509F0C8
:10373000AFC0C8010E949F16882309F47EC080E0B4
:1037400092E08E199F0946018C159D0508F44C01E5
:10375000D8015B964D915C915C9716968D919D91E9
:103760000D90BC91A02D0297A109B109FA01258500
:1037700004C0880F991FAA1FBB1F2A95D2F7468540
:10378000578560897189840F951FA61FB71F9C01FB
:10379000AD01270D311D411D511D29013A01811433
:1037A00032E0930609F07AC080914402909145027C
:1037B000A0914602B091470284159505A605B7056C
:1037C00059F48FEF9FEFDC01809344029093450200
:1037D000A0934602B09347029501B301A2018091E4
:1037E000440C9091450C0E942013882331F19EEFE8
:1037F000B91AC818D908F80182859385A485B585BA
:10380000880D991DA11DB11D82879387A487B58757
:1038100053CFF801438954896589768982859385D8
:10382000A485B585481759076A077B0709F443CF74
:10383000C8010E940B1681113ECF81E090E0D801B3
:1038400013969C938E93129780E007C09E012F5F82
:103850003F4F0E94B314811102C090E077C089816C
:103860009A81AB81BC81F801238D348DF9012789C0
:1038700048EF5FEF60E070E0203121F048EF5FEF4C
:103880006FEF7FE084179507A607B70708F051CFC1
:10389000F80186839783A087B18751CFE114F104A3
:1038A00091F5D8011A964D915D916D917C911D977E
:1038B00053968D919D910D90BC91A02D481759075D
:1038C0006A077B0700F10E948D13882309F4B5CFA6
:1038D0004092440250924502609246027092470222
:1038E0008091780A81608093780A9701215A334F3A
:1038F000D501C901880D991DF9018E179F0759F04F
:103900004D914193FACF41E0C301B2010E94C81327
:103910008111EBCF92CF821B930BA80EB91E69CFFA
:10392000F80183899489A589B68984179507A60724
:10393000B70738F48481438B548B658B768B806812
:103940008483F801848183FD18C0C1010F900F901A
:103950000F900F90DF91CF911F910F91FF90EF90FB
:10396000DF90CF90BF90AF909F908F907F906F909F
:103970005F904F903F902F900895C8010E94E518E6
:10398000882309F45ACFE1CFCF93DF931F92CDB7AD
:10399000DEB7698341E050E0BE016F5F7F4F0E9458
:1039A000351B0F90DF91CF910895CF93DF93EC01FA
:1039B000E98DFA8D309749F481E090E09B838A830A
:1039C00090E080E0DF91CF91089513821282898D7B
:1039D0009A8D0E94351BE98DFA8D22813381232B2C
:1039E00059F7F0CFFC01DB0112968D919C91139752
:1039F0009383828382E993E09183808314968C91F0
:103A00001497848315968C911597858316964D91FE
:103A10005D916D917C91199746835783608771877B
:103A20001A964D915D916D917C911D9742875387B8
:103A3000648775871E964D915D916D917C9151972C
:103A400046875787608B718B52968C915297828BE9
:103A500053964D915D916D917C915697438B548B0C
:103A6000658B768B57964D915D916D917C915A97B0
:103A7000478B508F618F728F5B968D919C91948F45
:103A8000838F0895DC015996ED91FC91309721F0D8
:103A900081E09581911101C080E00895CF93DF937B
:103AA000EC01898D9A8D009741F00E941419898D3F
:103AB0009A8D0E9464B71A8E198EDF91CF91089566
:103AC000EF92FF920F931F93CF93DF93EC017B0153
:103AD0008A011B821A8288EE93E0A0E0B0E08C831A
:103AE0009D83AE83BF8382E194E0998388838DE1D7
:103AF00090E00E94C8B69A8F898F009779F02DE1E7
:103B0000F701DC0101900D922A95E1F74CE050E0BD
:103B1000B801CE010C960E9433B9188EDF91CF9177
:103B20001F910F91FF90EF900895E091480CF09154
:103B3000490C80819091470C892B80830895AF9226
:103B4000BF92CF92DF92EF92FF920F931F93CF938A
:103B5000DF9300D01F92CDB7DEB78C016B017A01E5
:103B600080914A0C8333E9F45B016801C40ED51ED1
:103B7000C016D106A9F10E94600C8FE00E946B0C68
:103B8000812F0E946B0C802F0E946B0C0F5F1F4FC8
:103B900080E00E946B0CF50181935F010E94951DEE
:103BA000E7CF843369F50E94600C19830A838F2D57
:103BB0008F778B83EC8264E070E0CE0101960E94E7
:103BC000460CA70170E060E0C6010E9403B9E11451
:103BD000F10421F0B701C6010E94460C0E94951D18
:103BE000C7010F900F900F900F90DF91CF911F9111
:103BF0000F91FF90EF90DF90CF90BF90AF9008951E
:103C00000E94600C0F3F110509F030F419820A83FD
:103C10001B8263E070E0D1CF17FD0BC019820A83CD
:103C200033E0169507953A95E1F7007E08600B831F
:103C3000F0CFC80126E0969587952A95E1F7807E1A
:103C400019830A830115104C18F480618B83E1CF2E
:103C50008861FCCFCF93DF931F92CDB7DEB7209161
:103C60004B0C30E0322F2227260F371F90E0982F81
:103C7000882741E050E0BE016F5F7F4F820F931FA6
:103C80000E949F1D89810F90DF91CF910895AF927F
:103C9000BF92CF92DF92EF92FF920F931F93CF9339
:103CA000DF9300D000D01F921F92CDB7DEB78C01FA
:103CB0007B016A0180914A0C8333E1F45801A40E20
:103CC000B51EA016B10609F46FC00E94600C80EF0B
:103CD0000E946B0C812F0E946B0C802F0E946B0C3A
:103CE0000F5F1F4FF70181917F010E946B0C0E94B3
:103CF000951DE7CF5B01A40EB51E8433C1F40E946D
:103D0000600C19830A838D2D80688B83CC8264E0DC
:103D100070E0CE0101960E94460CAE14BF0409F477
:103D200041C0F70181917F010E946B0CF6CF0E9488
:103D3000600C0F3F110509F028F419820A8384E012
:103D40008B830CC017FD17C019820A8333E01695C8
:103D500007953A95E1F7007E0C600B8386E0C81664
:103D6000D104A0F5F701DE011496EA15FB0599F0E0
:103D700081918D93FACFC80126E0969587952A9573
:103D8000E1F7807E19830A830115104C10F48461D9
:103D9000D7CF8C61D5CFB6016D5F7F4FCE01019635
:103DA0000E94460C0E94951DC60128960FB6F894F5
:103DB000DEBF0FBECDBFDF91CF911F910F91FF905E
:103DC000EF90DF90CF90BF90AF90089563E070E0E8
:103DD000CE0101960E94460CF70181917F010E945D
:103DE0006B0CAE14BF04C1F7DDCFCF93DF931F92EE
:103DF000CDB7DEB741E050E0BE016F5F7F4F90E08E
:103E000080E00E949F1D89810F90DF91CF910895DE
:103E1000CF93DF93C4E1D0E00E94F51E882361F0C8
:103E200061E070E080E090E00E94500E2197A1F7E1
:103E300080E0DF91CF91089581E0FBCFCF93DF93B6
:103E40001F92CDB7DEB7898341E050E0BE016F5FBE
:103E50007F4F90E080E00E94471E0F90DF91CF914E
:103E6000089563E070E00C942A1EDA01E0914B0C97
:103E7000F0E0FE2FEE27E60FF71F90E0982F88273F
:103E8000A901BD018E0F9F1F0C94471ECF93DF9396
:103E90001F921F92CDB7DEB779836A8322E030E0AC
:103EA000AE014F5F5F4F60E170E00E94351F0F90E1
:103EB0000F90DF91CF910895CF93DF931F921F92C0
:103EC000CDB7DEB779836A8322E030E0AE014F5F81
:103ED0005F4F64E070E00E94351F0F900F90DF91FC
:103EE000CF910895CF93DF931F92CDB7DEB7209186
:103EF0004B0C30E0322F2227260F371F90E0982FEF
:103F00008827498341E050E0BE016F5F7F4F820FF9
:103F1000931F0E94471E0F90DF91CF910895CF937A
:103F2000C82F462F61E070E00E94721F61E070E0D0
:103F30008C2F0E942A1E8111F9CFCF910895DA01AA
:103F4000E0914B0CF0E0FE2FEE27E60FF71F90E01C
:103F5000982F8827A901BD018E0F9F1F0C949F1DCC
:103F60006F927F929F92AF92BF92CF92DF92EF9229
:103F7000FF920F931F93CF93DF931F921F92CDB7A2
:103F8000DEB7982E8B013A01690122E030E0AE01E4
:103F90004F5F5F4F64E270E00E949F1FE980FA80EC
:103FA000FE24EF24FE24E00EF11E970137704091AD
:103FB0004A0C092D10E0C801433309F04CC00896A3
:103FC000982F8827990F990F990F820F931F4733C6
:103FD00009F446C0A9014C0D5D1D4130584008F45C
:103FE0003FC060E078E05B01A21AB30AA501B3010B
:103FF0000E94471EA6014A195B09B3016A0D7B1D89
:1040000080914A0C833349F5085F1F4F000F000F62
:10401000000F80E0902F0E94471EEC0CFD1CF982DF
:10402000EA8222E030E0AE014F5F5F4F64E270E071
:10403000892D0E94351F0F900F90DF91CF911F9116
:104040000F91FF90EF90DF90CF90BF90AF909F9037
:104050007F906F9008954096B3CF005F1F4FD6CFEB
:10406000A601B301D8CFEF92FF921F93CF93DF93B6
:104070001F921F92CDB7DEB7182F22E030E0AE01BD
:104080004F5F5F4F60E270E00E949F1FE980FA80FF
:10409000FE24EF24FE2422E030E0AE014F5F5F4FAC
:1040A00060E270E0812F0E949F1F89819A8198278A
:1040B00089279827E816F90689F487E0189FF00108
:1040C0001124EA50F44FF582E482C7010F900F905B
:1040D000DF91CF911F91FF90EF9008957C01DBCF8E
:1040E000FF920F931F93CF93DF931F921F92CDB731
:1040F000DEB7F82E22E030E0AE014F5F5F4F66E2A0
:1041000070E00E949F1F09811A8110270127102744
:1041100022E030E0AE014F5F5F4F66E270E08F2D2E
:104120000E949F1F89819A819827892798270817BD
:10413000190749F4C8010F900F90DF91CF911F919B
:104140000F91FF9008958C01E3CF44E050E0BC0153
:104150008FE090E00C94471E08951F93CF93DF9358
:10416000182F80E591E00E940983812F0E9433205F
:10417000EC01812F0E94311F873121F08C3111F029
:10418000D0E0C0E0CE01DF91CF911F910895FC01F6
:104190008485883010F40C94AD2090E080E0089580
:1041A000CF92DF92EF92FF921F93CF93DF93182F5E
:1041B0007B01EA014130584010F0C0E0D8E080E5D2
:1041C00091E00E940983812F0E9433206C01812F8E
:1041D0000E94311F873111F08C3121F5CC16DD069C
:1041E00070F380E591E00E9409839E01A70170E0D1
:1041F00060E0812F0E94B01F60E270E0812F0E947A
:104200008F1F62E070E0812F0E942A1E84FD0DC086
:10421000812F0E94311F8823B9F080E591E00E9430
:104220000983EFCFD0E0C0E0DCCF40E162E070E096
:10423000812F0E94721FCE01DF91CF911F91FF90BD
:10424000EF90DF90CF900895D0E0C0E0F4CF0F93CF
:104250001F93CF93DF938C01EA01FC0184858830A2
:1042600048F40E94D020892B39F481E090E0F801D5
:1042700093838283D0E0C0E0CE01DF91CF911F9184
:104280000F910895CF92DF92EF92FF920F931F93B9
:10429000CF93DF938B017A016C0129EBC20ED11C05
:1042A000F6014081EC012A96442349F050E0BC011C
:1042B00067567F4FCE010E942721F6011082A70189
:1042C000B801CE01DF91CF911F910F91FF90EF9038
:1042D000DF90CF900C942721CF93DF93EC01C7544C
:1042E000DF4FE88121E02E0F2883E80FF92FF11D21
:1042F000E756FF4F6083203249F4BC0167567F4F79
:1043000040E250E00A960E942721188281E090E066
:10431000DF91CF9108951F93CF93DF931F92CDB775
:10432000DEB7182F80E591E00E940983812F0E945B
:10433000720C27E0129FF0011124EA50F44F228101
:104340003381377041E050E0BE016F5F7F4F820FD5
:10435000931F0E949F1D89810F90DF91CF911F9124
:104360000895FC01808D883040F4218D328D232BFF
:1043700021F00E948B2190E008958FEF9FEF089528
:10438000CF93DF93FC012485283028F08FEF9FEF37
:10439000DF91CF910895EC010190F081E02D008430
:1043A000F185E02D1995892B89F38C850E948B214D
:1043B00090E0EECF1F93CF93DF93182F87E0189FE5
:1043C000E0011124CA50D44F88819981009761F48B
:1043D00080E591E00E940983812F0E9470202E8148
:1043E000821B910999838883DF91CF911F91089552
:1043F000FC018485883010F40C94DA2190E080E090
:1044000008954F925F927F928F929F92AF92BF9248
:10441000CF92DF92EF92FF920F931F93CF93DF9390
:104420001F921F92CDB7DEB7782E6B014A01A82EDE
:10443000B12C27E0829FC0011124FC01EA50F44F07
:104440007F010081118180E591E00E9409830815B8
:10445000190554F4872D0E947020F70126818C01E4
:10446000021B1109118300830115110519F5872D10
:104470000E94311F843159F0882349F001E010E097
:104480008C3111F410E000E0119501951109C8017B
:104490000F900F90DF91CF911F910F91FF90EF90B0
:1044A000DF90CF90BF90AF909F908F907F905F9064
:1044B0004F900895801691060CF4840187E08A9D40
:1044C000F0018B9DF00D1124EA50F44FE280F3804F
:1044D000C114D10451F12701F7E05F22872D0E941A
:1044E000720C840D951D20914A0C273309F453C09A
:1044F0009801240D351D2130384008F44CC020E0CF
:1045000038E0490184189508A401B6010E949F1D56
:104510002601480C591C6801C818D908872D0E942B
:10452000720CA601B2010E949F1DE00EF11E87E0F1
:104530008A9DF0018B9DF00D1124EA50F44FF38217
:10454000E28220813181201B310B318320838681DF
:10455000800F912F911D8A3F910510F4232BF1F4C8
:1045600087E08A9DF0018B9DF00D1124EA50F44FF5
:104570001682F982EA8222E030E0AE014F5F5F4F9F
:1045800068E270E0872D0E94351F60E470E0872D9F
:104590000E948F1F7CCFA801B601C5CF868377CF3D
:1045A000CF93DF93FC01218D328D2115310529F444
:1045B0008FEF9FEFDF91CF910895EC01808D42172F
:1045C000530708F0A9010E9401221816190684F762
:1045D000298D3A8D281B390B3A8F298FEBCF0F93FA
:1045E0001F93CF93DF931F92CDB7DEB7FC01218DD0
:1045F000328D232B41F48FEF9FEF0F90DF91CF91FE
:104600001F910F9108958C0141E050E0BE016F5F52
:104610007F4FFC01808D0E940122181619065CF75D
:10462000F801818D928D0197928F818F898190E021
:10463000E4CF0F931F93CF93DF9300D000D01F924E
:104640001F92CDB7DEB78C01D80159964D915C9180
:104650005A974115510551F0ED91FC91048CF58D5F
:10466000E02D70E060E0C8011995EECFF801808D73
:104670000E94DA21892BB1F148E050E0BE016F5F62
:104680007F4FD80158968C910E9401221816190666
:10469000F4F4D801509684E0FE01319601900D9219
:1046A0008A95E1F78D8190E0982F88272E81820FDF
:1046B000911DF801958B848B8F81282F30E0322F4C
:1046C00022278885820F932F911D928F818F2896A4
:1046D0000FB6F894DEBF0FBECDBFDF91CF911F9113
:1046E0000F91089590E080E0F2CFCF93DF931F9277
:1046F000CDB7DEB741E050E0BE016F5F7F4FFC01F8
:1047000084850E9401221816190634F4898190E0EC
:104710000F90DF91CF9108958FEF9FEFF9CFFC01BC
:104720008485883010F40C94012290E080E0089594
:10473000CF93C82F80E591E00E94098368E070E084
:104740008C2FCF910C948F1FCF93C82F80E591E0D1
:104750000E94098360E170E08C2FCF910C948F1F31
:10476000CF92DF92EF92FF920F931F93CF93DF933D
:1047700000D000D0CDB7DEB78C016B017A01FC010F
:10478000808D883010F40E94A42380E394E09A8303
:104790008983F60182819381A481B5818B839C8377
:1047A000AD83BE83B701CE0101960E949789F801BF
:1047B000808F8830A0F4F586E486128E118E81E019
:1047C00026960FB6F894DEBF0FBECDBFDF91CF9116
:1047D0001F910F91FF90EF90DF90CF90089580E0B0
:1047E000EFCFCF93DF93EC01888D883020F40E94C7
:1047F000A42388E0888FDF91CF910895CF93C82FAD
:1048000080E591E00E9409838C2FCF910C94311F99
:10481000EF92FF920F931F93CF93DF937C018091D0
:104820004A0CD4E0833309F0D8E00EE21CE0C0E08B
:10483000F801219131918F01F70184819581281729
:10484000390729F0CF5FDC13F3CF80E006C08C2F4F
:104850000E94FE238431B1F781E0DF91CF911F9157
:104860000F91FF90EF9008959F92AF92BF92CF92D9
:10487000DF92EF92FF920F931F93CF93DF93EC01A0
:104880007B0180914A0C811121C01B821A8288EE23
:1048900093E0A0E0B0E08C839D83AE83BF8384EE81
:1048A00093E09983888388E08C8788EE93E09E87E5
:1048B0008D87CE01DF91CF911F910F91FF90EF90E7
:1048C000DF90CF90BF90AF909F90089534E0932EEB
:1048D000833311F028E0922E8EE2C82E8CE0D82E81
:1048E00010E098E0B92EA12CD6012D913D916D01DB
:1048F000F701848195812817390791F4812F0E944F
:10490000FE23082F873111F08C3139F5812F0E9459
:10491000DA21892B59F50C3119F4812F0E94982343
:104920001F5F9112E1CFA11008C0D701ED91FC915A
:104930000084F185E02DC70119951B821A8288EE4B
:1049400093E0A0E0B0E08C839D83AE83BF8384EED0
:1049500093E099838883BC86A8CF843149F0811184
:10496000DFCFF601329711821082DACFB12ED8CF85
:10497000AA24A394D5CF8F929F92AF92BF92CF9249
:10498000DF92EF92FF920F931F93CF93DF93CDB7F8
:10499000DEB72F970FB6F894DEBF0FBECDBF5C0118
:1049A0004B017A0180914A0C8823C9F104E08333DA
:1049B00009F008E0B501CE0101960E9434248EE290
:1049C000C82E8CE0D82E10E0F601219131916F01B4
:1049D000F501848195812817390751F4812F0E94B0
:1049E000FE23873129F4A701B401812F0E94D02032
:1049F0001F5F0113E9CFC7012F960FB6F894DEBFF2
:104A00000FBECDBFDF91CF911F910F91FF90EF901F
:104A1000DF90CF90BF90AF909F908F900895F12C32
:104A2000E12CE9CFCF93DF93EC018C858830D0F473
:104A30000E94FE23843189F0882379F0883169F05F
:104A400021E08C3159F4E881F9810084F185E02D71
:104A5000CE01199521E0892B09F420E0822FDF9106
:104A6000CF91089580E0FBCFCF92DF92EF92FF923B
:104A7000CF93DF93EC018C85883068F40E949823F3
:104A80000E94830E6B017C018C850E94FE238111A4
:104A900009C088E08C87DF91CF91FF90EF90DF9085
:104AA000CF90089561E070E080E090E00E94500EA9
:104AB0000E94830EAB01BC014C195D096E097F0990
:104AC0008D859E85B0E0A0E0481759076A077B07EF
:104AD000D8F28C850E94A423DCCFCF93DF93EC0126
:104AE0008C85883060F40E94FE23873111F08C3170
:104AF00031F48C850E94AD208115984088F3DF91B8
:104B0000CF910895CF92DF92EF92FF920F931F9370
:104B1000CF93DF93CDB7DEB7AF970FB6F894DEBF74
:104B20000FBECDBF8C016B017A0180E394E09A83C4
:104B300089831B821C821D821E821C861B8648EE76
:104B400053E060E070E04D875E876F87788B2AEBDB
:104B500033E03A872987988F8F8B198E1A8E1B8E98
:104B60001C8E28E029A39BA78AA71CA61DA61EA60B
:104B70001FA6D8011C968C91883060F40E94FE23F9
:104B8000882321F0F80184850E94982388E0D801C9
:104B90001C968C938091451090914610A0914710DF
:104BA000B09148108EA39FA3A8A7B9A78B839C831D
:104BB000AD83BE8318861F82AE01465D5F4FB6018E
:104BC000CE0101960E94A7860097C1F0D801ED9111
:104BD000FC910684F785E02D80E394E09DA38CA3EF
:104BE0008CA59DA5AEA5BFA58EA39FA3A8A7B9A779
:104BF000A701BE016C5D7F4FC8011995AF960FB636
:104C0000F894DEBF0FBECDBFDF91CF911F910F9102
:104C1000FF90EF90DF90CF9008958F929F92AF9288
:104C2000BF92CF92DF92EF92FF920F931F93CF9399
:104C3000DF9300D000D000D01F92CDB7DEB79091A7
:104C40004A0C911115C018E0812F2A960FB6F894DE
:104C5000DEBF0FBECDBFDF91CF911F910F91FF90AF
:104C6000EF90DF90CF90BF90AF909F908F9008957E
:104C700028E0F22E933311F494E0F92E6B01082F03
:104C800080E591E00E9409839E012F5F3F4F59010B
:104C9000490110E0812F0E94311FF40181934F01DF
:104CA0008823C1F01F5FF112F5CFF12CF50191912E
:104CB0005F019D3149F0983139F09A51923020F0DE
:104CC000F3941F11F3CFBFCF60E170E08F2D0E94EE
:104CD0008F1F1F2DE12EF12CF701EE0FFF1FE25D5C
:104CE000F34F1182108283EE93E00197F1F7402F8A
:104CF00070E060E0812F0E94721F4FEF62E070E071
:104D0000812F0E94721FB601CD2889F480919002F4
:104D10009091910201968115F0EC9F0798F1909384
:104D20009102809390026091900270919102812F84
:104D30000E945C1F61E070E0812F0E948F1F27E0BE
:104D40002E9DC0012F9D900D11249C012A50344F9F
:104D50007901F9011182108222E030E0AE01475F53
:104D60005F4F68E270E0812F0E949F1F89859A85BE
:104D7000982789279827F7019383828316821582C3
:104D8000148262CF80E090ECCACF0F931F93CF9331
:104D9000DF93EC018B01888D883010F40E94A423EE
:104DA000B80182E00E940D26888F883050F41D875C
:104DB0000C871A8E198E81E0DF91CF911F910F9190
:104DC000089580E0F9CF9F92AF92BF92CF92DF9289
:104DD000EF92FF920F931F93CF93DF938C015B01B0
:104DE000942EE52EFC01C688D788F08C80E591E0F2
:104DF0000E9409838F2D0E943320C92DDE2D8C1730
:104E00009D0708F4EC019E01A501B6018F2D0E94BB
:104E1000B01FF801868997898C0F9D1F978B868B11
:104E2000CE01DF91CF911F910F91FF90EF90DF9016
:104E3000CF90BF90AF909F900895CF93FC01C08D0D
:104E400080E591E00E94098360E270E08C2F0E946F
:104E50008F1F62E070E08C2F0E942A1E84FD16C016
:104E600062E070E08C2F0E942A1E83FF0AC048E196
:104E700062E070E08C2F0E94721F80E090E0CF9182
:104E8000089580E591E00E940983E3CF40E162E06C
:104E900070E08C2F0E94721F81E0F0CFFF920F9381
:104EA0001F93CF93DF93EB01FC01178A168A2A81A7
:104EB000211109C02B81211106C02C81211103C0B1
:104EC0002D81222301F141155105E9F08A01FC01F0
:104ED000F08C80E591E00E940983AE014E5F5F4F48
:104EE00024E030E06CE070E08F2D0E94351FB801A7
:104EF0008F2D0E94461F81E090E0DF91CF911F919E
:104F00000F91FF90089580E0F7CF7F928F929F924C
:104F1000AF92BF92CF92DF92EF92FF920F931F93C7
:104F2000CF93DF93CDB7DEB7A6970FB6F894DEBF69
:104F30000FBECDBF8C01762E942E852E20E2A22EA0
:104F4000CE0101967C01DC01EA2D1D92EA95E9F77C
:104F50006801F3E4CF0ED11C80E394E09AA389A307
:104F60008FEF8BA38CA38DA38EA343E450E0BE01EF
:104F70006F5D7F4FC6010E944E27019609F4BFC0A6
:104F800081E089838A8386E0B82EBB821C82D801A7
:104F900014966D917D918D919C9117970E94ADB65D
:104FA0006D837E838F83988789869A8680E890E0D8
:104FB0009C878B874CE150E0B701C6010E94E32635
:104FC000FE0137968AE1DF011D928A95E9F74801D3
:104FD000B8E08B0E911CF401D70101900D92BA94A8
:104FE000E1F740E150E0B701C6010E94E326F70176
:104FF0001192AA94E9F796E0A92EB12C40E250E074
:10500000B701C6010E94E326F1E0AF1AB108B1F77B
:1050100083E6898392E89A8393E59B838C8385E377
:105020008D8381E08E837F829DE3988797E09987C7
:105030008A8786E0F401DE011B9601900D928A9525
:10504000E1F78CE0898B8A8B62E374E0CE014396B2
:105050000E941EB9D8011B966C91CE0149960E9400
:105060008589F8016485CE014B960E948589D80117
:105070001D966C91CE014D960E9485894EE150E0BF
:10508000B701C6010E94E326B3E07B121EC082E393
:10509000898384E08A83F80196859B8397859C8326
:1050A00090899D8391899E8396E39F838887828DD3
:1050B0008987838D8A87848D8B87858D8C874CE04B
:1050C00050E0B701C6010E94E32687E3898386E0AA
:1050D0008A8391E09B8393E09C838D838FE08E8312
:1050E0008AE38F838BE388878FEF898749E050E0DD
:1050F000B701C6010E94E326C6010E941D27A6969D
:105100000FB6F894DEBF0FBECDBFDF91CF911F91D8
:105110000F91FF90EF90DF90CF90BF90AF909F9056
:105120008F907F9008950F931F93CF938C01FC0174
:105130006481758181E20E940D26C82F8830F8F4C1
:1051400080E591E00E9409838C2F0E94311F8331FA
:1051500031F08C2FCF911F910F910C94982362E026
:1051600070E08C2F0E948F1FF80184819581EC2FB5
:10517000F0E0EE0FFF1FE25DF34F91838083CF914C
:105180001F910F9108950F931F93CF93DF931F9259
:105190001F92CDB7DEB7FC0124852830E0F48C01E6
:1051A00080E591E00E94098322E030E0AE014F5F8C
:1051B0005F4F60E170E0F80184850E949F1F898144
:1051C0009A819827892798270F900F90DF91CF9188
:1051D0001F910F91089590E080E0F6CF0F931F93F9
:1051E000CF93DF931F921F92CDB7DEB7FC012485CA
:1051F0002830E0F48C0180E591E00E94098322E0F0
:1052000030E0AE014F5F5F4F64E070E0F8018485ED
:105210000E949F1F89819A819827892798270F903C
:105220000F90DF91CF911F910F91089590E080E052
:10523000F6CFCF92DF92EF92FF921F93CF93DF933F
:10524000EC017B016A018C85883048F40E94FE23C2
:10525000882319F08C850E94982388E08C87F701B9
:1052600082819381A481B5810097A105B10551F494
:1052700090E080E0DF91CF911F91FF90EF90DF9061
:10528000CF9008958F3F9F4FAF4FBF4F89F370E08E
:1052900060E081E20E940D26182F8C87883040F74D
:1052A00080E591E00E940983A7014E5F5F4F24E0F3
:1052B00030E06CE070E0812F0E94351FB601812F35
:1052C0000E94461F64E070E0812F0E948F1F0E94A1
:1052D000830E6B017C018C850E94FE23873111F1C6
:1052E0008C3101F1882321F20E94830EAB01BC01B5
:1052F0004C195D096E097F098D859E85B0E0A0E09F
:1053000084179507A607B70738F061E070E080E0E2
:1053100090E00E94500EDFCF8C850E94A42388E08D
:105320008C87A6CF81E090E0A5CFCF93DF93EC01EF
:1053300080E394E0998388831A821B821C821D82F9
:1053400080E591E00E940983BE016E5F7F4F44E0DB
:1053500050E08FE090E00E949F1DCE01DF91CF9141
:1053600008959F92AF92BF92CF92DF92EF92FF92F9
:105370000F931F93CF93DF935C017B018B01D0E0F0
:10538000C0E0F80191908F016501CC0EDD1EC601D1
:105390000E94E9B4981621F0692DC6010E94F1B46B
:1053A0002196C533F1E0DF0761F7C701DF91CF91A7
:1053B0001F910F91FF90EF90DF90CF90BF90AF9033
:1053C0009F90089581E08093EF028091F0028823FE
:1053D00041F088E08093781360E08DE693E10C94CF
:1053E000FE0E08958091F0028823F9F08091EF027B
:1053F0008823D9F081E00E94FC838BE39FE1019731
:10540000F1F760E080E00E940D8461EC76E08DE6CB
:1054100093E10E94608E61E080E00E940D8461EB68
:1054200076E08DE693E10C94608E08950F931F93C0
:10543000CF93DF932091F002222309F45CC02091E6
:10544000EF02222309F457C0EA018C016F3F7F4F1E
:10545000F1F461E080E00E940D84B8018DE693E1F3
:105460000E94408E60EA76E08DE693E10E94608EB5
:1054700061E0F80184810E940D84BE01DD0F880B7C
:10548000990BDF91CF911F910F910C94500E0E94B8
:10549000830EAB01BC0180916D0990916E09A091C2
:1054A0006F09B09170098C599F4FAF4FBF4F841750
:1054B0009507A607B707F8F461E080E00E940D8425
:1054C000B8018DE693E10E94408E6FE876E08DE6AC
:1054D00093E10E94608E61E0F80184810E940D8456
:1054E0000E94830E60936D0970936E0980936F091B
:1054F00090937009C2CFDF91CF911F910F910895C2
:105500008F929F92AF92BF92CF92DF92EF92FF92D3
:105510000F931F93CF93DF938C01862F0B301105D0
:1055200009F09FC09091F612992309F0F89462E176
:105530000E945685EC018091F612882309F0789438
:10554000209701F180E090ECA9E7B4EC8093E91298
:105550009093EA12A093EB12B093EC128093ED12A9
:105560009093EE12A093EF12B093F012CE3F8FEF14
:10557000D80709F4A9C0CF3FDC0709F462C0CCEF1B
:10558000DFEF30C1C091F112E090F2126E2D70E0A9
:1055900090E080E00E94CCB32DEC3CEC4CEC5DE361
:1055A0000E942BB44B015C016C2F70E090E080E016
:1055B0000E94CCB39B01AC01C501B4010E9473B53C
:1055C0006093E9127093EA128093EB129093EC12BD
:1055D000D091F312F090F4126D2F6F7770E090E09D
:1055E00080E00E94CCB34B015C016F2D70E090E035
:1055F00080E00E94CCB32DEC3CEC4CEC5DE30E94CF
:105600002BB49B01AC01C501B4010E9473B5D7FD59
:1056100026C06093ED127093EE128093EF12909378
:10562000F012CE0DCD0FCF0D81E090E02091F5125C
:10563000C21302C090E080E0892B09F493C0CFEF41
:10564000DFEFCE01DF91CF911F910F91FF90EF908F
:10565000DF90CF90BF90AF909F908F90089590581B
:10566000D8CFCFEFDFEF0631110509F0BBC0909125
:10567000F612992309F0F89461E00E945685EC0136
:105680008091F612882309F07894209701F180E048
:1056900090ECA9E7B4EC8093E9129093EA12A093FE
:1056A000EB12B093EC128093ED129093EE12A09354
:1056B000EF12B093F012CF3FDC0719F2209709F4F4
:1056C00051C0229609F05BCFCEEFDFEF8BC0C091C7
:1056D000F212D091F1126091F1127091F2127627CC
:1056E0006727762790E080E00E94CAB32DEC3CEC5F
:1056F0004CEC5DE30E942BB46093E9127093EA12C4
:105700008093EB129093EC12E090F412F090F3126D
:105710006F2D6F77762F6E2D90E080E00E94CAB3D8
:105720002DEC3CEC4CEC5DE30E942BB4F7FC18C074
:105730006093ED127093EE128093EF129093F0123B
:105740008C2F8D0F8E0D8F0DC1E0D0E09091F51252
:10575000891302C0D0E0C0E0D195C195D109ABCF8B
:105760009058E6CFC090E912D090EA12E090EB1288
:10577000F090EC1220E030E048EC52E4C701B601B2
:105780000E9487B6D0E0C0E0181614F4CBEFDFEF2C
:1057900020E030E0A901C701B6010E94C5B387FF30
:1057A00002C0CAEFDFEFC090ED12D090EE12E09091
:1057B000EF12F090F01220E030E048EC52ECC7011C
:1057C000B6010E94C5B387FF02C0C9EFDFEF20E03A
:1057D00030E040EF52E4C701B6010E9487B61816C8
:1057E0000CF483C00C30110509F02BCF81E08093BD
:1057F0008F0E8CE58093B10E1092900E1092B20E27
:1058000060E08EEE9FE00E94E10B81E00E940C833D
:105810000E942B0E6B017C018091890E811168C062
:1058200081E08093890E8093880E9FEF9093870E7E
:105830001092860E94E09093850E8093640E809172
:10584000640E886B8093640E8091630E813009F042
:1058500028C11092630E0E942B0E6B017C01809177
:10586000640E8093BB0080918B0E90918C0EA09162
:105870008D0EB0918E0E892B8A2B8B2BA1F00E945E
:105880002B0E00918B0E10918C0E20918D0E30916D
:105890008E0E6C197D098E099F09061717072807B8
:1058A000390708F446C08091BC0083FDD8CF85EC51
:1058B0008093BC000E942B0E6B017C018091890EAD
:1058C000813009F4F0C08091860E853008F00DC15A
:1058D0008091860EA5E6BEE0EDE7FAE090E098172D
:1058E00069F12D9121939F5FFACFC8EFDFEF7ACF57
:1058F00080918B0E90918C0EA0918D0EB0918E0E9A
:10590000892B8A2B8B2B09F487CF0E942B0E0091B9
:105910008B0E10918C0E20918D0E30918E0E6C1985
:105920007D098E099F09061717072807390708F010
:1059300073CF80918A0E0E947C1080E01092430CFD
:105940008093420C082F10E0CEEFDFEF882309F49C
:1059500078CECDEFDFEF053011050CF472CEC0E646
:10596000D9E08EEE9FE00E949A0B88872196CE01A7
:105970008056994080179107A4F3C091680900915F
:105980006909602F70E090E080E00E94CCB32DECBC
:105990003CEC4CEC5DE30E942BB46B017C016C2F62
:1059A00070E090E080E00E94CCB39B01AC01C701A5
:1059B000B6010E9473B56B017C01C0926009D09260
:1059C0006109E0926209F0926309D0916A0910912D
:1059D0006B096D2F6F7770E090E080E00E94CCB390
:1059E0004B015C01612F70E090E080E00E94CCB33D
:1059F0002DEC3CEC4CEC5DE30E942BB49B01AC0124
:105A0000C501B4010E9473B5D7FD71C060936409EC
:105A1000709365098093660990936709C00FCD0F55
:105A2000C10F80916C09C8130ACE20E030E048EC29
:105A300052E4C701B6010E9487B6D0E0C0E0181654
:105A400014F4CBEFDFEF20E030E040EA50E4C70190
:105A5000B6010E94C5B387FF02C0CAEFDFEFC09056
:105A60006409D0906509E0906609F090670920E02C
:105A700030E040EF51ECC701B6010E94C5B387FF8B
:105A800002C0C9EFDFEF20E030E040EF52E4C70191
:105A9000B6010E9487B618160CF0D3CDC8EFDFEF21
:105AA000D0CD85EE05CF80918B0E90918C0EA0917C
:105AB0008D0EB0918E0E892B8A2B8B2B09F4FECE86
:105AC0000E942B0E00918B0E10918C0E20918D0E4A
:105AD00030918E0E6C197D098E099F0906171707E4
:105AE0002807390708F0EACE24CF85E0F3CE905896
:105AF0008DCFCF93DF93FB0122813381DC0113969D
:105B00003C932E9312974481558166817781149638
:105B10004D935D936D937C93179740855185628576
:105B2000738518964D935D936D937C931B971C968C
:105B3000EF012C969C01275E3F4F49914D93A21790
:105B4000B307D9F7218D328DFC01328F218FDF9180
:105B5000CF910895DF92EF92FF920F931F93CF930F
:105B6000DF93D82EC5E5DCE07E0101E010E0F7010F
:105B70008081F2E0EF0EF11C61E00E94FA0D90E0EE
:105B800080E00130110531F48091E812881F8827E8
:105B9000881F90E0880F991FFC01E55AF34F608140
:105BA000F701329780810E94CC0D64EF71E080E0B4
:105BB00090E00E94500E0F5F1F4F04301105B9F6A0
:105BC000DD2009F454C0EE24E394F12C81E0E816C2
:105BD000F10409F046C08091E8128095881F88275B
:105BE000881F90E08E01880F991FFC01E55AF34F42
:105BF000608188810E94CC0D68EE73E080E090E0C7
:105C00000E94500E91E0E916F10471F58091E812BE
:105C1000881F8827881F90E02296880F991FFC0113
:105C2000E55AF34F6081F80180810E94CC0D68EE47
:105C300073E080E090E00E94500EFFEFEF1AFF0A41
:105C400084E0E816F10411F668EE73E080E090E07D
:105C5000DF91CF911F910F91FF90EF90DF900C9407
:105C6000500E81E090E0BECF90E080E0D5CFDF9194
:105C7000CF911F910F91FF90EF90DF9008950F93B8
:105C80001F93CF93DF938C01EB01FE01649121966A
:105C9000662349F0D801ED91FC910190F081E02D4F
:105CA000C8011995F2CFDF91CF911F910F910895FF
:105CB000EF92FF920F931F93CF93DF93EC017B0141
:105CC0008A0164E374E00E943F2E6DE174E0CE012E
:105CD0000E943F2E6EEE73E0CE010E943F2EB70170
:105CE000CE010E94388E69E478E0CE010E94388EA1
:105CF0000115110521F0B801CE010E94388E69E42A
:105D000078E0CE01DF91CF911F910F91FF90EF903E
:105D10000C94388ECF93DF93EC0163ED73E00E9417
:105D20003F2E6DE174E0CE010E943F2E65EA73E0E4
:105D3000CE01DF91CF910C943F2ECF93DF93EC01F6
:105D4000FB01248135810E94408DCE01DF91CF91EE
:105D50000895EF92FF920F931F93CF93DF9300D09C
:105D600000D0CDB7DEB78C017B016DE574E00E94F9
:105D70002B8D8AE0E816F1042CF466E276E0C80187
:105D80000E94068CB701CE0101960E94878ABE014F
:105D90006F5F7F4FC8010E94108CCE0101960E9458
:105DA0008C8CC80126960FB6F894DEBF0FBECDBF0F
:105DB000DF91CF911F910F91FF90EF900895CF92B7
:105DC000DF92EF92FF920F931F93CF93DF93CDB7A4
:105DD000DEB7C455D1090FB6F894DEBF0FBECDBFF4
:105DE00065965FAF4EAF65972091D90B3091DA0B76
:105DF0002F5F3F4F3093DA0B2093D90B2091F50B97
:105E00002111C1C08B016C0181E08093F50B1092D0
:105E1000DA0B1092D90B6DE574E0CE01895B9F4FD0
:105E20000E942B8D6DE574E0CE01835B9F4F0E9435
:105E30002B8D50E040E069E374E0C6010E94582ECB
:105E40000130110509F08EC06DE574E08EE791E137
:105E50000E947D8A6DE574E08AE591E10E947D8A69
:105E60006596EEADFFAD65978081882309F474C017
:105E700000E210E09E012F5F3F4F40E250E0BE0184
:105E80006F5D7F4FCE018D5A9F4F0E947E84049795
:105E900039F3BE016F5D7F4FCE018F5B9F4F0E9434
:105EA0002B8DBE016F5B7F4FCE01895B9F4F0E94A0
:105EB000538CCE018F5B9F4F0E948C8CBE016F5F15
:105EC0007F4FCE018F5B9F4F0E942B8DBE016F5B7A
:105ED0007F4FCE01835B9F4F0E94538CCE018F5B1F
:105EE0009F4F0E948C8C2D968EAD9FAD2D97029763
:105EF000029730F462E574E08AE591E10E947D8AC0
:105F0000BE01695B7F4F8EE791E10E94108C639622
:105F10008EAD9FAD6397892B09F4A2CF6DEB75E031
:105F2000CE018F5B9F4F0E942B8DBE01635B7F4F25
:105F3000CE018F5B9F4F0E94B58B6AEB75E00E948C
:105F40009F8BBC018EE791E10E94108CCE018F5B8C
:105F50009F4F0E948C8C84CF6EE771E18AE591E1BE
:105F60000E94108C1092F50BCE01835B9F4F0E9414
:105F70008C8CCE01895B9F4F0E948C8C0FB6F8945D
:105F8000DEBF0FBECDBFCC5ADF4F0FB6F894DEBFD9
:105F90000FBECDBFDF91CF911F910F91FF90EF907A
:105FA000DF90CF9008950F931F93CF93DF9300D08E
:105FB00000D0CDB7DEB72091D60B2223A9F08C01FB
:105FC00065E876E0CE0101960E942B8DB801CE01E6
:105FD00001960E94B58BBC0181E59FE00E944E8E28
:105FE000CE0101960E948C8C26960FB6F894DEBFE7
:105FF0000FBECDBFDF91CF911F910F9108950F93E9
:106000001F93CF93DF93CDB7DEB72C970FB6F894DD
:10601000DEBF0FBECDBF8C010E94AA0FBC01C8011C
:106020000E94A92E0E94A20FBC01CE0107960E94D9
:10603000A92E6FE476E0CE0101960E942B8DBE0161
:10604000695F7F4FCE0101960E94B58BBC01C801EC
:106050000E94108CCE0101960E948C8CCE01079676
:106060000E948C8C6AEB75E0C8010E94068C0E942D
:106070009A0FBC01CE0101960E94A92EBE016F5F4E
:106080007F4FC8010E94108CCE0101960E948C8C1B
:1060900069E574E0C8010E94068C0E94920FBC0161
:1060A000CE0101960E94A92EBE016F5F7F4FC801ED
:1060B0000E94108CCE0101960E948C8C69E574E0E0
:1060C000C8010E94068C0E94880FBC01CE01019677
:1060D0000E94A92EBE016F5F7F4FC8010E94108CE5
:1060E000CE0101960E948C8CC8012C960FB6F894B4
:1060F000DEBF0FBECDBFDF91CF911F910F910895ED
:106100000F931F93CF93DF93CDB7DEB72C970FB6C6
:10611000F894DEBF0FBECDBF8C010E94AA0FBC0158
:10612000C8010E94A92E0E94A20FBC01CE010796B1
:106130000E94A92E6FE476E0CE0101960E942B8D7D
:10614000BE01695F7F4FCE0101960E94B58BBC01F5
:10615000C8010E94108CCE0101960E948C8CCE0149
:1061600007960E948C8C0E94420F0E94680A6091E0
:10617000B60B70E0CE0107960E94A92E6FE476E080
:10618000CE0101960E942B8DBE01695F7F4FCE012B
:1061900001960E94B58BBC01C8010E94108CCE01F3
:1061A00001960E948C8CCE0107960E948C8C6AEB23
:1061B00075E0C8010E94068C0E949A0FBC01CE01B6
:1061C00001960E94A92EBE016F5F7F4FC8010E94F9
:1061D000108CCE0101960E948C8C69E574E0C80198
:1061E0000E94068C0E94920FBC01CE0101960E9473
:1061F000A92EBE016F5F7F4FC8010E94108CCE0197
:1062000001960E948C8C69E574E0C8010E94068C9E
:106210000E94880FBC01CE0101960E94A92EBE01EA
:106220006F5F7F4FC8010E94108CCE0101960E94C3
:106230008C8CC8012C960FB6F894DEBF0FBECDBF74
:10624000DF91CF911F910F910895CF92DF92EF923E
:10625000FF920F931F93CF93DF9300D000D0CDB761
:10626000DEB77C01FB01848195818A01081B190B33
:10627000101611069CF0C7010E94108DC7012696CA
:106280000FB6F894DEBF0FBECDBFDF91CF911F9147
:106290000F91FF90EF90DF90CF900895CE0101967F
:1062A0000E94228DCC24C394D12C6AEB75E0CE01E0
:1062B00001960E94068CFFEFCF1ADF0A0C151D0510
:1062C000A4F7BE016F5F7F4FC7010E94108DCE0102
:1062D00001960E948C8CD2CF0F931F93CF93DF93A4
:1062E00000D000D0CDB7DEB78C018091670A88233B
:1062F00029F0B80184EB9EE00E944E8E6EE170E0C2
:1063000080E090E00E94500EB80181E59FE00E947D
:106310004E8E8091460C882311F16AE070E080E097
:1063200090E00E94500EB801CE0101960E94228D8D
:10633000BE016F5F7F4F81E593E10E94408E6AE46A
:1063400078E081E593E10E94388ECE0101960E94AB
:106350008C8C64E170E080E090E00E94500E269604
:106360000FB6F894DEBF0FBECDBFDF91CF911F9166
:106370000F9108950F931F93CF93DF9300D000D018
:10638000CDB7DEB7FC0124813581232B49F18C0187
:106390008091670A882329F0BF0184EB9EE00E9468
:1063A000408E6EE170E080E090E00E94500EB801F7
:1063B00081E59FE00E94408E8091460C882381F009
:1063C000B801CE0101960E94228DBE016F5F7F4F02
:1063D00081E593E10E94408ECE0101960E948C8C53
:1063E00026960FB6F894DEBF0FBECDBFDF91CF91DA
:1063F0001F910F9108952F923F924F925F926F924B
:106400007F928F929F92AF92BF92CF92DF92EF9244
:10641000FF920F931F93CF93DF93CDB7DEB7C25890
:10642000D1090FB6F894DEBF0FBECDBF6C015B0182
:1064300088EE482E83E0582E612C712C02E114E086
:106440009BE5892E912C8C0E9D1E8CE0880E911C54
:106450001B019FEF291A390AD6015996ED90FC903D
:10646000F7018581823008F493C082859385A485E5
:10647000B5858F719927AA27BB27892B8A2B8B2B50
:1064800009F086C040E250E0BE016F5F7F4FC70158
:106490000E949917803209F07BC08981882309F412
:1064A00077C0853E79F38E3269F38C8583FDEACF20
:1064B00022961FAE1EAE229782E993E09FAF8EAF69
:1064C00024961FAE2497BE016F5F7F4FE0E080E00F
:1064D0004EE2DB019D91BD019032A1F0883049F47C
:1064E00026E730E02C0F3D1F2E0F311DD9014C93B4
:1064F000EF5F26E730E02C0F3D1F2E0F311DD90135
:106500009C93EF5F8F5F8B3021F786E790E08C0FD5
:106510009D1F8E0F911DFC011082D60159966D9121
:106520007C9121E0AE014A585F4FCE01CE960E9489
:106530002819882369F1BE01625C7F4FCE018196E4
:106540000E94F21CAE014A585F4FBE016F5D7F4F43
:10655000CE01855A9F4F0E94601DCE01855A9F4FE4
:106560000E94421D882309F4ACC0F12CFA141B04CC
:106570002CF569E0CE0101960E94F78CCE010196C0
:106580000E94BA31CE0101960E948C8CF394EECF1A
:106590006F961FAE1EAE6F97A3964CAE5DAE6EAEFD
:1065A0007FAEA3976D961FAF0EAF6D97E6961FAEA9
:1065B0001EAEE697A8961FAEA897CFCFB401CE0126
:1065C00001960E942B8DCE0101960E94BA31CE0118
:1065D00001960E948C8CE696EEADFFADE697309763
:1065E00009F447C08581823008F443C066E874E04E
:1065F000CE0101960E942B8DCE0101960E946C3136
:10660000CE0101960E948C8C6F968EAD9FAD6F97D8
:106610009C838B83A3968CAD9DADAEADBFADA39790
:106620008D839E83AF83B887A7968CAD9DADAEADAD
:10663000BFADA79789879A87AB87BC871A830983E1
:106640008DE0F401DE011D9601900D928A95E1F72F
:10665000E6968EAD9FADE6979B8F8A8FB101CE01F6
:1066600001960E94FB31CE01855A9F4F0E944E1D1C
:10667000F3CE6BE574E0CE0101960E942B8DCE0126
:1066800001960E94BA31CE0101960E948C8CE6964A
:10669000EEADFFADE69740E050E0BA01309721F053
:1066A0004389548965897689CE0101960E94B38A0F
:1066B000CE0101960E946C31CE0101960E948C8C15
:1066C000D2CFCE57DF4F0FB6F894DEBF0FBECDBF8F
:1066D000DF91CF911F910F91FF90EF90DF90CF90BE
:1066E000BF90AF909F908F907F906F905F904F90F2
:1066F0003F902F900895DF92EF92FF920F931F9398
:10670000CF93DF93CDB7DEB762970FB6F894DEBFB5
:106710000FBECDBF8C01109271096DE574E0CE0102
:106720000D960E942B8DFF24F39481E59FE00E943B
:10673000C00920917109181619067CF5211133C082
:1067400081E59FE00E949E098A3009F04DC0898949
:106750009A89892B09F450C0F09271096EE574E0B2
:10676000CE0101960E942B8DBE01635F7F4FCE014B
:1067700001960E94B58BBC01CE0107960E94228D26
:10678000CE0107960E94D32FCE0107960E948C8CD3
:10679000CE0101960E948C8C2FC0F12CE12CDD24BF
:1067A000D394222381F189899A8920917109211139
:1067B0009DC0009709F09AC06DE574E0C8010E9481
:1067C0002B8DCE010D960E948C8CC80162960FB65F
:1067D000F894DEBF0FBECDBFDF91CF911F910F9117
:1067E000FF90EF90DF9008958D3009F4B0CF682FBF
:1067F000CE010D960E94F28B6AE070E080E090E09E
:106800000E94500E92CF84EB9EE00E94C0091816A1
:10681000190614F584EB9EE00E949E098A30A9F0C7
:106820008D3099F09091710991110FC0682FCE01B0
:106830000D960E94F28B8FEFE81AF80A65E070E07F
:1068400080E090E00E94500EDECF89899A89892BE2
:10685000A9F3D0927109F2CF64E170E080E090E09A
:106860000E94500EEF2809F49ECF89899A89892BBE
:1068700009F499CF8091D60B882389F165E876E0F9
:10688000CE0101960E942B8DBE016F5F7F4FCE011E
:106890000D960E94848BF82ECE0101960E948C8C5E
:1068A000F1101DC067E674E0CE0101960E942B8DA9
:1068B000CE0101960E94BA31CE0101960E948C8CC5
:1068C000BE01635F7F4FCE0101960E94228DCE01F3
:1068D00001960E946C31CE0101960E948C8C64E17D
:1068E00070E080E090E00E94500E5DCF019709F0CB
:1068F00045C06DE275E0CE0107960E942B8DBE016A
:10690000695F7F4FCE010D960E94848BF12C81111F
:1069100015C06EE674E0CE0101960E942B8DBE017B
:106920006F5F7F4FCE010D960E94848BFF24F394FE
:106930008111F12CCE0101960E948C8CCE0107961C
:106940000E948C8CFF20A1F050E040E0BE01635F0C
:106950007F4FCE0101960E949D2EBE016F5F7F4F3B
:1069600081E291E10E94538CCE0101960E948C8CB1
:1069700064E170E080E090E00E94500EBE01635F31
:106980007F4FC8010E94108D1CCF0F931F93CF9390
:10699000DF93CDB7DEB72C970FB6F894DEBF0FBEEE
:1069A000CDBF2C893D89FE017496A3E5BCE090E043
:1069B00080E032962817390734F0408151814D9399
:1069C0005D930196F6CFCE5BDE4F88819981C254EC
:1069D000D140281739070CF037C2DC01AA0FBB1FC2
:1069E000AD5AB34F880F991FFC01EF5AF34F8081C6
:1069F000918101968D939C938C8D9D8D90935C0CD1
:106A000080935B0C8E8D9F8D90935E0C80935D0CBC
:106A1000AD968FADAD97BE0164597F4F8F3209F0AF
:106A20001CC2CE0107960E942B8D60E774E0CE0158
:106A300001960E942B8DBE01695F7F4FCE010196AA
:106A40000E94B58BBC0185E193E10E943C8CCE0194
:106A500001960E948C8CCE0107960E948C8C65E179
:106A600073E1CE0101960E94228DCE0101960E9413
:106A70006C31CE0101960E948C8C66E874E0CE01E8
:106A800001960E942B8DBE016F5F7F4F85E193E1E0
:106A90000E94648B182FCE0101960E948C8C40912D
:106AA000191350911A13112309F4DEC1BA0162506F
:106AB000710985E193E10E94538B682FCE01019605
:106AC0000E94F78CBE016F5F7F4F87EF92E10E94BB
:106AD000538CCE0101960E948C8C64EE71E1CE0144
:106AE00007960E942B8D68E874E0CE0101960E9403
:106AF0002B8DBE01695F7F4FCE0101960E94B58B41
:106B0000BC018FE093E10E943C8CCE0101960E9473
:106B10008C8CCE0107960E948C8C24968FAD249786
:106B20001F928F9323968FAD23971F928F93229658
:106B30008FAD22971F928F9321968FAD21971F9231
:106B40008F938EE894E09F938F9388E69AE09F93CB
:106B50008F930E945CB9CE52DF4F88819981C25DCC
:106B6000D0409093800280937F02BE016C527F4F91
:106B7000CE0101960E942B8DBE016F5F7F4F89E091
:106B800093E10E94538CCE0101960E948C8CBE0131
:106B900061527F4FCE0101960E942B8DBE016F5F27
:106BA0007F4F83E093E10E94538CCE0101960E94B7
:106BB0008C8C40910713509108134250510963E0A7
:106BC00073E1CE0101960E949D2ECE0101960E9496
:106BD000EB8A6C5960939702CE0101960E948C8CCF
:106BE000CC5EDE4F688179818A819B81C451D1401E
:106BF0000E94CCB30FB6F894DEBF0FBECDBF9B0191
:106C0000AC010E948CB6882389F08CE390E0A0E070
:106C1000B0E0CC5EDE4F88839983AA83BB83C451E6
:106C2000D140CD5EDE4F1882C351D140CD5EDE4FE4
:106C30008881C351D140882399F0CC5EDE4F888192
:106C40009981AA81BB81C451D14080936E029093F7
:106C50006F02A0937002B093710281E08093500C98
:106C6000C85EDE4F688179818A819B81C851D1409D
:106C70009B01AC010E948CB6882361F080E090E01B
:106C8000A0E7B2E4C85EDE4F88839983AA83BB8302
:106C9000C851D140C45EDE4F68817981CC51D1406A
:106CA000072E000C880B990B0E94CCB39B01AC0102
:106CB0000E948CB6882341F082E090E0C45EDE4FF3
:106CC00099838883CC51D140CE5BDE4F6881798136
:106CD000C254D140072E000C880B990B0E94CCB3F4
:106CE0009B01AC010E948CB6882341F083E090E0C8
:106CF000CE5BDE4F99838883C254D140C45CDE4FA3
:106D000008811981CC53D140B801012E000C880BA9
:106D1000990B0E94CCB39B01AC010E948CB68111EF
:106D200003C01016110644F080E590E0C45CDE4F0D
:106D300099838883CC53D140C45CDE4F888199818C
:106D4000CC53D14090933F0280933E0288E2FE01F3
:106D5000E551FF4FABE3BAE001900D928A95E1F760
:106D6000CE5CDE4F88819981AA81BB81C253D1401C
:106D70008093290290932A02A0932B02B0932C02B5
:106D8000CA5CDE4F88819981AA81BB81C653D140FC
:106D90008093250290932602A0932702B0932802A5
:106DA000C65CDE4F88819981CA53D14090934902D5
:106DB00080934802CC5BDE4F68817981C454D14016
:106DC000072E000C880B990B0E94CCB39B01AC01E1
:106DD0000E948CB6882341F088E390E0CC5BDE4FC4
:106DE00099838883C454D140CC5BDE4F88819981DC
:106DF000C454D14090938202809381021092670A1A
:106E0000C053DF4F88819981C05DD04097FD03C09A
:106E100081E08093670A6091E61270E090E080E084
:106E20000E94CAB39B01AC010E948CB681111092E2
:106E3000E6122C960FB6F894DEBF0FBECDBFDF91E1
:106E4000CF911F910F9108958091570C9091580CFC
:106E500090935A0C8093590CCFCDCE0107960E9487
:106E60002B8D65E774E0E3CD4150510965E173E195
:106E7000CE0101960E949D2EBE016F5F7F4F87EF6E
:106E800092E10E94538CCE0101960E948C8C65E1A8
:106E900073E1CE0101960E94228D66E874E0CE0176
:106EA00001960E949F8BBC0185E193E10E943C8C7E
:106EB00010CEDF92EF92FF920F931F93CF93DF9349
:106EC000CDB7DEB762970FB6F894DEBF0FBECDBF69
:106ED0002091F002222379F12091EF02222359F12F
:106EE0007A018C016F3F7F4FA1F560E080E00E9446
:106EF0000D84D12CB8018DE693E10E94408E6EE79F
:106F000076E08DE693E10E94608EF801848160E076
:106F10008D0D0E940D840E94830E60935F0E70930E
:106F2000600E8093610E9093620EB701FF0C880B88
:106F3000990B0E94500E62960FB6F894DEBF0FBEFA
:106F4000CDBFDF91CF911F910F91FF90EF90DF9018
:106F5000089560E080E00E940D840E94830E28EE78
:106F600033E040E050E00E940FB5CA01B90120E8CB
:106F700031E541E050E00E9431B5AB01BC0120E0B9
:106F8000CE0101960E94CA8CBE016F5F7F4FCE0179
:106F900007960E94228D69E277E0CE0107960E9453
:106FA0009F8BBC01CE010D960E94228DCE010796CB
:106FB0000E948C8CCE0101960E948C8CBE01635F76
:106FC0007F4F8DE693E10E94408ED98860E08D2D41
:106FD0000E940D84CE010D960E948C8C8BCFCF9396
:106FE000DF9300D000D0CDB7DEB70E94F229CE01EA
:106FF00001960E94FF2F4AE050E06FEF7FEFCE0135
:1070000001960E945937CE0101960E948C8C61E056
:1070100080E00E940D84CE0101960E9495296DE6C4
:1070200073E1CE0101960E94D88D6AE974E08DE685
:1070300093E10E94388E0E94830E6093E30B70935D
:10704000E40B8093E50B9093E60B26960FB6F8942D
:10705000DEBF0FBECDBFDF91CF9108950F931F9379
:10706000CF93DF9300D000D0CDB7DEB78C01CE0137
:1070700001960E94FF2F4AE050E06FEF7FEFCE01B4
:1070800001960E945937CE0101960E948C8CB8015E
:10709000CE0101960E94228D4AE050E06FEF7FEF13
:1070A000CE0101960E94162ACE0101960E948C8C78
:1070B00026960FB6F894DEBF0FBECDBFDF91CF91FD
:1070C0001F910F910895EF92FF920F931F93CF930B
:1070D000DF9300D01F92CDB7DEB78C017B01FB019F
:1070E00084858830A8F080E394E0F8019183808360
:1070F0001282138214821582C8010F900F900F9094
:107100000F90DF91CF911F910F91FF90EF90089515
:1071100080E591E00E94098324E030E0AE014F5FFA
:107120005F4F6CE070E0F70184850E949F1FBE01F5
:107130006F5F7F4FC8010E94968EDECF3F924F92C5
:107140005F926F927F928F929F92AF92BF92CF92F7
:10715000DF92EF92FF920F931F93CF93DF93CDB700
:10716000DEB7EA970FB6F894DEBF0FBECDBF7C0145
:107170002A013B0169010E94830E4B015C018701DA
:107180000D5B1F4FC8010E941923181619069CF0A9
:107190000E94830E681979098A099B0946165706C9
:1071A0006806790608F466C162E370E080E090E06A
:1071B0000E94500EE7CF42E250E0BE016F5F7F4F6A
:1071C000C8010E94D02289818230D1F0312C832DD8
:1071D000EA960FB6F894DEBF0FBECDBFDF91CF9118
:1071E0001F910F91FF90EF90DF90CF90BF90AF90E5
:1071F0009F908F907F906F905F904F903F900895F9
:10720000F801848995898334910501F76D817E8128
:107210008F8198850E94ADB64B015C01F60180829A
:107220009182A282B38246E050E0B701685F7F4F4F
:10723000CE014D960E94DBB8892B41F6F701808183
:107240009181A281B38188169906AA06BB0608F42B
:10725000BDCF84819581A681B78188159905AA053E
:10726000BB0508F4B3CF89899A89AB89BC89868725
:107270009787A08BB18B4EEC50E070E060E0C801C6
:107280000E94D022312CC701829698AB8FA7F701BC
:10729000B696FAABE9AB08969CAB8BAB67019AE16B
:1072A000C90ED11CBD96FEABEDABC701429698AF9F
:1072B0008FABFD97FAAFE9AF4701FEE18F0E911C4E
:1072C000F801818D928D181619060CF080CFC80137
:1072D0000E94EF228333910509F4B2C014F5813086
:1072E000910509F464C044F4892B51F3C8010E944C
:1072F000EF22AC01552775C08330910509F462C0B7
:107300000697A1F7C8010E94EF22B82E44E050E092
:10731000B401C8010E94D022EB2DE450FF0BAF0155
:1073200060C08A33910509F45FC084F58533910507
:10733000B1F1C697D9F6C8010E94EF225C01B601EF
:10734000CE0189960E94968E8BA59CA5ADA5BEA563
:10735000892B8A2B8B2BB1F0EDA9FEA9408051809F
:1073600062807380B601CE0183960E94968E8DA1B5
:107370009EA1AFA1B8A5A501481659066A067B06CD
:1073800009F0B8CF44E050E0B60118C08B33910546
:1073900009F440C08F3F910509F492CFA7CFC801EF
:1073A0000E94EF22C8010E94EF22382E89CFC80127
:1073B0000E94EF2244E050E06FA978ADC8010E941E
:1073C000D0227ECFC8010E94EF22B82E44E050E0C8
:1073D00069AD7AADC8010E94D0228B2D8450990BE3
:1073E000AC0170E060E0EACFC8010E94EF2244E007
:1073F00050E069A97AA9C8010E94D022F70166A1CC
:1074000077A180A591A50E94ADB666A377A380A7BA
:1074100091A756CFC8010E94EF2244E050E06BA92B
:107420007CA9C8010E94D022F70162A573A584A59A
:1074300095A50E94ADB662A773A784A795A740CF74
:10744000C8010E94EF2244E050E06FA578A9C8016E
:107450000E94D022F70162A173A184A195A10E948C
:10746000ADB662A373A384A395A366A777A780ABE9
:1074700091AB26CF33243A94AACE2F923F924F92CB
:107480005F926F927F928F929F92AF92BF92CF92B4
:10749000DF92EF92FF920F931F93CF93DF9300D071
:1074A00000D0CDB7DEB78C010E9430AB2FEC37E0B7
:1074B00040E050E00E9431B5DC01CB010196A11DF6
:1074C000B11DF80184839583A683B783808391835C
:1074D000A283B3835801F3E4AF0EB11CC5010E942F
:1074E000F12364E470E0C5010E94C526882309F4F5
:1074F00045C10E94830E2B013C01480182E4880EA5
:10750000911C48EEC42E43E0D42EE12CF12C52E025
:10751000252E1E821D82D4018C918330B1F1811100
:1075200066C0F80184819581A681B7810196A11D6D
:10753000B11D84839583A683B7830E94830E64194B
:10754000750986099709A70196010E940FB5A9013F
:1075500061E0C8010E94852781E0D4018C938D8170
:107560009E810197C1F20E94830E641975098609F4
:107570009709D801D6962D913D914D915C91D9975F
:10758000261737074807590720F6C5010E94F1233F
:10759000F80184819581A681B7810196A11DB11D55
:1075A00084839583A683B7830E94830EF801FE9699
:1075B00060837183828393838D819E8126960FB62B
:1075C000F894DEBF0FBECDBFDF91CF911F910F9119
:1075D000FF90EF90DF90CF90BF90AF909F908F90F3
:1075E0007F906F905F904F903F902F9008958430E0
:1075F000F1F4F80184819581A681B7810196A11DDE
:10760000B11D84839583A683B7830E94830E64197A
:10761000750986099709A70196010E940FB5A9016E
:1076200063E0C8010E948527D4012C9298CF813055
:1076300051F5F80142AD53AD64AD75AD9E012F5FBC
:107640003F4FC8010E949E38382EF2E08F1390C041
:1076500089819A81AB81BC81F80184839583A6835B
:10766000B7830E94830E6419750986099709A701DB
:1076700096010E940FB5A90163E0C8010E94852709
:10768000D4013C926CCF823009F069CFF80142AD51
:1076900053AD64AD75AD9E012F5F3F4FC8010E9491
:1076A0009E38382EF5E08F135DC0E3E0D401EC93F3
:1076B000F80182A193A1A4A1B5A1892B8A2B8B2BC0
:1076C00041F484E893E0A0E0B0E082A393A3A4A3F4
:1076D000B5A3F80186A197A1A0A5B1A5892B8A2BF6
:1076E0008B2B61F482A193A1A4A1B5A1B695A79516
:1076F0009795879586A397A3A0A7B1A7F80182A520
:1077000093A5A4A5B5A5892B8A2B8B2BA9F482A1BF
:1077100093A1A4A1B5A1AC01BD0123E07695679525
:10772000579547952A95D1F7841B950BA60BB70B58
:1077300082A793A7A4A7B5A7F80186A197A1A0A5A2
:10774000B1A586A797A7A0ABB1AB82A593A5A4A529
:10775000B5A582AB93ABA4ABB5AB81E090E09E83C3
:107760008D83FDCE96E0891303C0D4011C92F7CE21
:10777000BFEF3B12F4CEF4011082F1CE1E821D82C7
:107780001BCF8F929F92AF92BF92EF92FF920F9377
:107790001F93CF93DF9300D000D0CDB7DEB7009119
:1077A0004C0C10914D0CF12CE12C0115110509F434
:1077B000DAC00E94830E4B015C0178012EE3E20ED9
:1077C000F11CF70180819181A281B381A50194010F
:1077D000281B390B4A0B5B0BCA01B901683E33E029
:1077E000730781059105A0F128EE33E040E050E0F9
:1077F0000E940FB5861A970AA80AB90AD7018D9276
:107800009D92AD92BC921397F80186A597A5A0A969
:10781000B1A949015A01880C991CAA1CBB1C8815E6
:107820009905AA05BB0508F0B0C016A617A610AAB0
:1078300011AAF80182A993A9A4A9B5A98815990547
:10784000AA05BB0508F0AAC012AA13AA14AA15AA71
:10785000F80186A597A5A0A9B1A9892B8A2B8B2B06
:1078600009F0A5C0EE5BFF4F8081833009F09FC017
:1078700084E08083C8010E943D3A01967C01F801B2
:1078800082A993A9A4A9B5A9892B8A2B8B2BA1F432
:10789000EE5BFF4F8081833011F081110DC01082AB
:1078A000F8013E9684E1DF011D928A95E9F7C8014F
:1078B0000E943D3A03967C01B2E0EB16F10429F0F8
:1078C000E4E0EE16F10409F04EC080E591E00E947C
:1078D000098360914C0C70914D0C625F7F4FCE011B
:1078E00001960E94968ECE0103960E94A52060917B
:1078F0004C0C70914D0C6A5E7F4FCE0101960E9438
:10790000968E44E050E0BE016D5F7F4F81E090E0D5
:107910000E94471E60914C0C70914D0C6E5E7F4F23
:10792000CE0101960E94968E44E050E0BE016D5F4C
:107930007F4F85E090E00E94471E60914C0C709153
:107940004D0C625E7F4FCE0101960E94968E8B8118
:107950009C81AD81BE818093451090934610A09389
:107960004710B0934810C70126960FB6F894DEBFB3
:107970000FBECDBFDF91CF911F910F91FF90EF9080
:10798000BF90AF909F908F900895821B930BA40B94
:10799000B50B86A797A7A0ABB1AB4BCF821B930BC0
:1079A000A40BB50B82AB93ABA4ABB5AB51CFF12C11
:1079B000E12C65CFEF92FF920F931F93CF93DF934C
:1079C000CDB7DEB7E8970FB6F894DEBF0FBECDBFD8
:1079D0006DE574E0CE0187960E942B8D6DE574E015
:1079E000CE018D960E942B8D82E0E82EF12C2496FC
:1079F000FFAEEEAE249786E0EBEFF2E0DE01D39629
:107A000001900D928A95E1F786E0FE01F396DE0182
:107A1000AC5BBF4F01900D928A95E1F701E010E059
:107A20002C961FAF0EAF2C972E961FAE1EAE2E9724
:107A300088E0E1E0F3E0DE01599601900D928A952D
:107A4000E1F788E0FE017996DE01A25BBF4F01906D
:107A50000D928A95E1F788E1E9E0F3E0DE01119605
:107A600001900D928A95E1F788E1FE013196DE01E1
:107A7000AA5ABF4F01900D928A95E1F78091210398
:107A800090912203A0912303B0912403E2968CAF3E
:107A90009DAFAEAFBFAFE2976EE974E0CE018796BF
:107AA0000E947D8A60E0CE0187960E94F28B4BA5F2
:107AB0005CA5BE016E587F4FCE0187960E945F89FC
:107AC00067E977E0CE018D960E94178C64E275E03D
:107AD00087EF92E10E947D8A60E0CE018D960E9440
:107AE000F28B49A95AA9BE0166567F4FCE018D96E9
:107AF0000E945F896DE574E0CE0187960E947D8AC1
:107B00006DE574E0CE018D960E947D8AC250DF4FF4
:107B100019821882CE5FD0401092670A80917F024E
:107B200090918002C050DF4F99838883C050D1402C
:107B300080E090E0A0E7B2E4CA5BDE4F88839983DF
:107B4000AA83BB83C654D140C65BDE4FF982E8826C
:107B5000CA54D14080E090E0A0E2B2E4C45BDE4FC2
:107B600088839983AA83BB83CC54D14080E090E082
:107B7000A4E3B2E4C05BDE4F88839983AA83BB830E
:107B8000C055D14084EB90E0CC5ADE4F9983888376
:107B9000C455D14088E790E0CA5ADE4F9983888364
:107BA000C655D1408CE291E0A0E0B0E0C85ADE4F6B
:107BB00088839983AA83BB83C855D140C45ADE4FBA
:107BC00019830883CC55D140C25ADE4FF982E8822E
:107BD000CE55D14060E089E093E10E94F28B60E0F5
:107BE00083E093E10E94F28B40910D1350910E13AC
:107BF000BE016E5F7E4F89E093E10E945F894091F4
:107C0000071350910813BE01635F7E4F83E093E139
:107C10000E945F8988E2EBE3FAE0DE01A75EBE4FD7
:107C200001900D928A95E1F78CE390E0A0E0B0E03E
:107C3000CE5BDE4F88839983AA83BB83C254D14035
:107C4000CF5BDE4F1882C154D14084EE98E3AEE89A
:107C5000B2E4C05ADE4F88839983AA83BB83C0569F
:107C6000D14084EE98E3AEE8B1E4CC59DE4F88838E
:107C70009983AA83BB83C456D140C859DE4F198368
:107C80000883C856D14080E590E0C659DE4F9983FD
:107C90008883CA56D14083E090E0C059DE4F998373
:107CA0008883C057D14088E390E0CE58DE4F998357
:107CB0008883C257D140CC58DE4F1882C457D14078
:107CC0008FEF9FEFCB58DE4F99838883C557D14004
:107CD00084EF91E09093530280935202BE016E5B59
:107CE0007F4F0E94B12964EF71E080E090E00E9434
:107CF000500E60E877E0CE0181960E94198DCE018A
:107D000081960E946C31CE0181960E948C8CCE01AE
:107D10008D960E948C8CCE0187960E948C8CE89662
:107D20000FB6F894DEBF0FBECDBFDF91CF911F918C
:107D30000F91FF90EF9008956F927F929F92AF9274
:107D4000BF92CF92DF92EF92FF920F931F93CF9348
:107D5000DF93CDB7DEB7C353D1400FB6F894DEBF83
:107D60000FBECDBF3C016B015A017E0121E8E20E3E
:107D7000F11C6CE072E1C7010E942B8D66E874E093
:107D80008E010F5F1F4FC8010E942B8DB701C801E4
:107D90000E94B58BBC01CE01885D9E4F0E94228D52
:107DA000C8010E948C8CC7010E948C8CB301CE014B
:107DB000825D9E4F0E942B8D34E0C316D10409F0E2
:107DC00097C066EA74E0CE01885D9E4F0E94068CE3
:107DD0009924939460E0CE01885D9E4F0E94F28BBF
:107DE000C45DDE4F48815981CC52D140B701CE01EC
:107DF000885D9E4F0E945F898091D60B8823B9F0E1
:107E000062ED74E0C8010E942B8DC8010E94BA3156
:107E1000C8010E948C8CBE01685D7E4FC8010E9423
:107E2000228DC8010E946C31C8010E948C8CE0EA4E
:107E3000F8E080E091E0DF019C011D92215030408C
:107E4000E1F7992009F462C0C25DDE4F6881798153
:107E5000CE52D140CF010E941EB96DE574E0CE0133
:107E6000825D9E4F0E947D8AA0903E02B0903F02AC
:107E70008091D90B9091DA0B01969093DA0B809355
:107E8000D90B2091F50B222341F06EE170E00E94A6
:107E900091B6181619060CF4BBC181E08093F50B5E
:107EA0001092DA0B1092D90BA50168E67AE083E90B
:107EB00091E10E9482256C018FE1682E712C31E0E6
:107EC000C316D10409F43DC181E0681A710809F4B0
:107ED00090C16AE070E080E090E00E94500EA50141
:107EE00068E67AE083E991E10E9482256C01E7CFA0
:107EF00066EB74E0C114D10411F065EC74E0CE01BE
:107F0000885D9E4F0E94068C912C64CFD5018C9188
:107F100011969C91C114D10491F49F938F931F9259
:107F20001F928BEE94E09F938F93FF93EF930E94A9
:107F30005CB90FB6F894DEBF0FBECDBF8ECF9F9356
:107F40008F93DF92CF92C15DDE4F8881CF52D140B7
:107F50008F93C25DDE4F8881CE52D1408F9382EEE7
:107F600094E09F938F93FF93EF930E945CB9E1CFCE
:107F700081E080934E0C41E060EA78E0CE018F5FB3
:107F80009E4F0E947391CE018F5F9E4F0E94421DB3
:107F9000882309F4ACC060EC75E083E991E10E94AC
:107FA000848E6DE675E083E991E10E94848E6CE534
:107FB00075E083E991E10E94608EC65EDE4FE88144
:107FC000F981CA51D14040E050E0BA01309721F028
:107FD00043895489658976894C535F4F6F4F7F4F32
:107FE0002AE083E991E10E948C8D83E991E10E946E
:107FF000228E83E991E10E94228E63E375E083E99A
:1080000091E10E94848E6BEF74E083E991E10E941C
:10801000608E60EA78E0CE018E5D9E4F0E942B8DCF
:10802000BE016E5D7E4FCE01845E9E4F0E94228D0A
:108030006EEF74E0CE01845E9E4F0E949F8BBC0168
:1080400083E991E10E944E8ECE01845E9E4F0E9494
:108050008C8CCE018E5D9E4F0E948C8C64ED74E002
:1080600083E991E10E94848E83E991E10E94228E4E
:108070005801F12CE12CCE018F5F9E4F0E94100C15
:10808000892BB9F0CE018F5F9E4F0E94B718D501A2
:108090008D935D01BFEFEB1AFB0AE0E8EE16F104E9
:1080A00051F740E850E0B80183E991E10E942721AF
:1080B000DFCFE114F10431F0A701B80183E991E1C8
:1080C0000E94272183E991E10E94228E69EA74E0EF
:1080D00083E991E10E94848E83E991E10E94228EDE
:1080E000CE018F5F9E4F0E944E1D10924E0C61E09C
:1080F00070E080E090E00E94500E10924E0C1092C2
:10810000F50BCE01825D9E4F0E948C8CCE01885D66
:108110009E4F0E948C8CC601CD5CDE4F0FB6F8944A
:10812000DEBF0FBECDBFDF91CF911F910F91FF90AA
:10813000EF90DF90CF90BF90AF909F907F906F9027
:108140000895FF92EF9285E195E09F938F931F939F
:108150000F930E945CB9B80183E991E10E94268ED9
:1081600088E69AE09F938F9386E295E09F938F93A2
:108170001F930F930E945CB9B80183E991E10E94BB
:10818000268E0FB6F894DEBF0FBECDBF9110F0CE95
:1081900066E674E083E991E10E94848E80EA98E0CB
:1081A000DC010D900020E9F7CD01815A98409F93A2
:1081B0008F9380E095E09F938F931F930F930E947E
:1081C0005CB9B80183E991E10E94268E60EA78E00B
:1081D00083E991E10E94268E62E574E083E991E1F2
:1081E0000E94848E0F900F900F900F900F900F9021
:1081F0007ECF66E474E0C8010E94198DC8010E9418
:108200006C31C8010E948C8C10924E0C1092F50BB0
:108210008091460C811116C062ED75E0C8010E9484
:10822000198DC8010E94BA31C8010E948C8C60EA85
:1082300078E0C8010E942B8DC8010E946C31C801F2
:108240000E948C8C62E370E080E090E00E94500E0F
:1082500083E991E10E94342583E991E10E946D2533
:10826000E0EAF8E080E091E0DF019C011D922150FE
:108270003040E1F780E8D7011D928A95E9F7D12CCB
:10828000C12C3FCFEF92FF920F931F93CF93DF93B9
:10829000CDB7DEB768970FB6F894DEBF0FBECDBF7F
:1082A00081E08093F50B0E94C13B8C0160ED77E08B
:1082B00080E090E00E94500E8BE0E82EF12C0D7FC4
:1082C0000130110571F481E0E81AF10851F00E94C3
:1082D000C13B8C0160ED77E080E090E00E94500EA1
:1082E000EECF0E94A28E7C0168EE73E080E090E009
:1082F0000E94500E0BE010E0EF2899F40150110994
:1083000081F060ED77E080E090E00E94500E0E94E6
:10831000A28E7C0168EE73E080E090E00E94500E37
:10832000EBCF8DE490E10E9493281092F50B0E9410
:10833000EF376DE574E0CE0107960E942B8D66E065
:1083400077E0CE010D960E94198DCE0143960E94D2
:108350009529888D1F928F938F891F928F938E8975
:108360001F928F938D891F928F938EE894E09F9335
:108370008F9386EA99E09F938F930E945CB966EA97
:1083800079E0CE0101960E942B8DBE016F5F7F4F79
:10839000CE0107960E94538CCE0101960E948C8CD0
:1083A000BE01635F7F4FCE0101960E94228DCE01F8
:1083B00001960E94BA31CE0101960E948C8CBE01BA
:1083C000695F7F4FCE0101960E94228DCE010196FA
:1083D0000E946C31CE0101960E948C8CBE01695FB7
:1083E0007F4FCE0101960E94228DAE014F5F5F4FFD
:1083F00063E070E080E092E00E949C3E8C01CE0140
:1084000001960E948C8C0FB6F894DEBF0FBECDBFD4
:10841000012B59F56CEF76E0CE0101960E94198D83
:10842000CE0101960E94BA31CE0101960E948C8C39
:10843000BE01635F7F4FCE0101960E94228DCE0167
:1084400001960E94BA31CE0101960E948C8C60E6A2
:1084500071E1CE0101960E94228DCE0101960E940B
:108460006C31CE0101960E948C8CCE010D960E943B
:108470008C8CCE0107960E948C8C68960FB6F8946F
:10848000DEBF0FBECDBFDF91CF911F910F91FF9047
:10849000EF9008953F924F925F926F927F928F92EA
:1084A0009F92AF92BF92CF92DF92EF92FF920F9383
:1084B0001F93CF93DF93CDB7DEB762970FB6F894D3
:1084C000DEBF0FBECDBF69EE76E0CE0101960E9401
:1084D000198DCE0101960E946C31CE0101960E9449
:1084E0008C8C04E010E032E7C32E39E0D32E40E359
:1084F000E42E53EE752E66E0662E7CEE572EE1E3F9
:10850000FE2EFEE44F2EA4E33A2E68EB72E283E3E4
:1085100091E10E94C526F6018E2D11928A95E9F708
:10852000709272096092740950927509F0927E09F6
:1085300040927F09F09280093092810960E472E0F4
:10854000CE0101960E94968E4BE750E0BE016F5F10
:108550007F4F83E391E10E944E2740E350E062E7C2
:1085600079E083E391E10E94E32683E391E10E94B5
:108570001D2768EE73E080E090E00E94500E83E3D8
:1085800091E10E941923892B09F053C00150110970
:1085900009F080C08091A2099091A309A091A4093B
:1085A000B091A509892B8A2B8B2B09F08DC06DE525
:1085B00074E08EE791E10E947D8A6EE771E1CE0161
:1085C00001960E94228DAE014F5F5F4F70E060E028
:1085D00083E892E00E949C3E8C01CE0101960E94AD
:1085E0008C8C012B71F461ED76E0CE0101960E9436
:1085F000198DCE0101960E946C31CE0101960E9428
:108600008C8C62960FB6F894DEBF0FBECDBFDF91A3
:10861000CF911F910F91FF90EF90DF90CF90BF907F
:10862000AF909F908F907F906F905F904F903F9012
:10863000089540E350E062E779E083E391E10E942E
:10864000D02260919A0970919B0976276727762737
:1086500090E080E0CB017727662700919C0910917C
:108660009D0910270127102730E020E0602B712B97
:10867000822B932B7E508A4A93480E948F0E0E9431
:10868000420F6093A2097093A3098093A409909369
:10869000A50980CF8090A2099090A309A090A40979
:1086A000B090A50968EE73E080E090E00E94500E63
:1086B0002AE0B501A40181E59FE00E948C8D81E54F
:1086C0009FE00E94228E21CF68EE73E080E090E070
:1086D0000E94500E0E94420F6093ED0B7093EE0BC0
:1086E0008093EF0B9093F00B0E94420F6093E70B87
:1086F0007093E80B8093E90B9093EA0BCE010196FF
:108700000E948030CE0101960E946C31CE0101960C
:108710000E948C8C0E949A0FBC01CE0107960E9489
:10872000A92E69E574E0CE0107960E94068C0E948E
:10873000920FBC01CE0101960E94A92EBE016F5F6F
:108740007F4FCE0107960E94108CCE0101960E94A9
:108750008C8C69E574E0CE0107960E94068C0E941D
:10876000880FBC01CE0101960E94A92EBE016F5F49
:108770007F4FCE0107960E94108CCE0101960E9479
:108780008C8C6FE275E0CE0101960E942B8DBE01AC
:10879000695F7F4FCE0101960E94B58BBC01CE016F
:1087A0000D960E94228D4AE050E06FEF7FEFCE01E0
:1087B0000D960E945937CE010D960E948C8CCE01E9
:1087C00001960E948C8CCE0107960E948C8C68EEDC
:1087D00073E080E090E00E94500E0E94AA0FBC015E
:1087E000CE010D960E94A92E0E94A20FBC01CE01BF
:1087F00001960E94A92E6FE476E0CE0107960E94B2
:108800002B8DBE016F5F7F4FCE0107960E94B58B07
:10881000BC01CE010D960E94108CCE0107960E94DD
:108820008C8CCE0101960E948C8C0E94420F0E947B
:10883000680A6091B60B70E0CE0101960E94A92EE5
:108840006FE476E0CE0107960E942B8DBE016F5F2C
:108850007F4FCE0107960E94B58BBC01CE010D96CD
:108860000E94108CCE0107960E948C8CCE0101963E
:108870000E948C8C65E375E0CE0101960E942B8DE1
:10888000BE01635F7F4FCE0101960E94B58BBC0194
:10889000CE0107960E94228D4AE050E06FEF7FEFF5
:1088A000CE0107960E945937CE0107960E948C8C04
:1088B000CE0101960E948C8CCE010D960E948C8C6C
:1088C00068EE73E080E090E00E94500ECE010196C9
:1088D0000E94FF2F4AE050E06FEF7FEFCE0101963C
:1088E0000E9459378ACECF92DF92EF92FF920F9378
:1088F0001F93CF93DF93CDB7DEB768970FB6F89489
:10890000DEBF0FBECDBF6DE574E0CE0143960E9481
:108910002B8D65EE78E0CE0101960E94198DCE0177
:1089200001960E94BA31CE0101960E948C8C6CA1F6
:108930007DA1CE0101960E94878ACE0101960E94F8
:108940006C31CE0101960E948C8C6DEC78E0CE01EA
:1089500001960E94198DCE0101960E94BA31CE0176
:1089600001960E948C8CCE5ADE4F68817981C25567
:10897000D140CE0101960E94878ACE0101960E94C5
:108980006C31CE0101960E948C8C60EC78E0CE01B7
:1089900001960E94198DCE0101960E94BA31CE0136
:1089A00001960E948C8C03E51CE0EE24E394F12CEC
:1089B000CE5ADE4F88819981C255D1408E159F05D0
:1089C0000CF44AC0F80182819381C6979CF16BE355
:1089D00075E0CE0101960E942B8DCE0101960E947A
:1089E000BA31CE0101960E948C8CF80162817381AC
:1089F00066537109CE0101960E94878ACE010196C5
:108A00000E94BA31CE0101960E948C8C6AEB75E00F
:108A1000CE0101960E942B8DCE0101960E94BA31A3
:108A2000CE0101960E948C8CFFEFEF1AFF0A0E5FB9
:108A30001F4FBECF6DE375E0CE0101960E942B8DD6
:108A4000CE0101960E94BA31CE0101960E948C8C13
:108A5000F80162817381CECF6AEB75E0CE01019699
:108A60000E942B8DCE0101960E946C31CE010196A1
:108A70000E948C8C61EB78E0CE0101960E94198DEA
:108A8000CE0101960E94BA31CE0101960E948C8CD3
:108A900060915B0C70915C0CCE0101960E94878AFC
:108AA000CE0101960E94BA31CE0101960E948C8CB3
:108AB0006AEB75E0CE0101960E942B8DCE010196E6
:108AC0000E94BA31CE0101960E948C8C60915D0C9F
:108AD00070915E0CCE0101960E94878ACE010196AC
:108AE0000E946C31CE0101960E948C8C6AE978E07C
:108AF000CE0101960E94198DCE0101960E94BA31D5
:108B0000CE0101960E948C8CBE01605D7F4FCE012C
:108B100001960E942B8DCE0101960E94BA31CE01A2
:108B200001960E948C8C6AEB75E0CE0101960E9442
:108B30002B8DCE0101960E94BA31CE0101960E9482
:108B40008C8CBE016C5C7F4FCE0101960E942B8DF8
:108B5000CE0101960E946C31CE0101960E948C8C50
:108B60006AE878E0CE0101960E94198DCE01019647
:108B70000E946C31CE0101960E948C8C8E010C5D9E
:108B80001F4FEE24E394F12C680188E0C80ED11C3D
:108B90008CA19DA18E159F050CF449C0B701CE0193
:108BA00007960E94878A65E876E0CE0101960E94CA
:108BB0002B8DBE01695F7F4FCE0101960E94B58B60
:108BC000BC01CE010D960E94228DCE010D960E9411
:108BD000BA31CE010D960E948C8CCE0101960E9476
:108BE0008C8CCE0107960E948C8C6FE476E0CE01CF
:108BF00001960E942B8DCE0101960E94BA31CE01C2
:108C000001960E948C8CB801645E7F4FCE01019664
:108C10000E942B8DCE0101960E946C31CE010196EF
:108C20000E948C8CEFEFEE1AFE0A8601ADCF69E749
:108C300078E0CE0101960E94198DCE0101960E9426
:108C4000BA31CE0101960E948C8C7E01F2EBEF1AB4
:108C5000FEEFFF0A10E000E0F70161917F0170E094
:108C6000CE0101960E94878ACE0101960E94BA31F8
:108C7000CE0101960E948C8C0330110571F06FE3D8
:108C800075E0CE0101960E942B8DCE0101960E94C7
:108C9000BA31CE0101960E948C8C0F5F1F4F0430B9
:108CA0001105D1F66AEB75E0CE0101960E942B8D7D
:108CB000CE0101960E946C31CE0101960E948C8CEF
:108CC000C45BDE4F68817981CC54D140072E000C03
:108CD000880B990B0E94CCB39B01AC010E948CB60F
:108CE000882341F080E590E0C45BDE4F9983888360
:108CF000CC54D140C45BDE4F88819981CC54D140A3
:108D000090933F0280933E026FE578E0CE0101969A
:108D10000E94198DCE0101960E94BA31CE010196B2
:108D20000E948C8C68E67AE0CE0101960E942B8D21
:108D3000CE0101960E94BA31CE0101960E948C8C20
:108D40006DE578E0CE0101960E94198DCE01019665
:108D50000E94BA31CE0101960E948C8C60913E0235
:108D600070913F02CE0101960E94878ACE01019642
:108D70000E946C31CE0101960E948C8C6EE478E0EA
:108D8000CE0101960E94198DCE0101960E94BA3142
:108D9000CE0101960E948C8CBE016C5A7F4FCE0191
:108DA00001960E942B8DCE0101960E946C31CE015E
:108DB00001960E948C8C61E475E0CE0101960E94C0
:108DC0002B8DCE0101960E94BA31CE0101960E94F0
:108DD0008C8CBE0164587F4FCE0101960E942B8D72
:108DE000CE0101960E946C31CE0101960E948C8CBE
:108DF000C052DF4F88819981C05ED040892B71F4C9
:108E000066E478E0CE0101960E94198DCE010196AC
:108E10000E946C31CE0101960E948C8CC052DF4FB3
:108E200088819981C05ED040019771F46CE378E04D
:108E3000CE0101960E94198DCE0101960E946C31DF
:108E4000CE0101960E948C8CC052DF4F888199819F
:108E5000C05ED040029771F463E378E0CE010196E2
:108E60000E94198DCE0101960E946C31CE010196AF
:108E70000E948C8C6DE278E0CE0101960E94198DE3
:108E8000CE0101960E94BA31CE0101960E948C8CCF
:108E9000CE51DF4F68817981C25ED040CE0101960C
:108EA0000E94878ACE0101960E946C31CE01019604
:108EB0000E948C8C64E278E0CE0101960E94198DAC
:108EC000CE0101960E94BA31CE0101960E948C8C8F
:108ED000CC5ADE4F88819981C455D140C6970CF495
:108EE0003FC16BE375E0CE0101960E942B8DCE0150
:108EF00001960E94BA31CE0101960E948C8CCC5A08
:108F0000DE4F68817981C455D14066537109CE0125
:108F100001960E94878ACE0101960E946C31CE0193
:108F200001960E948C8C4091DF0B5091E00B609178
:108F3000E10B7091E20B21E0CE0107960E94948C28
:108F40006CE475E0CE0101960E942B8DBE01695F35
:108F50007F4FCE0101960E94B58B68E575E00E94B7
:108F60009F8BBC01CE010D960E94228DCE010D96E5
:108F70000E946C31CE010D960E948C8CCE01019620
:108F80000E948C8CCE0107960E948C8C4091DB0B4A
:108F90005091DC0B6091DD0B7091DE0B21E0CE0176
:108FA00007960E94948C6DE575E0CE0101960E94B3
:108FB0002B8DBE01695F7F4FCE0101960E94B58B5C
:108FC00068E575E00E949F8BBC01CE010D960E9462
:108FD000228DCE010D960E946C31CE010D960E941D
:108FE0008C8CCE0101960E948C8CCE0107960E943B
:108FF0008C8C65E078E0CE0101960E94198DCE013F
:1090000001960E94BA31CE0101960E948C8C40914B
:10901000290250912A0260912B0270912C0225E0C6
:10902000CE0101960E94948CCE0101960E946C3173
:10903000CE0101960E948C8C6AEE77E0CE010196FB
:109040000E94198DCE0101960E94BA31CE0101967F
:109050000E948C8C4091250250912602609127023B
:109060007091280225E0CE0101960E94948CCE01D9
:1090700001960E946C31CE0101960E948C8C69EDA4
:1090800077E0CE0101960E94198DCE0101960E94D3
:10909000BA31CE0101960E948C8C60916C02709165
:1090A0006D02CE0101960E94878ACE0101960E9430
:1090B0006C31CE0101960E948C8C60EC77E0CE0181
:1090C00001960E94198DCE0101960E94BA31CE01FF
:1090D00001960E948C8CC65BDE4F68817981CA54F0
:1090E000D140CE0101960E94878ACE0101960E944E
:1090F0006C31CE0101960E948C8C69EA77E0CE013A
:1091000001960E94198DCE0101960E94BA31CE01BE
:1091100001960E948C8CC95ADE4F68817981C755AF
:10912000D140CE0101960E94878ACE0101960E940D
:109130006C31CE0101960E948C8CCE0143960E9428
:109140008C8C68960FB6F894DEBF0FBECDBFDF9152
:10915000CF911F910F91FF90EF90DF90CF900895E6
:109160006DE375E0CE0101960E942B8DCE01019634
:109170000E94BA31CE0101960E948C8CCC5ADE4FEF
:1091800068817981C455D140C2CE2F923F924F92CF
:109190005F926F927F928F929F92AF92BF92CF9287
:1091A000DF92EF92FF920F931F93CF93DF93CDB790
:1091B000DEB7EC970FB6F894DEBF0FBECDBF9CA70D
:1091C0008BA71B0170E060E00E94538B182F6DE5A8
:1091D00074E0CE0149960E942B8D80916C02909193
:1091E0006D02019709F07AC082E090E00E94078941
:1091F00088E090E0909324028093230289E090E03D
:1092000090932202809321028091390A90913A0A28
:109210009093380A8093370A80911D0290911E0224
:10922000A0911F02B09120028093190290931A021C
:10923000A0931B02B0931C028091350290913602DC
:10924000A0913702B09138028093390290933A028C
:10925000A0933B02B0933C028091360A8093350A7A
:109260008091310A9091320AA091330AB091340A68
:1092700080932D0A90932E0AA0932F0AB093300A60
:109280008AE390E090931802809317028091DF0B9D
:109290009091E00BA091E10BB091E20B8093630AF7
:1092A0009093640AA093650AB093660A80911502B0
:1092B00090911602909314028093130280912902D8
:1092C00090912A02A0912B02B0912C0280932D0242
:1092D00090932E02A0932F02B093300280916C02E3
:1092E00090916D02029709F07AC083E090E00E94AD
:1092F00007898AE090E090932402809323028BE018
:1093000090E0909322028093210280912B0A909109
:109310002C0A9093380A8093370A80910F0290911B
:109320001002A0911102B091120280931902909341
:109330001A02A0931B02B0931C02809131029091FB
:109340003202A0913302B09134028093390290939B
:109350003A02A0933B02B0933C0280912A0A809388
:10936000350A8091260A9091270AA091280AB09187
:10937000290A80932D0A90932E0AA0932F0AB09366
:10938000300A8BE390E0909318028093170280914B
:10939000DB0B9091DC0BA091DD0BB091DE0B809389
:1093A000630A9093640AA093650AB093660A809159
:1093B0000D0290910E0290931402809313028091FB
:1093C000250290912602A0912702B0912802809355
:1093D0002D0290932E02A0932F02B09330021335EA
:1093E000C1F41092380A1092370A8091D60B882364
:1093F00071F065E675E0CE0101960E942B8DCE01DD
:1094000001960E946C31CE0101960E948C8CE12C59
:10941000E1C0C1010197029708F06EC181E090E0C0
:10942000A0E0B0E08093190290931A02A0931B026F
:10943000B0931C02ABA5BCA514968D919C91159779
:10944000029750F141E050E0BD01CE0101960E942B
:109450009D2EBE016F5F7F4FCE0149960E94538CB7
:10946000CE0101960E948C8CCE014996B1E02B165C
:10947000310471F50E94E08A20E030E040E251E4DE
:109480000E942BB40E9451B66093190270931A0285
:1094900080931B0290931C0281E090E09093380A25
:1094A0008093370A1134F9F48091D60B882371F038
:1094B0006AE675E0CE0101960E942B8DCE010196E1
:1094C0000E946C31CE0101960E948C8CE12C4FC021
:1094D0000E94E08A20912D0230912E0240912F02AD
:1094E00050913002CDCF163409F0F0C08091D60BE8
:1094F000882371F063E775E0CE0101960E942B8D01
:10950000CE0101960E94BA31CE0101960E948C8C48
:10951000EE24E394F12CD090210260E08D2D0E9486
:10952000CC0D64E670E080E090E00E94500E009167
:1095300023026E2D802F0E94CC0D64EF71E080E03D
:1095400090E00E94500E60E08D2D0E94CC0D64E6EC
:1095500070E080E090E00E94500E6E2D802F0E94FF
:10956000CC0D64EF71E080E090E00E94500E80919D
:10957000D60B882379F14091190250911A0260911B
:109580001B0270911C022AE0CE0101960E94CA8C37
:10959000BE016F5F7F4FCE0107960E94228D67E864
:1095A00075E0CE0107960E949F8BBC01CE010D96FF
:1095B0000E94228DCE010D960E946C31CE010D9637
:1095C0000E948C8CCE0107960E948C8CCE01019655
:1095D0000E948C8C8090190290901A02A0901B021D
:1095E000B0901C02181419041A041B040CF046C590
:1095F000163409F44CC4123509F44DC410912302F9
:109600006E2D812F0E94CC0D64EF71E080E090E020
:109610000E94500E6E2D812F0E94CC0D60ED77E0E0
:1096200080E090E00E94500E6E2D812F0E94CC0DA4
:109630006CED75E080E090E00E94500E81E090E0DB
:109640009093380A8093370A1091210261E0812FAC
:109650000E94CC0D61E070E080E090E00E94500E2E
:1096600060E0812F0E94CC0D6AE070E080E090E025
:109670000E94500EC12CD12C7601C3948C149D04F1
:10968000AE04BF0409F409C461E0812F0E94CC0D2F
:1096900061E070E080E090E00E94500E60E0812F79
:1096A0000E94CC0D6091390270913A0280913B0288
:1096B00090913C026F5F7F4F8F4F9F4F0E94500EE3
:1096C000FFEFCF1ADF0AEF0AFF0AD8CF123591F465
:1096D0008091D60B882371F06DE775E0CE0101967D
:1096E0000E942B8DCE0101960E94BA31CE010196C7
:1096F0000E948C8CE12C0FCF2114310429F0E3E07F
:109700002E16310409F083CE80916C0290916D0287
:1097100020E137E240E050E08130910521F420E47F
:109720003CE940E050E02FA738AB49AB5AAB21E011
:1097300030E03093380A2093370A3093490220935F
:109740004802029761F433E02316310441F480911A
:10975000DA129091DB129093490280934802409173
:109760004802509149025EA74DA7052F001F002710
:10977000001F81E090E09093490280934802E090BE
:10978000210260E08E2D0E94CC0D64E670E080E046
:1097900090E00E94500EF0902302602F8F2D0E94C7
:1097A000CC0D64EF71E080E090E00E94500E602FDD
:1097B0008F2D0E94CC0D68EE73E080E090E00E9457
:1097C000500E60E08E2D0E94CC0D64E670E080E0CB
:1097D00090E00E94500E602F8F2D0E94CC0D64EF00
:1097E00071E080E090E00E94500E8FEF9FEF909329
:1097F000140280931302812C912C54011FA218A6ED
:1098000019A61AA61BA21CA21DA21EA21F8E18A278
:1098100019A21AA2412C512C32011FAA18AE19AE5E
:109820001AAE1BAA1CAA1DAA1EAAF090210261E072
:109830008F2D0E94CC0D61E070E080E090E00E94EE
:10984000500E60E08F2D0E94CC0D61E070E080E052
:1098500090E00E94500EC501B40126E030E040E0E7
:1098600050E00E9431B5672B682B692B09F0F8C0D6
:10987000A2E0B0E0BCAFABAFC12CD12C760180919F
:109880001702863308F0865320917B00982F98703A
:10989000277F922B90937B008770806480937C005D
:1098A00080917A00806480937A0080917A0086FDAE
:1098B000FCCF8091780060917900762F682F072E79
:1098C000000C880B990B0E94CCB39B01AC01C70123
:1098D000B6010E9473B56B017C0162E070E080E02C
:1098E00090E00E94500E2BAD3CAD2130310509F0C7
:1098F000ADC020E030EC4FEF54E4C701B6010E9448
:10990000DFB56B017C018091D60B882399F12DEC9A
:109910003CEC4CE45EE3C701B6010E9487B687FDCC
:1099200029C022E0B701A601CE0107960E94948CBF
:109930006EE875E0CE0101960E942B8DBE01695F35
:109940007F4FCE0101960E94B58BBC01CE010D96D2
:109950000E94228DCE010D960E946C31CE010D9693
:109960000E948C8CCE0101960E948C8CCE010796B1
:109970000E948C8C2AE939E949E95EE3C701B60106
:109980000E9487B687FD13C041145104610471041D
:1099900011F4240135018BA19CA1ADA1BEA1892B9D
:1099A0008A2B8B2B21F48BA29CA2ADA2BEA22DEC04
:1099B0003CEC4CE45EE3C701B6010E94C5B3181647
:1099C0000CF449C0411451046104710409F448C005
:1099D0002F8D38A149A15AA1232B242B252B69F4C3
:1099E0008FA198A5A9A5BAA5892B8A2B8B2B09F441
:1099F00003C18F8E98A2A9A2BAA22F8D38A149A126
:109A00005AA1421653066406750654F58091130256
:109A10009091140297FFF5C0109214021092130255
:109A2000420E531E641E751ED301C201B595A79543
:109A3000979587958FAB98AFA9AFBAAF1F8E18A235
:109A400019A21AA2412C512C32010AC0E1E0F0E027
:109A5000FCAFEBAF14CF411451046104710469F6FB
:109A6000E0901302F090140292E0E916F1043CF445
:109A7000F7FCE3C0A3E02A16310409F0DEC08FA48E
:109A800098A8A9A8BAA8BAE08B0E911CA11CB11C79
:109A90008FA598A9A9A9BAA988169906AA06BB06EE
:109AA0000CF4C3CEF2E0EF16F1040CF479C06BA90C
:109AB0007CA98DA99EA92FA938AD49AD5AAD621BCD
:109AC000730B840B950B0E94CCB34B015C01B70167
:109AD000FF0C880B990B0E94CCB39B01AC01C50114
:109AE000B4010E94DFB520E030E044EB53E40E9473
:109AF000DFB56B017C01C0922D02D0922E02E09264
:109B00002F02F092300220E030E040E85FE30E9454
:109B100087B687FDACC080916C0290916D02813058
:109B2000910509F090C0C092D212D092D312E09267
:109B3000D412F092D512C0922902D0922A02E09259
:109B40002B02F0922C026FE277E0CE0101960E9488
:109B5000198DCE0101960E94BA31CE0101960E9464
:109B60008C8C40912D0250912E0260912F027091A9
:109B7000300225E0CE0101960E94948CCE01019620
:109B80000E946C31CE0101960E948C8C84EF91E092
:109B9000909353028093520264EB71E10E94B129C9
:109BA00033E02316310429F0E02E2114310409F0AA
:109BB00011CD8BA59CA50E94E08A6B017C01C0920F
:109BC000630AD092640AE092650AF092660A20E085
:109BD00030E044EB53E4C701B6010E9487B687FD2D
:109BE0006AC020E030E044EB53E4C701B6010E94B4
:109BF00072B56B017C01EBCF8FA298A6A9A6BAA67D
:109C0000F8CE2114310409F02BCF01969093140261
:109C1000809313022F8D38A149A15AA1420E531EE1
:109C2000641E751ED301C201B595A79597958795BA
:109C30008BAB9CABADABBEAB01CFEFEF8E1A9E0AE8
:109C4000AE0ABE0A25CF029709F07DCFC092D61288
:109C5000D092D712E092D812F092D912C092250277
:109C6000D0922602E0922702F09228026CCF63E1A4
:109C700077E0CE0101960E94198DCE0101960E94D7
:109C8000BA31CE0101960E948C8C40912D025091E8
:109C90002E0260912F027091300225E0CE010196D4
:109CA0000E94948CCE0101960E946C31CE010196E7
:109CB0000E948C8C75CF20E030E0A901C701B6016D
:109CC0000E94C5B387FF0BC020E030E044EB53E4B3
:109CD000C701B6010E9473B56B017C01ECCFC09245
:109CE0002D0AD0922E0AE0922F0AF092300A4FA04D
:109CF00058A469A47AA48BA19CA1ADA1BEA1481AC5
:109D0000590A6A0A7B0A21143104D9F410922D0AE7
:109D100010922E0A10922F0A1092300AADA5BEA5FD
:109D2000C12CD12C7601C394812C912C5401B7FF06
:109D30001CC0812C912C5401CC24CA94DC2C7601BB
:109D400014C0EDA5FEA5C12CD12C7601C394F7FF5C
:109D500004C0CC24CA94DC2C760180902D0A90900B
:109D60002E0AA0902F0AB090300A20912D02309137
:109D70002E0240912F0250913002C501B4010E9481
:109D80002BB44B015C01A3019201C701B6010E94F3
:109D9000FFB40E94CCB320E030E040E05FE30E94DB
:109DA0002BB49B01AC01C501B4010E9472B50E94A5
:109DB00051B66093190270931A0280931B0290931C
:109DC0001C028091D60B882309F441C02AE04FA1E0
:109DD00058A569A57AA5CE010D960E94CA8C2AE0E5
:109DE0004BA15CA16DA17EA1CE0107960E94CA8CF9
:109DF00065E975E0CE0101960E942B8DBE01695F79
:109E00007F4FCE0101960E94B58B6AEB75E00E94F0
:109E10009F8BBE01635F7F4F0E94B58BBC01CE015B
:109E200043960E94228DCE0143960E946C31CE0152
:109E300043960E948C8CCE0101960E948C8CCE01A0
:109E400007960E948C8CCE010D960E948C8C80917E
:109E5000190290911A02A0911B02B0911C02E12CF0
:109E600012E5B7FFB7CBB095A095909581959F4F20
:109E7000AF4FBF4F8093190290931A02A0931B0219
:109E8000B0931C02EE24E394F12C16E4A3CBEE2451
:109E9000E394F12CB3CBE12CB1CB22E022163104B8
:109EA00024F42114310409F0E1C061E080E00E9453
:109EB0000D8432E02316310424F42114310409F016
:109EC0009CC0C090630AD090640AE090650AF0904C
:109ED000660A20E030E044EB53E4C701B6010E947B
:109EE00087B687FD0BC020E030E044EB53E4C701A8
:109EF000B6010E9472B56B017C01EBCF20E030E02F
:109F0000A901C701B6010E94C5B387FF0BC020E0BD
:109F100030E044EB53E4C701B6010E9473B56B0116
:109F20007C01ECCFC092630AD092640AE092650A89
:109F3000F092660A80916C0290916D020197B1F4E3
:109F40006DE475E08FE091E10E947D8A8091630A63
:109F50009091640AA091650AB091660A8093DF0B24
:109F60009093E00BA093E10BB093E20B80916C0215
:109F700090916D020297B1F46EE575E08FE091E18A
:109F80000E947D8A8091630A9091640AA091650A7B
:109F9000B091660A8093DB0B9093DC0BA093DD0BF2
:109FA000B093DE0B4091630A5091640A6091650A98
:109FB0007091660A20E0CE0107960E94948C6FE0B3
:109FC00071E1CE0101960E94228DBE01695F7F4F33
:109FD000CE0101960E94B58B69E575E00E949F8BCA
:109FE000BC018FE091E10E943C8CCE0101960E9461
:109FF0008C8CCE0107960E948C8C41E02416310493
:10A0000039F54091190250911A0260911B0270912A
:10A010001C0221E0CE0107960E94CA8C6DE975E012
:10A02000CE0101960E942B8DBE01695F7F4FCE014C
:10A0300001960E94B58BBC018FE091E10E943C8C9F
:10A04000CE0101960E948C8CCE0107960E948C8CCA
:10A050006FE071E1CE0101960E94228DCE01019642
:10A060000E942E38CE0101960E948C8C109219020B
:10A0700010921A0210921B0210921C0280916C0224
:10A0800090916D028130910509F083C08091370A6B
:10A090009091380A90933A0A8093390A8091190274
:10A0A00090911A02A0911B02B0911C0280931D0294
:10A0B00090931E02A0931F02B09320028091390258
:10A0C00090913A02A0913B02B0913C0280933502FC
:10A0D00090933602A0933702B09338028091350AEC
:10A0E0008093360A80912D0A90912E0AA0912F0A12
:10A0F000B091300A8093310A9093320AA093330AC8
:10A10000B093340A8091630A9091640AA091650A21
:10A11000B091660A8093DF0B9093E00BA093E10B64
:10A12000B093E20B80911302909114029093160267
:10A1300080931502232881F480912D0290912E02A4
:10A14000A0912F02B09130028093290290932A02AD
:10A15000A0932B02B0932C02CE0149960E948C8CC6
:10A16000EC960FB6F894DEBF0FBECDBFDF91CF9156
:10A170001F910F91FF90EF90DF90CF90BF90AF9025
:10A180009F908F907F906F905F904F903F902F9017
:10A190000895029709F78091370A9091380A9093B1
:10A1A0002C0A80932B0A8091190290911A02A09197
:10A1B0001B02B0911C0280930F0290931002A09397
:10A1C0001102B09312028091390290913A02A0914B
:10A1D0003B02B0913C028093310290933202A093F3
:10A1E0003302B09334028091350A80932A0A809119
:10A1F0002D0A90912E0AA0912F0AB091300A8093D7
:10A20000260A9093270AA093280AB093290A8091DE
:10A21000630A9091640AA091650AB091660A8093DE
:10A22000DB0B9093DC0BA093DD0BB093DE0B8091E6
:10A2300013029091140290930E0280930D02232832
:10A2400009F08ACF80912D0290912E02A0912F02C9
:10A25000B09130028093250290932602A0932702AA
:10A26000B093280279CF2F923F924F925F926F92D4
:10A270007F928F929F92AF92BF92CF92DF92EF9296
:10A28000FF920F931F93CF93DF93CDB7DEB7E59780
:10A290000FB6F894DEBF0FBECDBF6DE271E1CE0107
:10A2A0008E960E94228D0EA51FA50115110571F035
:10A2B000D8018D918D01882349F0082E000C990B4F
:10A2C0000E94D3B8F80131978083F2CF64E77DE034
:10A2D000CE0101960E94198DBE016F5F7F4FCE01A6
:10A2E0008E960E94848B182FCE0101960E948C8C32
:10A2F000112309F401C145E050E06DE271E1CE01A6
:10A3000001960E949D2EBE016F5F7F4F89E091E113
:10A310000E94538CCE0101960E948C8C89E091E1C1
:10A320000E94F68A60E089E091E10E94F28B409100
:10A330000D1150910E116CE072E189E091E10E94E3
:10A340005F8966E874E0CE0101960E942B8DBE0104
:10A350006F5F7F4F89E091E10E94848B182FCE01BF
:10A3600001960E948C8C60E774E0111102C065E7D1
:10A3700074E0CE0101960E942B8D69E071E1CE015F
:10A3800001960E94B58BBC0185E193E10E943C8C53
:10A39000CE0101960E948C8C85E193E10E94F68AA1
:10A3A0004091191350911A134150510965E173E11D
:10A3B000CE0101960E949D2EBE016F5F7F4F87EFF9
:10A3C00092E10E94538CCE0101960E948C8C87EF03
:10A3D00092E10E94EB8A0E94CCB39B01AC010E94E7
:10A3E0008CB6882309F448C06091191370911A1330
:10A3F0006250710985E193E10E94538B682FCE0171
:10A4000001960E94F78CBE016F5F7F4F87EF92E14C
:10A410000E94538CCE0101960E948C8C66E874E0F9
:10A42000CE0101960E942B8DBE016F5F7F4F87EF9B
:10A4300092E10E94848B182FCE0101960E948C8C91
:10A440001123D1F06091191370911A13635071099F
:10A4500085E193E10E94538B682FCE0101960E9403
:10A46000F78CBE016F5F7F4F87EF92E10E94538CA4
:10A47000CE0101960E948C8C84EF91E09093530260
:10A480008093520264EB71E10E94B12964E670E0AE
:10A4900080E090E00E94500E80913D02882371F090
:10A4A0006DE271E1CE0101960E94228DCE010196EE
:10A4B0000E94D32FCE0101960E948C8CCE018E96E5
:10A4C0000E948C8C81E0E5960FB6F894DEBF0FBE3B
:10A4D000CDBFDF91CF911F910F91FF90EF90DF9053
:10A4E000CF90BF90AF909F908F907F906F905F9034
:10A4F0004F903F902F9008956EE67DE0CE0101963B
:10A500000E94198DBE016F5F7F4FCE018E960E9413
:10A51000848B182FCE0101960E948C8C112309F494
:10A5200047C045E050E06DE271E1CE0101960E9426
:10A530009D2EBE016F5F7F4F89E091E10E94538C99
:10A54000CE0101960E948C8C89E091E10E94F68AEE
:10A5500060E089E091E10E94F28B40910D115091F1
:10A560000E1164EE71E189E091E10E945F8964EE71
:10A5700071E1CE014C960E942B8D68E874E0CE010B
:10A5800001960E942B8DBE01645E7F4FCE01019625
:10A590000E94B58BBC018FE093E10E943C8CCE0100
:10A5A00001960E948C8CCE014C960E948C8C64CFBC
:10A5B0006AE67DE0CE0101960E94198DBE016F5FB3
:10A5C0007F4FCE018E960E94848B182FCE0101966C
:10A5D0000E948C8C1123E1F043E050E06DE271E1C8
:10A5E000CE0101960E949D2EBE016F5F7F4F89E0D4
:10A5F00091E10E94538CCE0101960E948C8C69E0FF
:10A6000071E1CE0101960E94228DCE010196CDCF3F
:10A6100065E67DE0CE0101960E94198DBE016F5F57
:10A620007F4FCE018E960E94848B182FCE0101960B
:10A630000E948C8C112301F144E050E06DE271E145
:10A64000CE0101960E949D2EBE016F5F7F4F89E073
:10A6500091E10E94538CCE0101960E948C8C89E07E
:10A6600091E10E94EB8A709373126093721270935F
:10A67000800260937F0200CF6FE57DE0CE010196FE
:10A680000E94198DBE016F5F7F4FCE018E960E9492
:10A69000848B182FCE0101960E948C8C112309F413
:10A6A00049C045E050E06DE271E1CE0101960E94A3
:10A6B0009D2EBE016F5F7F4F89E091E10E94538C18
:10A6C000CE0101960E948C8C89E091E10E94EB8A78
:10A6D0007093CF126093CE1284EF91E09093530267
:10A6E0008093520264EB71E10E94B12964E670E04C
:10A6F00080E090E00E94500E65E876E0CE01019681
:10A700000E942B8D6DE271E1CE0101960E94B58B06
:10A71000BC01CE014C960E94228DCE014C960E9427
:10A720006C31CE014C960E948C8CCE0101960E9419
:10A730008C8CB2CE6AE57DE0CE0101960E94198D27
:10A74000BE016F5F7F4FCE018E960E94848B182FC3
:10A75000CE0101960E948C8C1123E1F044E050E080
:10A760006DE271E1CE0101960E949D2EBE016F5FE8
:10A770007F4F89E091E10E94538CCE0101960E94A7
:10A780008C8C89E091E10E94EB8A7093D1126093E6
:10A79000D012A2CF61E57DE0CE0101960E94198D15
:10A7A000BE016F5F7F4FCE018E960E94848B182F63
:10A7B000CE0101960E948C8C1123E1F048E050E01C
:10A7C0006DE271E1CE0101960E949D2EBE016F5F88
:10A7D0007F4F89E091E10E94538CCE0101960E9447
:10A7E0008C8C89E091E10E94EB8A7093E81260936F
:10A7F000E71272CF6CE47DE0CE0101960E94198DC4
:10A80000BE016F5F7F4FCE018E960E94848B182F02
:10A81000CE0101960E948C8C1123A1F044E050E0FF
:10A820006DE271E1CE0101960E949D2EBE016F5F27
:10A830007F4F89E091E10E94538CCE0101960E94E6
:10A840008C8C54CF64E47DE0CE0101960E94198D7A
:10A85000BE016F5F7F4FCE018E960E94848B182FB2
:10A86000CE0101960E948C8C1123A1F047E050E0AC
:10A870006DE271E1CE0101960E949D2EBE016F5FD7
:10A880007F4F89E091E10E94538CCE0101960E9496
:10A890008C8CFCCD6CE37DE0CE0101960E94198D7D
:10A8A000BE016F5F7F4FCE018E960E94848B182F62
:10A8B000CE0101960E948C8C1111D8CF62E37DE00D
:10A8C000CE0101960E94198DBE016F5F7F4FCE01B0
:10A8D0008E960E94848B182FCE0101960E948C8C3C
:10A8E000112321F081E00E94AA2DD0CD6BE27DE002
:10A8F000CE0101960E94198DBE016F5F7F4FCE0180
:10A900008E960E94848B182FCE0101960E948C8C0B
:10A91000112319F00E944241B9CD61E27DE0CE01E0
:10A9200001960E94198DBE016F5F7F4FCE018E96FA
:10A930000E94848B182FCE0101960E948C8C1123CB
:10A9400009F483C066E17DE0CE0101960E94198D75
:10A95000BE016F5F7F4FCE018E960E94848B182FB1
:10A96000CE0101960E948C8C112309F452C04AE05A
:10A9700050E06DE271E1CE0101960E949D2EBE0174
:10A980006F5F7F4F89E091E10E94538CCE01019669
:10A990000E948C8C89E091E10E94EB8A0E948F0ECC
:10A9A0000E94420F6093ED0B7093EE0B8093EF0BC0
:10A9B0009093F00B0E94420F6093E70B7093E80BAB
:10A9C0008093E90B9093EA0BCE014C960E94803065
:10A9D00064EA75E0CE0101960E942B8DBE01645E93
:10A9E0007F4FCE0101960E94B58BBC01CE018296AD
:10A9F0000E94228DCE0182960E946C31CE018296F9
:10AA00000E948C8CCE0101960E948C8CCE014C96BB
:10AA100078C24BE050E06DE271E1CE0101960E94F8
:10AA20009D2EBE016F5F7F4F89E091E10E94538CA4
:10AA3000CE0101960E948C8C89E091E10E94EB8A04
:10AA400060587F488F4F9F4FA9CF60E17DE0CE01D6
:10AA500001960E94198DBE016F5F7F4FCE018E96C9
:10AA60000E94848B182FCE0101960E948C8C11239A
:10AA700009F46AC045E050E06DE271E1CE01019653
:10AA80000E949D2EBE016F5F7F4F89E091E10E9481
:10AA9000538CCE0101960E948C8C0E94420F6093D1
:10AAA000ED0B7093EE0B8093EF0B9093F00B89E01E
:10AAB00091E10E94EB8A60936E0270936F02809323
:10AAC0007002909371026093B4127093B5128093E8
:10AAD000B6129093B7122091B3122093500C672BAB
:10AAE000682B692B11F41092500C84EF91E0909335
:10AAF00053028093520264EB71E10E94B12964E633
:10AB000070E080E090E00E94500E61E07DE0CE01B8
:10AB100001960E94198DCE0101960E94BA31CE0194
:10AB200001960E948C8C40916E0250916F02609150
:10AB3000700270917102CE0101960E94B38ACE011B
:10AB400001960E946C31DBC166EF7CE0CE0101967C
:10AB50000E94198DBE016F5F7F4FCE018E960E94BD
:10AB6000848B182FCE0101960E948C8C1123D9F171
:10AB70004AE050E06DE271E1CE0101960E949D2E07
:10AB8000BE016F5F7F4F89E091E10E94538CCE013F
:10AB900001960E948C8C89E091E10E94EB8A6130E1
:10ABA00071058105910519F481E08093B31289E064
:10ABB00091E10E94EB8A672B682B692B11F41092AC
:10ABC000B3128091B3128093500C882309F484CD82
:10ABD0000E94420F6093ED0B7093EE0B8093EF0B8E
:10ABE0009093F00B79CD6DEE7CE0CE0101960E9442
:10ABF000198DBE016F5F7F4FCE018E960E94848BB0
:10AC0000182FCE0101960E948C8C1123A1F048E0F0
:10AC100050E06DE271E1CE0101960E949D2EBE01D1
:10AC20006F5F7F4F89E091E10E94538CCE010196C6
:10AC30000E948C8C61CD67EE7CE0CE0101960E9473
:10AC4000198DBE016F5F7F4FCE018E960E94848B5F
:10AC5000182FCE0101960E948C8C112321F145E022
:10AC600050E06DE271E1CE0101960E949D2EBE0181
:10AC70006F5F7F4F89E091E10E94538CCE01019676
:10AC80000E948C8C89E091E10E94EB8A6130710511
:10AC900021F481E08093510CFFCB672B09F0FCCBB2
:10ACA0001092510CF9CB63EE7CE0CE0101960E942C
:10ACB000198DBE016F5F7F4FCE018E960E94848BEF
:10ACC000182FCE0101960E948C8C112351F163E064
:10ACD00070E08DE291E10E94538B682FCE010196C6
:10ACE0000E94F78CBE016F5F7F4F89E091E10E9467
:10ACF000538CCE0101960E948C8C89E091E10E94D8
:10AD0000F68A89E091E10E94EB8A9B01215031098A
:10AD10002330310508F0C0CB7093E3126093E21248
:10AD2000ABCB6CED7CE0CE0101960E94198DBE018B
:10AD30006F5F7F4FCE018E960E94848B182FCE01BD
:10AD400001960E948C8C112309F46AC066E070E0C1
:10AD50008DE291E10E94538B682FCE0101960E94F3
:10AD6000F78CBE016F5F7F4F89E091E10E94538CA9
:10AD7000CE0101960E948C8C89E091E10E94F68AB6
:10AD800060E089E091E10E94F28B89E091E10E940C
:10AD9000EB8A6B01CB010197039708F07DCB48E06C
:10ADA00050E06DE271E1CE0101960E949D2EBE0140
:10ADB0006F5F7F4F89E091E10E94538CCE01019635
:10ADC0000E948C8C89E091E10E94F68A80910D119D
:10ADD00090910E110997A8F028E030E050E040E093
:10ADE00069E071E1CE0101960E94408DBE016F5F66
:10ADF0007F4F89E091E10E94538CCE0101960E9421
:10AE00008C8CB601B3E0660F771FBA95E1F76853F3
:10AE10007E4E48E050E089E091E10E945F892CCBB2
:10AE200064ED7CE0CE0101960E94198DBE016F5F3A
:10AE30007F4FCE018E960E94848B182FCE010196F3
:10AE40000E948C8C112309F488C06DE574E0CE015A
:10AE500001960E942B8D47E050E0BE01625D7F4F5E
:10AE6000CE014C960E949D2EBE01645E7F4FCE01A6
:10AE700001960E94538CCE014C960E948C8C6BE301
:10AE800075E0CE014C960E942B8DBE01645E7F4F13
:10AE9000CE0101960E94848B182FCE014C960E9401
:10AEA0008C8C112389F141E050E0BE016F5F7F4F30
:10AEB000CE014C960E949D2ECE014C960E94EB8AAC
:10AEC0008B010A5C1F4FCE014C960E948C8C109314
:10AED000E5120093E412109382020093810284EF42
:10AEE00091E0909353028093520264EB71E10E94CF
:10AEF000B12964E670E080E090E00E94500ECE013F
:10AF000001960E948C8CC8CA6DE375E0CE014C9608
:10AF10000E942B8DBE01645E7F4FCE0101960E9480
:10AF2000848B182FCE014C960E948C8C112379F0C3
:10AF300041E050E0BE016F5F7F4FCE014C960E9412
:10AF40009D2ECE014C960E94EB8A8B01BCCFCE0188
:10AF500001960E94EB8A8B01BACF6DEC7CE0CE01AA
:10AF600001960E94198DBE016F5F7F4FCE018E96B4
:10AF70000E94848B182FCE0101960E948C8C112385
:10AF800009F4AAC06DEB75E0CE0101960E942B8DED
:10AF900046E050E0BE016F5F7F4FCE018E960E946B
:10AFA0008FA98C01CE0101960E948C8C980146E0FD
:10AFB00050E0BE01625D7F4FCE0101960E94408D40
:10AFC000CE0101960E94EB8A6B01CE0101960E9490
:10AFD0008C8C6DE574E0CE0101960E942B8DA8014A
:10AFE0004F5F5F4FBE01625D7F4FCE014C960E9466
:10AFF0009D2EBE01645E7F4FCE0101960E94538C50
:10B00000CE014C960E948C8C6BE375E0CE014C9681
:10B010000E942B8DBE01645E7F4FCE0101960E947F
:10B02000848B182FCE014C960E948C8C112321F119
:10B0300041E050E0BE016F5F7F4FCE014C960E9411
:10B040009D2ECE014C960E94EB8A8B010A5C1F4F0D
:10B05000CE014C960E948C8CF6013196EE0FFF1FAC
:10B06000EC54FE4E11830083F601EE0FFF1FED5AE4
:10B07000F34F1183008333CF6DE375E0CE014C961F
:10B080000E942B8DBE01645E7F4FCE0101960E940F
:10B09000848B182FCE014C960E948C8C112379F052
:10B0A00041E050E0BE016F5F7F4FCE014C960E94A1
:10B0B0009D2ECE014C960E94EB8A8B01C9CFCE010A
:10B0C00001960E94EB8A0091550C1091560C01508C
:10B0D0001109060F171FC0CF66EC7CE0CE014C961D
:10B0E0000E94198DBE01645E7F4FCE018E960E9434
:10B0F000848B11E0811115C06FEB7CE0CE010196CD
:10B100000E94198DBE016F5F7F4FCE018E960E9407
:10B11000848B11E0811101C010E0CE0101960E94E4
:10B120008C8CCE014C960E948C8C112309F4F0C1BA
:10B130006AEB75E0CE014C960E942B8D65EB75E0B5
:10B14000CE0101960E942B8DAE01445E5F4FBE0181
:10B150006F5F7F4FCE018E960E9496A8CE0101961A
:10B160000E948C8CCE014C960E948C8C6AEB75E010
:10B17000CE014C960E942B8D67EB75E0CE010196B7
:10B180000E942B8DAE01445E5F4FBE016F5F7F4F0B
:10B19000CE018E960E9496A8CE0101960E948C8CBC
:10B1A000CE014C960E948C8C6AEB75E0CE014C96D9
:10B1B0000E942B8D69EB75E0CE0101960E942B8DCC
:10B1C000AE01445E5F4FBE016F5F7F4FCE018E9632
:10B1D0000E9496A8CE0101960E948C8CCE014C96BE
:10B1E0000E948C8C6DEB75E0CE014C960E942B8DED
:10B1F0006CEB75E0CE0101960E942B8DAE01445E92
:10B200005F4FBE016F5F7F4FCE018E960E9496A862
:10B21000CE0101960E948C8CCE014C960E948C8CA3
:10B220006DEB75E0CE014C960E942B8D63EE76E0BF
:10B23000CE0101960E942B8DAE01445E5F4FBE0190
:10B240006F5F7F4FCE018E960E9496A8CE01019629
:10B250000E948C8CCE014C960E948C8CCE018E96D6
:10B260000E94F68A0E94420F6093F10B7093F20BDA
:10B270008093F30B9093F40B06E010E054E6852ED8
:10B28000912CA12CB12C22242394312C6801B3E001
:10B29000CB0ED11C8AA99BA90197C816D90608F024
:10B2A000FBC8B801CE018E960E94538B682FCE0149
:10B2B0004C960E94F78C7801E2E0EE0EF11C0F5FD5
:10B2C0001F4F9701A801BE01625D7F4FCE0101961D
:10B2D0000E94408DCE0101960E94EB8A2B01CE0187
:10B2E00001960E948C8C6AEB75E0CE0101960E945B
:10B2F0002B8DA701BE016F5F7F4FCE018E960E94FE
:10B300008FA97C01CE0101960E948C8C6DE574E0C2
:10B31000CE0101960E942B8DC20101979DAB8CAB93
:10B320001E141F0424F59701A601BE01625D7F4F24
:10B33000CE0182960E94408DBE016E5D7F4FCE0190
:10B3400001960E94538CCE0182960E948C8CACA9EF
:10B35000BDA9139718F187010F5F1F4FCE0101960A
:10B360000E948C8CCE014C960E948C8C8FCFA601B3
:10B37000BE01625D7F4FCE0182960E949D2EBE016E
:10B380006E5D7F4FCE0101960E94538CCE01829656
:10B390000E948C8CECA9FDA9339700F770E060E067
:10B3A000CE014C960E94538B823509F050C0CE01DD
:10B3B00001960E94EB8A672B682B692BB1F4F2018E
:10B3C000EE0FFF1FE952FD4F11821082F201EE0FC6
:10B3D000FF1FEE0FFF1FE154FD4F82E090E0A0E061
:10B3E000B0E080839183A283B383CE0101960E9453
:10B3F000EB8A613071058105910509F067C0F201A2
:10B40000EE0FFF1FE952FD4F31822082440C551C84
:10B41000440C551CF201E154FD4F80819181A281C1
:10B42000B381181619061A061B0624F08082918231
:10B43000A282B382CE0101960E94EB8A623071052E
:10B4400081059105D4F1F201E154FD4F51C08634DC
:10B4500009F041C0CE0101960E94EB8A672B682B50
:10B46000692B39F4F201EE0FFF1FEC5AFD4F1182E8
:10B470001082CE0101960E94EB8A61307105810530
:10B48000910539F4F201EE0FFF1FEC5AFD4F3182A6
:10B490002082440C551C440C551CF201E154FD4F14
:10B4A00080819181A281B381181619061A061B06A4
:10B4B00024F080829182A282B3820E94420FF20124
:10B4C000E152FD4F60837183828393831E141F04B6
:10B4D0000CF441CF43CF843481F4CE0101960E9415
:10B4E000EB8A440C551C440C551CF201E45AFD4FE8
:10B4F0006083718382839383E0CF843539F7CE01F3
:10B5000001960E94EB8A440C551C440C551C9BCFA1
:10B5100069EB7CE0CE0101960E94198DBE016F5F40
:10B520007F4FCE018E960E94848B082FCE0101960C
:10B530000E948C8C002309F49DC045E050E06DE230
:10B5400071E1CE0101960E949D2EBE016F5F7F4F7B
:10B5500089E091E10E94538CCE0101960E948C8C6F
:10B5600089E091E10E94F68A60E089E091E10E9421
:10B57000F28B6FE375E0CE014C960E942B8D69E053
:10B5800071E1CE0101960E94228DAE014E5D5F4FAA
:10B59000BE01645E7F4FCE0101960E94BAA9182FAA
:10B5A000CE0101960E948C8CCE014C960E948C8C10
:10B5B000112311F40C944C528E010E5D1F4F5EED61
:10B5C000C52E52E1D52E60E4A62E62E0B62EF12CF7
:10B5D000E12CD8016D918D01F60161936F01D501C8
:10B5E0006D935D01CE0101960E941EA8CE010196C9
:10B5F0000E94BA31CE0101960E948C8CB3E0EB160A
:10B60000F10471F06FE375E0CE0101960E942B8D7D
:10B61000CE0101960E94BA31CE0101960E948C8C17
:10B62000EFEFEE1AFE0AF4E0EF16F10491F66DE585
:10B6300074E0CE0101960E942B8DCE0101960E94EE
:10B640006C31CE0101960E948C8C64EB71E180918B
:10B650005202909153020E94B12964E670E080E0AA
:10B6600090E00E94500E61EA7CE0CE0101960E94BB
:10B67000198D65CA6CE97CE0CE0101960E94198D96
:10B68000BE016F5F7F4FCE018E960E94848B082F84
:10B69000CE0101960E948C8C002309F47CC044E00A
:10B6A00050E06DE271E1CE0101960E949D2EBE0137
:10B6B0006F5F7F4F89E091E10E94538CCE0101962C
:10B6C0000E948C8C89E091E10E94F68A60E089E01A
:10B6D00091E10E94F28B40910D1150910E1168E69C
:10B6E0007AE089E091E10E945F896FE375E0CE0125
:10B6F0004C960E942B8D69E071E1CE0101960E946B
:10B70000228DAE014E5D5F4FBE01645E7F4FCE0164
:10B7100001960E94BAA9182FCE0101960E948C8C26
:10B72000CE014C960E948C8C112311F40C944C5237
:10B730008E010E5D1F4F40EEE42E41E1F42E6E01AE
:10B7400086E2C80ED11CD8016D918D01F70161937D
:10B750007F01CE0101960E941EA8CE0101960E9493
:10B760006C31CE0101960E948C8C0C151D0559F789
:10B7700084EF91E0909353028093520264EB71E165
:10B780000E94B12964E670E080E090E00E94500ED3
:10B7900061E97CE06ACF6AE87CE0CE0101960E9414
:10B7A000198DBE016F5F7F4FCE018E960E94848BF4
:10B7B000082FCE0101960E948C8C0023F1F146E007
:10B7C00050E06DE271E1CE0101960E949D2EBE0116
:10B7D0006F5F7F4F89E091E10E94538CCE0101960B
:10B7E0000E948C8C89E091E10E94F68A80910D1173
:10B7F00090910E11892B11F40C944C5289E091E137
:10B800000E94EB8A7093DD126093DC1270933F020A
:10B8100060933E0284EF91E0909353028093520232
:10B8200064EB71E10E94B12964E670E080E090E091
:10B830000E94500E66E77CE018CF6FE67CE0CE01F8
:10B8400001960E94198DBE016F5F7F4FCE018E96CB
:10B850000E94848B082FCE0101960E948C8C0023BD
:10B8600021F162E67CE0CE0101960E94198D44E64A
:10B8700050E06FEF7FEFCE0101960E94162ACE01B5
:10B8800001960E948C8C81E08093E61284EF91E017
:10B89000909353028093520264EB71E10E94B129AC
:10B8A000F0E0E0E019950C944C526AE57CE0CE01A2
:10B8B00001960E94198DBE016F5F7F4FCE018E965B
:10B8C0000E94848B082FCE0101960E948C8C00234D
:10B8D00059F00E94209464E670E080E090E00E94BD
:10B8E000500E61E47CE0C1CE69E37CE0CE010196BC
:10B8F0000E94198DBE016F5F7F4FCE018E960E9410
:10B90000848B082FCE0101960E948C8C002301F1BC
:10B910006FEB75E0CE0101960E942B8D6DEF72E109
:10B92000CE0101960E94B58BBC018FE091E10E948F
:10B930003C8CCE0101960E948C8C6FE071E1CE01AF
:10B9400001960E94228DCE0101960E946C318DC419
:10B9500062E37CE0CE0101960E94198DBE016F5F0B
:10B960007F4FCE018E960E94848B082FCE010196C8
:10B970000E948C8C0023B1F163E27CE08FE091E1C6
:10B980000E94178C69E073E183E093E10E943C8C94
:10B9900063E073E1CE0101960E94228DBE016F5FCC
:10B9A0007F4FCE014C960E94228DCE014C960E9474
:10B9B000ABA9BC018FE091E10E94108CCE014C96A6
:10B9C0000E948C8CCE0101960E948C8C6FE071E1FC
:10B9D000CE0101960E94228DCE0101960E946C310B
:10B9E0000C9445546AE17CE0CE0101960E94198DC9
:10B9F000BE016F5F7F4FCE018E960E94848B082F11
:10BA0000CE0101960E948C8C002331F00E944A42A4
:10BA100010923D020C944C5265E17CE0CE010196FF
:10BA20000E94198DBE016F5F7F4FCE018E960E94DE
:10BA3000848B082FCE0101960E948C8C002309F480
:10BA400041C06DEB75E0CE0101960E942B8D4091B7
:10BA50003111509132118D819E81481B590BBE01CD
:10BA60006F5F7F4F8DE291E10E9448A8AC014F5F6C
:10BA70005F4F6DE271E1CE014C960E949D2EBE019A
:10BA8000645E7F4F89E091E10E94538CCE014C9619
:10BA90000E948C8CCE0101960E948C8C89E091E1F1
:10BAA0000E94EB8A6115710531F481E08093F00208
:10BAB0000E947295ADCF6130710509F0A9CF109247
:10BAC000F002F6CF61E17CE0CE0101960E94198D73
:10BAD000BE016F5F7F4FCE018E960E94848B082F30
:10BAE000CE0101960E948C8C002309F438C143E0FA
:10BAF00050E06DE271E1CE0101960E949D2EBE01E3
:10BB00006F5F7F4F89E091E10E94538CCE010196D7
:10BB10000E948C8C69E071E1CE0101960E94228D19
:10BB2000CE0101960E94D32FCE0101960E948C8CEB
:10BB300084EF91E0909353028093520269E071E1A7
:10BB4000CE0101960E94228DCE0101960E94ABA9E2
:10BB5000BC0189E093E10E943C8CCE0101960E94D9
:10BB60008C8C69E071E1CE0101960E94228DCE019C
:10BB700001960E94ABA9BC0183E093E10E943C8C3A
:10BB8000CE0101960E948C8C40910D1350910E13A2
:10BB900064E772E189E093E10E945F8940910713B5
:10BBA000509108136FE772E183E093E10E945F898F
:10BBB00064EB71E180915202909153020E94B1298D
:10BBC0006AEC75E0CE0101960E942B8D69E071E16F
:10BBD000CE0101960E94B58BBC01CE0182960E94D7
:10BBE000228DCE0101960E948C8C809170129091D2
:10BBF0007112892B39F4BE016E5D7F4F84EB9EE09C
:10BC00000E94408E68EB7BE080E090E00E94500E46
:10BC10008091701290917112029709F087C069E0CB
:10BC200071E1CE0188960E94228D62ED75E0CE0111
:10BC300001960E942B8DCE0101960E949E95CE0109
:10BC400001960E948C8C64EF71E080E090E00E948D
:10BC5000500E65ED75E0CE0101960E942B8DCE0150
:10BC600001960E949E95CE0101960E948C8C6CEDEF
:10BC700075E080E090E00E94500E6EED75E0CE0120
:10BC800001960E942B8DCE0101960E949E95CE01B9
:10BC900001960E948C8C64EF71E080E090E00E943D
:10BCA000500E6CEE75E0CE0101960E942B8DCE01F8
:10BCB00001960E949E95CE0101960E948C8C64EFA5
:10BCC00071E080E090E00E94500E6AEC75E0CE01D9
:10BCD00001960E942B8DBE01685D7F4FCE010196BB
:10BCE0000E94B58BBC01CE014C960E94228DCE01E4
:10BCF00001960E948C8CCE014C960E94F68ABE0161
:10BD0000645E7F4FCE0101960E94228DCE01019686
:10BD10000E949E95CE0101960E948C8CCE014C967D
:10BD20000E948C8CCE0188960E948C8C68EB7BE004
:10BD300080E090E00E94500E64E772E1CE0101962F
:10BD40000E942B8DCE0101960E94D32FCE01019629
:10BD50000E948C8C10923D02CE018296D2C86CE07B
:10BD60007CE0CE0101960E94198DBE016F5F7F4F6E
:10BD7000CE018E960E94848B81111091670ACE01AC
:10BD800001960E948C8C112309F486C044E050E097
:10BD90006DE271E1CE0101960E949D2EBE016F5FA2
:10BDA0007F4F89E091E10E94538CCE0101960E9461
:10BDB0008C8C6AEF75E0CE0101960E942B8D69E0B4
:10BDC00071E1CE0101960E94B58BBC01CE014C966B
:10BDD0000E94228DCE0101960E948C8C809170125F
:10BDE00090917112892B39F4BE01645E7F4F84EB10
:10BDF0009EE00E94408E68E873E180E090E00E943F
:10BE0000500E8091701290917112029759F561E075
:10BE100076E0CE0101960E942B8D80910D119091BC
:10BE20000E11892B19F56AE076E0CE0101960E9489
:10BE30007D8ABE01645E7F4FCE0182960E94228D74
:10BE4000CE0182960E949E95CE0182960E948C8C95
:10BE500068E873E180E090E00E94500ECE01019608
:10BE60000E948C8C10923D020C940655BE016F5FAF
:10BE70007F4FCE0182960E94228DCE0182960E9433
:10BE80009E95CE0182960E948C8C60E777E180E0DF
:10BE900090E00E94500ECDCF68E07CE0CE0101968C
:10BEA0000E94198DBE016F5F7F4FCE018E960E945A
:10BEB000848B81111091670ACE0101960E948C8CAF
:10BEC000112309F462C06DE271E189E091E10E9401
:10BED0003C8C81E080933D026DE271E1CE010196E0
:10BEE0000E94228DCE0101960E94D32FCE01019691
:10BEF0000E948C8C8091701290917112029709F1BE
:10BF000069E071E184EB9EE00E94408E68EB7BE08B
:10BF100080E090E00E94500ECE0101960E9437967C
:10BF2000BE016F5F7F4F8DE291E10E94538CCE0185
:10BF300001960E948C8C60ED77E080E090E00E949A
:10BF4000500E8091701290917112029771F469E015
:10BF500071E1CE0101960E94228DCE0101960E94D0
:10BF60009E95CE0101960E948C8C8091311190910A
:10BF70003211892B09F44CCD65E876E0CE010196AB
:10BF80000E942B8D6DE271E1A2C462E07CE0CE01E3
:10BF900001960E94198DBE016F5F7F4FCE018E9674
:10BFA0000E94848B182FCE0101960E948C8C112345
:10BFB00009F495C18091701290917112019709F066
:10BFC00027CD63E176E0CE0188960E942B8DBE01DD
:10BFD000685D7F4F84EB9EE00E94408E6CE271E0D2
:10BFE00080E090E00E94500ECE0182960E9437962B
:10BFF00064E670E080E090E00E94500E10E000E007
:10C0000025E0C22ED12C3AE0A32EB12C6EE176E0D1
:10C01000CE0101960E942B8D50E040E0BE016F5F83
:10C020007F4FCE0182960E948FA97C01CE0101969E
:10C030000E948C8CA7014F5F5F4FBE016E5D7F4FEA
:10C04000CE0101960E949D2EBE016F5F7F4FCE01F3
:10C0500088960E94538CCE0101960E948C8C8CA5F0
:10C060009DA5892B09F170E060E0CE0188960E94C1
:10C07000538B082E000C990BC0970A97A8F460E226
:10C0800076E0CE0101960E942B8DBE016F5F7F4F3F
:10C09000CE0188960E94848BE82ECE0101960E94E4
:10C0A0008C8CFF24F394E110F12C65EF78E0CE0145
:10C0B00001960E94198D64E170E0CE0101960E9404
:10C0C00074AACE0101960E948C8C0F5F1F4F62E311
:10C0D00070E080E090E00E94500EC801B6010E941E
:10C0E00091B60197C1F4CE0101960E947B338D81F8
:10C0F0009E81892B09F4BEC0BE016F5F7F4F8DE228
:10C1000091E10E943C8C0E943351FF24F394CE01B4
:10C1100001960E948C8CCE0101960E943796BE013A
:10C120006F5F7F4FCE0182960E94538CCE010196A5
:10C130000E948C8C62E370E080E090E00E94500EE0
:10C140000436110519F0FF2009F460CF8091D60B59
:10C150008823F1F065E876E0CE014C960E942B8DA5
:10C16000BE01685D7F4FCE014C960E94B58BBC012D
:10C17000CE0101960E94228DCE0101960E946C3163
:10C18000CE0101960E948C8CCE014C960E948C8C24
:10C190008CA59DA5892B69F070E060E0CE018896A2
:10C1A0000E94538B082E000C990BC0970A9708F435
:10C1B0007AC068E276E0CE0101960E942B8DCE0116
:10C1C00082960E948C8CCE0188960E948C8C8D81E8
:10C1D0009E81009709F449C0E981FA8120812223D8
:10C1E00009F443C0079708F440C069EF7BE0CE0133
:10C1F0004C960E94198D68EC70E0CE014C960E941E
:10C2000074AACE014C960E948C8CBE016F5F7F4F4A
:10C21000CE014C960E94228D40ED57E06FEF7FEFEC
:10C22000CE014C960E94162ACE014C960E948C8C10
:10C2300064E376E0CE014C960E942B8D6DE271E1B5
:10C24000CE014C960E94B58BBC01CE0182960E9415
:10C25000228DCE0182960E946C31CE0182960E9480
:10C260008C8CCE014C960E948C8CCE0101960E9443
:10C270008C8CCECB043111050CF449CFC801B5012B
:10C280000E9491B6892B09F042CFBE01685D7F4FB5
:10C2900084EB9EE00E94408E68EC70E080E090E0CD
:10C2A0000E94500E34CF60E276E0CE0101960E94EB
:10C2B0002B8DBE016F5F7F4FCE0188960E94848BCD
:10C2C000182FCE0101960E948C8C111172CFBE01E5
:10C2D000685D7F4FCE0101960E94108D70CF64EF94
:10C2E0007BE0CE0101960E94198DBE016F5F7F4FEA
:10C2F000CE018E960E94848B182FCE0101960E944B
:10C300008C8C112309F4F7C025E030E044E050E0C4
:10C310006DE271E1CE0101960E94408DBE016F5F1A
:10C320007F4F89E091E10E94538CCE0101960E94DB
:10C330008C8C6DE271E1CE0101960E94228DCE01BE
:10C3400001960E94D32FCE0101960E948C8C89E029
:10C3500091E10E94EB8A6130710509F06EC0709323
:10C3600071126093701264E279E0CE0101960E942E
:10C37000198DCE0101960E94D32FCE0101960E9405
:10C380008C8C62E476E0CE014C960E942B8D63E0AB
:10C3900073E1CE014C960E94B58BBC01CE01019693
:10C3A0000E94228D48EC50E06FEF7FEFCE010196A6
:10C3B0000E945937CE0101960E948C8CCE014C967A
:10C3C0000E948C8C0E9401A840E052EC61E070E079
:10C3D00084EB9EE00E943A8484EF91E090935302B4
:10C3E0008093520281E08093670A64EB71E184EFED
:10C3F00091E00E94B12961E576E0CE014C960E9461
:10C400002B8D6DEF72E1CE014C960E94B58BBC0175
:10C41000CE0101960E94228D40ED57E06FEF7FEF35
:10C42000CE0101960E94162ACE0101960E948C8CA4
:10C43000CE014C960E948C8CEBCA61157105D1F52A
:10C44000109271121092701266E179E0CE0101969D
:10C450000E94198DCE0101960E94D32FCE01019624
:10C460000E948C8C68E476E0CE014C960E942B8D65
:10C4700063E073E1CE014C960E94B58BBC01CE0106
:10C4800001960E94228D48EC50E06FEF7FEFCE01C5
:10C4900001960E945937CE0101960E948C8CCE01E4
:10C4A0004C960E948C8C0E9401A840E855E260E006
:10C4B00070E08ECF62307105A9F4709371126093B1
:10C4C000701265E079E0CE0101960E94198DCE01CF
:10C4D00001960E94D32FCE0101960E948C8C6CE4B1
:10C4E00076E0C2CF77FF94CA1092670A70937112F8
:10C4F000609370128DCA6CEE7BE0CE0101960E94B3
:10C50000198DBE016F5F7F4FCE018E960E94848B86
:10C51000182FCE0101960E948C8C112309F441C082
:10C5200047E050E06DE271E1CE0101960E949D2E40
:10C53000BE016F5F7F4F89E091E10E94538CCE0175
:10C5400001960E948C8C66E276E0CE0101960E94F4
:10C550002B8DBE016F5F7F4F89E091E10E94848B3C
:10C56000182FCE0101960E948C8C111110924F0C45
:10C5700064E275E0CE0101960E942B8DBE016F5FD3
:10C580007F4F89E091E10E94848B182FCE010196A4
:10C590000E948C8C112309F4EFCC81E080934F0C26
:10C5A000EBCC65EE7BE0CE0101960E94198DBE01B9
:10C5B0006F5F7F4FCE018E960E94848B182FCE0125
:10C5C00001960E948C8C112381F146E050E06DE2CF
:10C5D00071E1CE0101960E949D2EBE016F5F7F4FDB
:10C5E00089E091E10E94538CCE0101960E948C8CCF
:10C5F00089E091E10E94E08A6093B8127093B912C9
:10C600008093BA129093BB1284EF91E090935302FF
:10C610008093520264EB71E10E94B12964E670E0FC
:10C6200080E090E00E94500EA7CC6CED7BE0CE0144
:10C6300001960E94198DBE016F5F7F4FCE018E96CD
:10C640000E94848B182FCE0101960E948C8C11239E
:10C6500001F148E050E06DE271E1CE0101960E94E7
:10C660009D2EBE016F5F7F4F89E091E10E94538C48
:10C67000CE0101960E948C8C89E091E10E94E08AB3
:10C680006093BE127093BF128093C0129093C11238
:10C69000BBCF62ED7BE0CE0101960E94198DBE01F9
:10C6A0006F5F7F4FCE018E960E94848B182FCE0134
:10C6B00001960E948C8C112301F149E050E06DE25B
:10C6C00071E1CE0101960E949D2EBE016F5F7F4FEA
:10C6D00089E091E10E94538CCE0101960E948C8CDE
:10C6E00089E091E10E94E08A6093C2127093C312C4
:10C6F0008093C4129093C51287CF68EC7BE0CE0183
:10C7000001960E94198DBE016F5F7F4FCE018E96FC
:10C710000E94848B182FCE0101960E948C8C1123CD
:10C72000F1F049E050E06DE271E1CE0101960E9426
:10C730009D2EBE016F5F7F4F89E091E10E94538C77
:10C74000CE0101960E948C8C89E091E10E94E08AE2
:10C750000E9451B67093C9126093C81255CF6DEB09
:10C760007BE0CE0101960E94198DBE016F5F7F4F65
:10C77000CE018E960E94848B182FCE0101960E94C6
:10C780008C8C1123F1F04AE050E06DE271E1CE01B2
:10C7900001960E949D2EBE016F5F7F4F89E091E15F
:10C7A0000E94538CCE0101960E948C8C89E091E10D
:10C7B0000E94E08A0E9451B67093C7126093C6121D
:10C7C00023CF61EB7BE0CE0101960E94198DBE0163
:10C7D0006F5F7F4FCE018E960E94848B182FCE0103
:10C7E00001960E948C8C112311F14BE050E06DE218
:10C7F00071E1CE0101960E949D2EBE016F5F7F4FB9
:10C8000089E091E10E94538CCE0101960E948C8CAC
:10C8100089E091E10E94E08A0E9451B66093CA12B9
:10C820007093CB128093CC129093CD12EDCE6AEA26
:10C830007BE0CE0101960E94198DBE016F5F7F4F94
:10C84000CE018E960E94848B182FCE0101960E94F5
:10C850008C8C112309F44FC046E050E06DE271E189
:10C86000CE0101960E949D2EBE016F5F7F4F89E031
:10C8700091E10E94538CCE0101960E948C8C89E03C
:10C8800091E10E94EB8A7093BD116093BC1189E025
:10C8900091E10E94EB8A70935C0C60935B0C84EFD7
:10C8A00091E0909353028093520264EB71E10E94F5
:10C8B000B12964E670E080E090E00E94500E66E5E9
:10C8C00076E0CE0101960E942B8D69E071E1CE01E8
:10C8D00001960E94B58BBC01CE014C960E94228D20
:10C8E000CE014C960E946C31CE014C960E948C8CED
:10C8F000CE0101969FCD62EA7BE0CE0101960E94B7
:10C90000198DBE016F5F7F4FCE018E960E94848B82
:10C91000182FCE0101960E948C8C1123B1F147E0B3
:10C9200050E06DE271E1CE0101960E949D2EBE01A4
:10C930006F5F7F4F89E091E10E94538CCE01019699
:10C940000E948C8C89E091E10E94EB8A7093BF1168
:10C950006093BE1189E091E10E94EB8A70935E0CB6
:10C9600060935D0C84EF91E09093530280935202A8
:10C9700064EB71E10E94B12964E670E080E090E030
:10C980000E94500E62E676E09CCF6CE97BE0CE011F
:10C9900001960E94198DBE016F5F7F4FCE018E966A
:10C9A0000E94848B182FCE0101960E948C8C11233B
:10C9B000E1F045E050E06DE271E1CE0101960E94A8
:10C9C0009D2EBE016F5F7F4F89E091E10E94538CE5
:10C9D000CE0101960E948C8C89E091E10E94EB8A45
:10C9E0007093BD126093BC120FCE66E97BE0CE015E
:10C9F00001960E94198DBE016F5F7F4FCE018E960A
:10CA00000E94848B182FCE0101960E948C8C1123DA
:10CA100061F00E94420F6093F10B7093F20B8093D0
:10CA2000F30B9093F40B0C94085D62E97BE0CE016C
:10CA300001960E94198DBE016F5F7F4FCE018E96C9
:10CA40000E94848B182FCE0101960E948C8C11239A
:10CA500089F143E050E0BE01625D7F4FCE01019657
:10CA60000E949D2EBE016F5F7F4F89E091E10E9481
:10CA7000538CCE0101960E948C8C80910D11909167
:10CA80000E11892B41F089E091E10E94EB8A7093AD
:10CA90006D0260936C0280916C0290916D0201971F
:10CAA000029708F469CA81E090E090936D02809348
:10CAB0006C0262CA6BE87BE0CE014C960E94198D35
:10CAC000BE01645E7F4FCE018E960E94848B11E082
:10CAD000811115C068E87BE0CE0101960E94198D96
:10CAE000BE016F5F7F4FCE018E960E94848B11E056
:10CAF000811101C010E0CE0101960E948C8CCE0104
:10CB00004C960E948C8C112309F468C061E87BE08C
:10CB1000CE0101960E94198DBE016F5F7F4FCE013D
:10CB20008E960E94848B182FCE0101960E948C8CC9
:10CB30001123A1F046E050E0BE01625D7F4FCE01BF
:10CB400001960E949D2EBE016F5F7F4F89E091E1AB
:10CB50000E94538CCE0101960E948C8C6EE77BE084
:10CB6000CE0101960E94198DBE016F5F7F4FCE01ED
:10CB70008E960E94848B182FCE0101960E948C8C79
:10CB80001123A1F042E050E0BE01625D7F4FCE0173
:10CB900001960E949D2EBE016F5F7F4F89E091E15B
:10CBA0000E94538CCE0101960E948C8C80910D11B5
:10CBB00090910E11892B09F4DFC969E071E1CE0172
:10CBC00001960E94228D61E070E0CE0101960E94E4
:10CBD000C548CE0101960E948C8CCEC967E77BE0E8
:10CBE000CE0182960E94198DBE016E5D7F4FCE01EF
:10CBF0008E960E94848B11E0811129C06FE67BE044
:10CC0000CE014C960E94198DBE01645E7F4FCE010D
:10CC10008E960E94848B11E0811115C067E67BE03F
:10CC2000CE0101960E94198DBE016F5F7F4FCE012C
:10CC30008E960E94848B11E0811101C010E0CE011C
:10CC400001960E948C8CCE014C960E948C8CCE0159
:10CC500082960E948C8C112309F4E6C060E67BE08A
:10CC6000CE0101960E94198DBE016F5F7F4FCE01EC
:10CC70008E960E94848B182FCE0101960E948C8C78
:10CC8000112309F466C046E050E0BE01625D7F4FAB
:10CC9000CE0101960E949D2EBE016F5F7F4F89E0FD
:10CCA00091E10E94538CCE0101960E948C8C89E008
:10CCB00091E10E94E08A6B017C0120E030E0A90153
:10CCC0000E9487B618160CF08EC0A701960160E08E
:10CCD00070E08AE794E40E94DFB50E9451B6609349
:10CCE000390270933A0280933B0290933C02809108
:10CCF000390290913A02A0913B02B0913C02181681
:10CD000019061A061B0664F081E090E0A0E0B0E08E
:10CD10008093390290933A02A0933B02B0933C0275
:10CD200080916C0290916D028130910509F068C08C
:10CD30008091390290913A02A0913B02B0913C025D
:10CD40008093350290933602A0933702B093380255
:10CD500013C947E050E0BE01625D7F4FCE010196EE
:10CD60000E949D2EBE016F5F7F4F89E091E10E947E
:10CD7000538CCE0101960E948C8C6CE974E0CE013C
:10CD800001960E942B8DBE016F5F7F4FCE018E9664
:10CD90000E94848B182FCE0101960E948C8C112347
:10CDA00031F081E090E090936D0280936C0263ED2E
:10CDB00075E0CE0101960E942B8DBE016F5F7F4F03
:10CDC000CE018E960E94848B182FCE0101960E9470
:10CDD0008C8C112309F46BCF82E090E090936D026C
:10CDE00080936C0264CF81E090E0A0E0B0E080939B
:10CDF000390290933A02A0933B02B0933C0277CF62
:10CE0000029709F0B9C88091390290913A02A09135
:10CE10003B02B0913C028093310290933202A09386
:10CE20003302B0933402A8C86BE57BE0CE014C9688
:10CE30000E94198DBE01645E7F4FCE018E960E94C6
:10CE4000648B11E0811115C064E57BE0CE01019691
:10CE50000E94198DBE016F5F7F4FCE018E960E949A
:10CE6000848B11E0811101C010E0CE0101960E9477
:10CE70008C8CCE014C960E948C8C112309F48EC2AE
:10CE800060E57BE0CE0101960E94198DBE016F5FC7
:10CE90007F4FCE018E960E94848B182FCE01019673
:10CEA0000E948C8C112309F4FCC001E010E0109367
:10CEB0006D0200936C0210934902009348026FE6E2
:10CEC00076E089E091E10E947D8A10934902009307
:10CED000480281E090E0A0E0B0E0809339029093B6
:10CEE0003A02A0933B02B0933C02809335029093A8
:10CEF0003602A0933702B093380269E071E1CE01A7
:10CF000001960E94228D62E070E0CE0101960E949F
:10CF1000C548CE0101960E948C8C6FE37BE0CE0168
:10CF200001960E94198DCE0101960E946C31CE01AE
:10CF300001960E948C8C6FE27BE0CE0101960E94EC
:10CF4000198DCE0101960E942E38CE0101960E94C5
:10CF50008C8C66E276E089E091E10E947D8A69E04E
:10CF600071E1CE0101960E94228D63E070E0CE0156
:10CF700001960E94C548CE0101960E948C8C82E0E9
:10CF800090E090936D0280936C026EE17BE0CE01A5
:10CF900001960E94198DCE0101960E946C31CE013E
:10CFA00001960E948C8C62E17BE0CE0101960E948A
:10CFB000198DCE0101960E942E38CE0101960E9455
:10CFC0008C8C6FE676E089E091E10E947D8A809109
:10CFD000DA129091DB1297FF06C063E776E089E0F2
:10CFE00091E10E947D8A69E071E1CE0101960E9483
:10CFF000228D62E070E0CE0101960E94C548CE010C
:10D0000001960E948C8C66E276E089E091E10E94B4
:10D010007D8A82E090E090936D0280936C0269E0DB
:10D0200071E1CE0101960E94228D63E070E0CE0195
:10D0300001960E94C548CE0101960E948C8C84EF17
:10D0400091E0909353028093520264EB71E10E944D
:10D05000B12964E670E080E090E00E94500E81E02B
:10D0600090E090936D0280936C021092DA0210921D
:10D07000D90282E090E0A0E0B0E08093C3029093F8
:10D08000C402A093C502B093C6020E94420F6093EF
:10D09000E3027093E4028093E5029093E6020C941D
:10D0A000BC5F6DE07BE0CE0101960E94198DBE0150
:10D0B0006F5F7F4FCE018E960E94848B182FCE011A
:10D0C00001960E948C8C11110C94BC5F6BE07BE08C
:10D0D000CE0101960E94198DBE016F5F7F4FCE0178
:10D0E0008E960E94848B182FCE0101960E948C8C04
:10D0F000112331F081E090E090936D0280936C02F7
:10D1000069E07BE0CE0101960E94198DBE016F5F40
:10D110007F4FCE018E960E94848B182FCE010196F0
:10D120000E948C8C112331F082E090E090936D028C
:10D1300080936C0281E090E0A0E0B0E0809339023F
:10D1400090933A02A0933B02B0933C0280916C0210
:10D1500090916D028130910509F099C09093490238
:10D160008093480262E07BE0CE0101960E94198D17
:10D17000BE016F5F7F4FCE018E960E94848B182F69
:10D18000CE0101960E948C8C112319F146E050E0EB
:10D19000BE01625D7F4FCE014C960E949D2E67E7D7
:10D1A00076E0CE0101960E942B8DBE01645E7F4F1A
:10D1B000CE0101960E94B58BBC0189E091E10E94ED
:10D1C0003C8CCE0101960E948C8CCE014C960E9424
:10D1D0008C8C8091390290913A02A0913B02B091DF
:10D1E0003C028093350290933602A0933702B093AD
:10D1F00038026FE676E089E091E10E947D8A69E07D
:10D2000071E1CE0101960E94228D62E070E0CE01B4
:10D2100001960E94C548CE0101960E948C8C61EF58
:10D220007AE0CE0101960E94198DCE0101960E94EE
:10D230006C31CE0101960E948C8C81E090E090933D
:10D2400049028093480266E276E089E091E10E941B
:10D250007D8A69E071E1CE0101960E94228D63E032
:10D2600070E0CE0101960E94C548CE0101960E9451
:10D270008C8C61EE7AE0CE0101960E94198DCE0170
:10D2800001960E942E38CE0101960E948C8C8091CE
:10D290006C0290916D02029711F00C94BC5F6DEDE1
:10D2A0007AE089E091E10E94178C8091DA129091E6
:10D2B000DB1297FF06C069ED7AE089E091E10E94F8
:10D2C000178C01E010E0109349020093480269E0D6
:10D2D00071E1CE0101960E94228D62E070E0CE01E4
:10D2E00001960E94C548CE0101960E948C8C66E290
:10D2F00076E089E091E10E947D8A68EC7AE0CE01D7
:10D3000001960E94198DCE0101960E946C31CE01CA
:10D3100001960E948C8C69E071E1CE0101960E9419
:10D32000228D63E070E0CE0101960E94C548CE01D7
:10D3300001960E948C8C6CEB7AE0CE0101960E94E3
:10D34000198DCE0101960E942E38CE0101960E94C1
:10D350008C8C8091DA129091DB12919581959109D4
:10D360009093DB128093DA121093490200934802E3
:10D3700084EF91E0909353028093520264EB71E149
:10D380000E94B12964E670E080E090E00E94500EB7
:10D3900010936D0200936C020C94BC5F65EB7AE015
:10D3A000CE0188960E94198DBE01685D7F4FCE0127
:10D3B0008E960E94848B01E081113DC062EB7AE081
:10D3C000CE0182960E94198DBE016E5D7F4FCE0107
:10D3D0008E960E94848B01E0811129C06EEA7AE06A
:10D3E000CE014C960E94198DBE01645E7F4FCE0126
:10D3F0008E960E94848B01E0811115C06AEA7AE062
:10D40000CE0101960E94198DBE016F5F7F4FCE0144
:10D410008E960E94848B01E0811101C000E0CE0154
:10D4200001960E948C8CCE014C960E948C8CCE0171
:10D4300082960E948C8CCE0188960E948C8C002350
:10D4400009F41FC263EA7AE0CE0101960E94198DA9
:10D45000BE016F5F7F4FCE018E960E94848B082F96
:10D46000CE0101960E948C8C46E050E0011117C05D
:10D4700069E776E0CE0101960E942B8DBE016F5FB9
:10D480007F4FCE018E960E94848B082FCE0101968D
:10D490000E948C8C002309F48BC042E050E0BE0156
:10D4A000625D7F4FCE0101960E949D2EBE016F5F8F
:10D4B0007F4F89E091E10E94538CCE0101960E943A
:10D4C0008C8C80910D1190910E11892B11F40C947C
:10D4D000BC5F67E776E0CE014C960E942B8DBE01C3
:10D4E000645E7F4F89E091E10E94848B811114C0BA
:10D4F00061EA7AE0CE0101960E94198DBE016F5F4C
:10D500007F4F89E091E10E94848B11E0811110E04E
:10D51000CE0101960E948C8CCE014C960E948C8C80
:10D52000C12CD12C7601112309F46AC189E091E163
:10D530000E94E08A6B017C0180916C0290916D02E7
:10D54000019709F09FC089E091E10E94E08A9B0168
:10D55000AC016091630A7091640A8091650A9091B0
:10D56000660A0E9473B56093630A7093640A80939D
:10D57000650A9093660A8090630A9090640AA0906E
:10D58000650AB090660A20E030E044EB53E4C50140
:10D59000B4010E9487B687FD86C020E030E044EBEE
:10D5A00053E4C501B4010E9472B54B015C01EBCF9D
:10D5B00043E050E0BE01625D7F4FCE0101960E94C4
:10D5C0009D2EBE016F5F7F4F89E091E10E94538CD9
:10D5D000CE0101960E948C8C6CE974E0CE0101961C
:10D5E0000E942B8DBE016F5F7F4FCE018E960E94F1
:10D5F000848B082FCE0101960E948C8C0023B1F001
:10D6000081E090E090936D0280936C028091DF0B3B
:10D610009091E00BA091E10BB091E20B8093630A33
:10D620009093640AA093650AB093660A63ED75E06F
:10D63000CE0101960E942B8DBE016F5F7F4FCE0100
:10D640008E960E94848B082FCE0101960E948C8CAE
:10D65000002309F436CF82E090E090936D0280932E
:10D660006C028091DB0B9091DC0BA091DD0BB091F3
:10D67000DE0B8093630A9093640AA093650AB093CB
:10D68000660A1FCF89E091E10E94E08A9B01AC010C
:10D690006091630A7091640A8091650A9091660AAC
:10D6A0000E9472B560CF20E030E0A901C501B4014D
:10D6B0000E94C5B387FF0BC020E030E044EB53E489
:10D6C000C501B4010E9473B54B015C01ECCF80929F
:10D6D000630A9092640AA092650AB092660A20E0FA
:10D6E00030E0A901C701B6010E9487B687FD15C0C9
:10D6F00063E377E0CE0101960E942B8D69E071E132
:10D70000CE0101960E94B58BBC0189E091E10E9497
:10D710003C8CCE0101960E948C8C20E030E0A90167
:10D72000C701B6010E94C5B387FF6AC080916C0231
:10D7300090916D02019799F520E030E0A901C701B1
:10D74000B6010E9487B618160CF092C020E030E0B7
:10D7500040E251E4C701B6010E9473B522E0AB017B
:10D76000BC01CE014C960E94948C67E776E0CE0116
:10D7700001960E942B8DBE01645E7F4FCE01019603
:10D780000E94B58BBC0189E091E10E943C8CCE01E6
:10D7900001960E948C8CCE014C960E948C8C8091BC
:10D7A0006C0290916D02019759F120E030E0A901DF
:10D7B000C701B6010E9487B6B701A60118160CF082
:10D7C000705822E0CE014C960E94948C67E776E078
:10D7D000CE0101960E942B8DBE01645E7F4FCE016B
:10D7E00001960E94B58BBC0189E091E10E943C8CBE
:10D7F000CE0101960E948C8CCE014C960E948C8C9E
:10D8000081E090E0909349028093480269E071E1E1
:10D81000CE0101960E94228D62E070E0CE01019659
:10D820000E94C548CE0101960E948C8C20E030E019
:10D83000A901C701B6010E94C5B387FD02C00C94BF
:10D84000BC5F80916C0290916D02019711F00C9475
:10D85000BC5F6CE776E089E091E10E947D8A69E037
:10D8600071E1CE0101960E94228D62E070E0ADC9A7
:10D87000A701960160E070E080E291E40E9472B539
:10D880006DCF6BE97AE0CE0182960E94198DBE01C0
:10D890006E5D7F4FCE018E960E94848B11E08111C8
:10D8A00029C064E97AE0CE014C960E94198DBE0130
:10D8B000645E7F4FCE018E960E94848B11E08111B1
:10D8C00015C06DE87AE0CE0101960E94198DBE0167
:10D8D0006F5F7F4FCE018E960E94848B11E0811185
:10D8E00001C010E0CE0101960E948C8CCE014C96B6
:10D8F0000E948C8CCE0182960E948C8C112309F49C
:10D900009BC0CE018E960E94F68A6FE676E089E093
:10D9100091E10E947D8A6CE974E0CE0101960E943B
:10D920002B8DBE016F5F7F4FCE018E960E94848B40
:10D93000182FCE0101960E948C8C112331F081E0CA
:10D9400090E090936D0280936C0263ED75E0CE01E0
:10D9500001960E942B8DBE016F5F7F4FCE018E9688
:10D960000E94848B182FCE0101960E948C8C11236B
:10D9700091F082E090E090936D0280936C02809130
:10D98000DA129091DB1297FF06C069E87AE089E02D
:10D9900091E10E94178C81E090E09093490280937E
:10D9A000480269E071E1CE0101960E94228D62E099
:10D9B00070E0CE0101960E94C548CE0101960E94FA
:10D9C0008C8C63E87AE0CE0101960E94198DBE012D
:10D9D0006F5F7F4FCE018E960E94848B182FCE01F1
:10D9E00001960E948C8C45E050E0111102C046E087
:10D9F00050E0BE01625D7F4FCE0101960E949D2ED8
:10DA0000BE016F5F7F4F89E091E10E94538CCE0190
:10DA100001960E948C8C80910D1190910E11892B92
:10DA200011F40C94BC5F69E071E1CE0101960E9493
:10DA3000228D63E070E0C9C86DE77AE0CE0182967E
:10DA40000E94198DBE016E5D7F4FCE018E960E94A1
:10DA5000848B11E0811129C066E77AE0CE014C96F3
:10DA60000E94198DBE01645E7F4FCE018E960E948A
:10DA7000848B11E0811115C06FE67AE0CE0101962A
:10DA80000E94198DBE016F5F7F4FCE018E960E945E
:10DA9000848B11E0811101C010E0CE0101960E943B
:10DAA0008C8CCE014C960E948C8CCE0182960E946A
:10DAB0008C8C112309F426C169E67AE0CE01019627
:10DAC0000E94198DBE016F5F7F4FCE018E960E941E
:10DAD000848B182FCE0101960E948C8C112309F49F
:10DAE00043C045E050E0BE01625D7F4FCE0101962C
:10DAF0000E949D2EBE016F5F7F4F89E091E10E94E1
:10DB0000538CCE0101960E948C8C80910D119091C6
:10DB10000E11892B61F089E091E10E94E08A609307
:10DB2000630A7093640A8093650A9093660AC090B2
:10DB3000630AD090640AE090650AF090660A20E0DB
:10DB400030E044EB53E4C701B6010E9487B687FD7D
:10DB500055C020E030E044EB53E4C701B6010E9419
:10DB600072B56B017C01EBCF46E050E0BE01625D17
:10DB70007F4FCE0101960E949D2EBE016F5F7F4FA9
:10DB800089E091E10E94538CCE0101960E948C8C19
:10DB90006CE974E0CE0101960E942B8DBE016F5F8F
:10DBA0007F4FCE018E960E94848B182FCE01019656
:10DBB0000E948C8C112331F081E090E090936D02F3
:10DBC00080936C0263ED75E0CE0101960E942B8D6F
:10DBD000BE016F5F7F4FCE018E960E94848B182FFF
:10DBE000CE0101960E948C8C112309F48ECF82E025
:10DBF00090E090936D0280936C0287CF20E030E03C
:10DC0000A901C701B6010E94C5B387FF0BC020E080
:10DC100030E044EB53E4C701B6010E9473B56B01D9
:10DC20007C01ECCFC092630AD092640AE092650A4C
:10DC3000F092660A80916C0290916D02019771F4E6
:10DC4000C092DF0BD092E00BE092E10BF092E20B7E
:10DC50006EE57AE08FE091E10E94178C8091630A73
:10DC60009091640AA091650AB091660A20916C02B5
:10DC700030916D022230310571F48093DB0B90936B
:10DC8000DC0BA093DD0BB093DE0B67E57AE08FE051
:10DC900091E10E94178C4091630A5091640A60914F
:10DCA000650A7091660A21E0CE014C960E94948C20
:10DCB0006FE071E1CE0101960E94228DBE01645E8B
:10DCC0007F4FCE0101960E94B58B68E575E00E94FA
:10DCD0009F8BBC018FE091E10E943C8CCE010196AC
:10DCE0000E948C8CCE014C960E948C8C6FE071E16E
:10DCF000CE0101960E94228DCE0101960E942E38FF
:10DD00000C94E96562E57AE0CE0182960E94198D55
:10DD1000BE016E5D7F4FCE018E960E94848B11E016
:10DD2000811129C06CE47AE0CE014C960E94198DD5
:10DD3000BE01645E7F4FCE018E960E94848B11E0FF
:10DD4000811115C066E47AE0CE0101960E94198D1A
:10DD5000BE016F5F7F4FCE018E960E94848B11E0D3
:10DD6000811101C010E0CE0101960E948C8CCE0181
:10DD70004C960E948C8CCE0182960E948C8C112332
:10DD800009F412C2C0903902D0903A02E0903B02EE
:10DD9000F0903C0261E47AE0CE0101960E94198D78
:10DDA000BE016F5F7F4FCE018E960E94848B182F2D
:10DDB000CE0101960E948C8C112309F465C044E0C9
:10DDC00050E0BE01625D7F4FCE0101960E949D2E04
:10DDD000BE016F5F7F4F89E091E10E94538CCE01BD
:10DDE00001960E948C8C80916C0290916D02813022
:10DDF000910509F093C0C0903502D0903602E090B2
:10DE00003702F090380281E090E0A0E0B0E080932B
:10DE1000350290933602A0933702B0933802809176
:10DE20000D1190910E11892B09F090C06BE37AE0EF
:10DE300089E091E10E94178C80910D1190910E1153
:10DE4000892B81F069E071E1CE0101960E94228D5B
:10DE500070E060E0CE0101960E94C548CE010196B7
:10DE60000E948C8C80916C0290916D0281309105A2
:10DE700009F08CC1C0923502D0923602E09237028E
:10DE8000F09238020C94BC5F45E050E0BE01625D48
:10DE90007F4FCE0101960E949D2EBE016F5F7F4F86
:10DEA00089E091E10E94538CCE0101960E948C8CF6
:10DEB0006CE974E0CE0101960E942B8DBE016F5F6C
:10DEC0007F4FCE018E960E94848B182FCE01019633
:10DED0000E948C8C112331F081E090E090936D02D0
:10DEE00080936C0263ED75E0CE0101960E942B8D4C
:10DEF000BE016F5F7F4FCE018E960E94848B182FDC
:10DF0000CE0101960E948C8C112309F46CCF82E023
:10DF100090E090936D0280936C0265CF029709F0B8
:10DF20007ECFC0903102D0903202E0903302F09068
:10DF3000340281E090E0A0E0B0E080933102909361
:10DF40003202A0933302B093340269CF60E876E0E6
:10DF5000CE0101960E942B8DBE016F5F7F4F89E03D
:10DF600091E10E94648B182FCE0101960E948C8C47
:10DF7000112309F477CF89E091E10E94E08A20E043
:10DF800030E0A9010E94C5B3811128C080916C02C4
:10DF900090916D02019731F466E37AE089E091E1B6
:10DFA0000E94178C80916C0290916D02029731F45F
:10DFB00060E37AE089E091E10E94178C80910D1175
:10DFC00090910E11892B09F44DCF69E071E1CE01DA
:10DFD00001960E94228D61E070E03CCF6DEB75E010
:10DFE000CE0101960E942B8DBE016F5F7F4F89E0AD
:10DFF00091E10E94648B182FCE0101960E948C8CB7
:10E00000112309F42FCF41E050E069E071E1CE0126
:10E0100001960E949D2ECE0101960E94E08A4B013E
:10E020005C01CE0101960E948C8C20E030E0A901B9
:10E03000C501B4010E94C5B3181634F0812C912C8F
:10E0400090E8A92E9FE3B92E00916C0210916D0209
:10E050000130110509F075C0A501940160E070E47C
:10E060008CE995E40E94DFB560932D0270932E0237
:10E0700080932F02909330026093D2127093D31248
:10E080008093D4129093D5126093290270932A0240
:10E0900080932B0290932C02B801CE014C960E94E3
:10E0A000878A63E876E0CE0101960E942B8DBE013F
:10E0B000645E7F4FCE0101960E94B58BBC01CE01FC
:10E0C00082960E94228DCE0182960E94BA31CE01A4
:10E0D00082960E948C8CCE0101960E948C8CCE017F
:10E0E0004C960E948C8C6EE17AE0CE0101960E94E3
:10E0F000198DCE0101960E94BA31CE0101960E947F
:10E100008C8C40912D0250912E0260912F027091C3
:10E11000300225E0CE0101960E94948CCE0101963A
:10E120000E946C31CE0101960E948C8C84EF91E0AC
:10E13000909353028093520264EB71E10E94B129E3
:10E1400091CE0230110509F0A7CFA501940160E03E
:10E1500070E48CE196E40E94DFB560932D02709329
:10E160002E0280932F02909330026093D612709308
:10E17000D7128093D8129093D9126093250270938E
:10E180002602809327029093280286CF029711F0EF
:10E190000C94BC5FC0923102D0923202E092330202
:10E1A000F09234020C94BC5F69E17AE0CE01829671
:10E1B0000E94198DBE016E5D7F4FCE018E960E942A
:10E1C000848B11E0811129C063E17AE0CE014C9685
:10E1D0000E94198DBE01645E7F4FCE018E960E9413
:10E1E000848B11E0811115C06DE07AE0CE010196BB
:10E1F0000E94198DBE016F5F7F4FCE018E960E94E7
:10E20000848B11E0811101C010E0CE0101960E94C3
:10E210008C8CCE014C960E948C8CCE0182960E94F2
:10E220008C8C112309F429C18AA99BA9059710F4A4
:10E230000C94BC5F44E050E0BE01625D7F4FCE01B4
:10E2400001960E949D2EBE016F5F7F4F89E091E194
:10E250000E94538CCE0101960E948C8C68E07AE07B
:10E26000CE0101960E94198DBE016F5F7F4FCE01D6
:10E270008E960E94848B182FCE0101960E948C8C62
:10E28000112309F49BC044E050E0BE01625D7F4F62
:10E29000CE0101960E949D2EBE016F5F7F4F89E0E7
:10E2A00091E10E94538CCE0101960E948C8C89E0F2
:10E2B00091E10E94E08A20E030E0A9010E9487B647
:10E2C000181614F00C94BC5F89E091E10E94E08A7A
:10E2D00060932D0270932E0280932F029093300250
:10E2E00020916C0230916D022130310509F0B0C0EF
:10E2F0006093D2127093D3128093D4129093D5125C
:10E300006093290270932A0280932B0290932C022F
:10E31000B901CE014C960E94878A63E876E0CE016F
:10E3200001960E942B8DBE01645E7F4FCE01019647
:10E330000E94B58BBC01CE0182960E94228DCE0137
:10E3400082960E94BA31CE0182960E948C8CCE01B8
:10E3500001960E948C8CCE014C960E948C8C66EFAC
:10E3600079E0CE0101960E94198DCE0101960E949E
:10E37000BA31CE0101960E948C8C40912D025091B1
:10E380002E0260912F027091300225E0CE0101969D
:10E390000E94948CCE0101960E946C31CE010196B0
:10E3A0000E948C8C84EF91E09093530280935202F0
:10E3B00064EB71E10E94B1290C94BC5F45E050E030
:10E3C000BE01625D7F4FCE0101960E949D2EBE016F
:10E3D0006F5F7F4F89E091E10E94538CCE010196DF
:10E3E0000E948C8C6CE974E0CE0101960E942B8D0A
:10E3F000BE016F5F7F4FCE018E960E94848B182FD7
:10E40000CE0101960E948C8C112331F081E090E0C6
:10E4100090936D0280936C0263ED75E0CE010196DE
:10E420000E942B8DBE016F5F7F4FCE018E960E94A2
:10E43000848B182FCE0101960E948C8C112309F435
:10E4400036CF82E090E090936D0280936C022FCFE4
:10E450002230310509F05CCF6093D6127093D71249
:10E460008093D8129093D91260932502709326025C
:10E4700080932702909328024BCF63EF79E0CE017F
:10E480004C960E94198DBE01645E7F4FCE018E9620
:10E490000E94848B11E0811115C06FEE79E0CE01EE
:10E4A00001960E94198DBE016F5F7F4FCE018E963F
:10E4B0000E94848B11E0811101C010E0CE01019611
:10E4C0000E948C8CCE014C960E948C8C112309F4F6
:10E4D00063C06CEE79E0CE0101960E94198DBE01F9
:10E4E0006F5F7F4FCE018E960E94848B182FCE01D6
:10E4F00001960E948C8C112399F042E050E06DE26D
:10E5000071E1CE0101960E949D2EBE016F5F7F4F8B
:10E5100089E091E10E94538CCE0101960E948C8C7F
:10E5200068EE79E0CE0101960E94198DBE016F5F01
:10E530007F4FCE018E960E94848B182FCE010196BC
:10E540000E948C8C112399F043E050E06DE271E160
:10E55000CE0101960E949D2EBE016F5F7F4F89E024
:10E5600091E10E94538CCE0101960E948C8C89E02F
:10E5700091E10E94EB8A653B710510F40C94BC5F3D
:10E5800065ED79E0CE0101960E94198DCE010196CC
:10E590000E94BA310C94E96561ED79E0CE010196F3
:10E5A0000E94198DBE016F5F7F4FCE018E960E9433
:10E5B000848B182FCE0101960E948C8C112309F4B4
:10E5C00074C026E030E044E050E06DE271E1CE013D
:10E5D00001960E94408DBE016F5F7F4F89E091E1FF
:10E5E0000E94538CCE0101960E948C8C6DEB75E0DD
:10E5F000CE0101960E942B8D409131115091321124
:10E600008D819E81481B590BBE016F5F7F4F8DE24C
:10E6100091E10E9448A8AC014F5F5F4F6DE271E14C
:10E62000CE014C960E949D2EBE01645E7F4F89E014
:10E6300091E10E94538CCE014C960E948C8CCE01AD
:10E6400001960E948C8C89E091E10E94E08A88E228
:10E65000EBE3FAE0ABE8B2E101900D928A95E1F7C5
:10E6600084EF91E0909353028093520264EB71E146
:10E670000E94B12960EB79E08FE091E10E94178C54
:10E6800044E050E06DE271E1CE0101960E949D2EC2
:10E69000BE016F5F7F4F8FE091E10E94108CCE0131
:10E6A00001960E948C8C0C949D5C68EA79E0CE0106
:10E6B00001960E94198DBE016F5F7F4FCE018E962D
:10E6C0000E94848B182FCE0101960E948C8C111110
:10E6D0000C94906261EA79E0CE0101960E94198D56
:10E6E000BE016F5F7F4FCE018E960E94848B182FE4
:10E6F000CE0101960E948C8C112371F141E068E9F2
:10E7000072E0CE0101960E947391BE016F5F7F4F50
:10E710008BE193E10E94792D8BE193E10E94421DF0
:10E720006DE279E0882311F40C94355B8BE193E181
:10E730000E94100C892B51F08BE193E10E94B718D5
:10E74000682F81E59FE00E949C82F0CF8BE193E1EE
:10E750000E944E1D0C944C5268E979E0CE0101965E
:10E760000E94198DBE016F5F7F4FCE018E960E9471
:10E77000848B182FCE0101960E948C8C1123E9F016
:10E780008DB79EB7855391400FB6F8949EBF0FBECC
:10E790008DBFADB7BEB7119685E391E0E4EBF1E133
:10E7A00001900D920197E1F70E9473440FB6F8941F
:10E7B000DEBF0FBECDBF0C944C5262E979E0CE01B2
:10E7C00001960E94198DBE016F5F7F4FCE018E961C
:10E7D0000E94848B182FCE0101960E948C8C1123ED
:10E7E00009F457C0EDB7FEB7E553F1400FB6F89402
:10E7F000FEBF0FBEEDBFADB7BEB7119685E391E08A
:10E80000E4EBF1E101900D920197E1F70E94DA3C0F
:10E810000FB6F894DEBF0FBECDBF61E879E0CE0140
:10E8200001960E94198DADB7BEB7A553B1400FB682
:10E83000F894BEBF0FBEADBF119685E391E0E4EB47
:10E84000F1E101900D920197E1F70E94C5340FB6F6
:10E85000F894DEBF0FBECDBF8DB79EB785539140F4
:10E860000FB6F8949EBF0FBE8DBFADB7BEB7119661
:10E8700085E391E0E4EBF1E101900D920197E1F77E
:10E880000E9473440FB6F894DEBF0FBECDBF0C9448
:10E890007F576DE779E0CE0101960E94198DBE0188
:10E8A0006F5F7F4FCE018E960E94848B182FCE0112
:10E8B00001960E948C8C1123F9F06AE679E0CE0172
:10E8C00001960E94198DBE016F5F7F4FCE014C965D
:10E8D0000E94228DCE014C960E946C31CE014C9646
:10E8E0000E948C8CEDB7FEB7E553F1400FB6F8945B
:10E8F000FEBF0FBEEDBFB9CF66E679E0CE0101964F
:10E900000E94198DBE016F5F7F4FCE018E960E94CF
:10E91000848B182FCE0101960E948C8C112309F450
:10E92000F5C06AE379E0CE0182960E94198DBE019E
:10E930006E5D7F4FCE0101960E94228DAE014F5F2A
:10E940005F4F62E070E082E792E00E949C3E8C01A3
:10E95000CE0101960E948C8C012B11F5BE016E5DDB
:10E960007F4FCE014C960E94228D67E876E0CE0163
:10E970004C960E949F8B60E671E10E94B58BBC01B2
:10E98000CE0101960E94228DCE0101960E946C312B
:10E99000CE0101960E948C8CCE014C960E948C8CEC
:10E9A00068EE73E080E090E00E94500EBE016E5D64
:10E9B0007F4FCE0101960E94228DAE014F5F5F4FC7
:10E9C00063E070E083E892E00E949C3E8C01CE01FF
:10E9D00001960E948C8C012B11F5BE016E5D7F4F5C
:10E9E000CE014C960E94228D67E976E0CE014C96CE
:10E9F0000E949F8B60E671E10E94B58BBC01CE0145
:10EA000001960E94228DCE0101960E946C31CE01AA
:10EA100001960E948C8CCE014C960E948C8C68EEE4
:10EA200073E080E090E00E94500E64E571E1CE0159
:10EA300001960E94228DAE014F5F5F4F61E070E052
:10EA400082EB92E00E949C3E8C01CE0101960E94D6
:10EA50008C8C012B09F564E571E1CE014C960E9486
:10EA6000228D67E976E0CE014C960E949F8B60E68E
:10EA700071E10E94B58BBC01CE0101960E94228DEE
:10EA8000CE0101960E946C31CE0101960E948C8CC1
:10EA9000CE014C960E948C8C68EE73E080E090E092
:10EAA0000E94500E80914F0C882311F40C94AC5EA0
:10EAB00043E162EB72E0CE0101960E947391BE01C8
:10EAC0006F5F7F4F81E593E10E94792D81E593E1AE
:10EAD0000E94421D882311F40C94AC5E64E571E140
:10EAE00081E593E10E944E8E66E970E080E090E05F
:10EAF0000E94500E81E593E10E944E1D62E370E09A
:10EB000080E090E00E94500E0C94AC5E62E679E0EA
:10EB1000CE0101960E94198DBE016F5F7F4FCE011D
:10EB20008E960E94848B182FCE0101960E948C8CA9
:10EB30001123A9F005E51CE0D8018C910E5F1F4F51
:10EB400060E00E94CC0D6CE271E080E090E00E94F9
:10EB5000500EBCE00B351B0779F70C944C526DE559
:10EB600079E0CE0101960E94198DBE016F5F7F4F43
:10EB7000CE018E960E94848B182FCE0101960E94A2
:10EB80008C8C1123C1F005E51CE08BE5E82E8CE0B0
:10EB9000F82EF80180810E5F1F4F61E00E94CC0DBE
:10EBA0006CE271E080E090E00E94500EE016F10609
:10EBB00081F70C944C5266E579E0CE0101960E94F3
:10EBC000198DBE016F5F7F4FCE018E960E94848BA0
:10EBD000182FCE0101960E948C8C112311F40C94F5
:10EBE0004C5227E030E046E050E06DE271E1CE01AA
:10EBF00001960E94408DBE016F5F7F4F89E091E1D9
:10EC00000E94538CCE0101960E948C8C89E091E188
:10EC10000E94EB8A672B71F41092D60B6DE271E1C2
:10EC2000CE0101960E94228DCE0101960E94D32F23
:10EC30000C94356181E08093D60BF0CF2F923F92F8
:10EC40004F925F926F927F928F929F92AF92BF92FC
:10EC5000CF92DF92EF92FF920F931F93CF93DF93A8
:10EC600000D000D01F921F92CDB7DEB76091810215
:10EC70007091820280917F02909180020E94802A8E
:10EC800084E1482E512C612C712C312C212C8FEFDA
:10EC9000281A380AC301B2010E94500E6091810205
:10ECA0007091820280917F02909180020E94802A5E
:10ECB0008C0183E02816310434F08EE128163104EB
:10ECC00044F4012B51F084E1480E511C611C711C6D
:10ECD000DECF0115110509F0A6C080917F02909149
:10ECE00080028B30910509F086C08090ED129090E3
:10ECF000EE12A090EF12B090F012C090E912D090F6
:10ED0000EA12E090EB12F090EC1264E670E080E022
:10ED100090E00E94500E6BE776E0CE0101960E94D3
:10ED2000198DCE0101960E942E38CE0101960E94C7
:10ED30008C8C61E082E00E940D8421E0B501A40189
:10ED4000CE0101960E94948CBE016F5F7F4F8DE6CD
:10ED500093E10E94408ECE0101960E948C8C6FED53
:10ED60008DE693E10E942B0F66E776E08DE693E156
:10ED70000E94608E20E0B701A601CE0101960E949C
:10ED8000948CBE016F5F7F4F8DE693E10E94408EB1
:10ED9000CE0101960E948C8C63EA76E08DE693E1C9
:10EDA0000E94388E89829A82AB82BC82CD82DE82BA
:10EDB000EF82F88629813A814B815C816D817E8169
:10EDC0008F81988528960FB6F894DEBF0FBECDBF11
:10EDD000DF91CF911F910F91FF90EF90DF90CF9037
:10EDE000BF90AF909F908F907F906F905F904F906B
:10EDF0003F902F9008958631910509F476CF0C97B6
:10EE000009F083CF8090640990906509A09066090D
:10EE1000B0906709C0906009D0906109E0906209E4
:10EE2000F090630972CF0F3F8FEF1807CCF068E6C0
:10EE300076E0CE0101960E94198D4AE050E070E024
:10EE400060E0CE0101960E945937CE0101960E94E2
:10EE50008C8C65E476E08FE091E10E94178C32C0E3
:10EE60000E3F8FEF1807B9F167E376E0CE01019608
:10EE70000E94198D4AE050E070E060E0CE010196FA
:10EE80000E945937CE0101960E948C8C68E276E090
:10EE90008FE091E10E94178CB801CE0101960E948B
:10EEA000878ABE016F5F7F4F8FE091E10E94108CD7
:10EEB000CE0101960E948C8C62E176E08FE091E1B8
:10EEC0000E94C88B19821A821B821C821D821E829C
:10EED0001F8218866FCF67E076E0CE0101960E9410
:10EEE000198D4AE050E070E060E0CE0101960E948A
:10EEF0005937CE0101960E948C8C67EE75E0ABCF3E
:10EF00002F923F924F925F926F927F928F929F9239
:10EF1000AF92BF92CF92DF92EF92FF920F931F9327
:10EF2000CF93DF93CDB7DEB7AC970FB6F894DEBFC3
:10EF30000FBECDBF8C017B018091D90B9091DA0B74
:10EF400001969093DA0B8093D90B2091F50B222335
:10EF500041F06AE070E00E9491B6181619060CF4B0
:10EF6000C0C281E08093F50B1092DA0B1092D90B9E
:10EF700050E040E069E374E0C8010E94582E82E04E
:10EF8000E816F10409F4C6C26DE574E08EE491E17F
:10EF90000E947D8A609181027091820280917F023D
:10EFA000909180020E94802A1C0162E17EE0C801EB
:10EFB0000E943F2E65EA76E0C8010E94388E67EF16
:10EFC00072E1CE0101960E94228DBE016F5F7F4FDC
:10EFD000C8010E94408ECE0101960E948C8C6EEA80
:10EFE00076E0C8010E94388E6BE677E0C8010E9487
:10EFF000608E6DEF72E1CE0101960E94228DBE01FE
:10F000006F5F7F4FC8010E94408E61E677E0C801C4
:10F010000E94608E6CE072E1CE0109960E942B8DF9
:10F02000BE01675F7F4FC8010E94408E64E577E0B4
:10F03000C8010E94608E64E772E1CE010F960E94C3
:10F040002B8DBE01615F7F4FC8010E94408E6DE431
:10F0500077E0C8010E94608ECE010F960E948C8CD2
:10F06000CE0109960E948C8CCE0101960E948C8C58
:10F070000E94830E28EE33E040E050E00E940FB57E
:10F0800029013A0163E477E0C8010E94608ECE0155
:10F0900001960E948030BE016F5F7F4FC8010E94C1
:10F0A000408ECE0101960E948C8CC301B20120E1FA
:10F0B0003EE040E050E00E9431B54B015C01B901F7
:10F0C000CE0187960E94A92E4CE3C42ED12CE12CB0
:10F0D000F12CC501B401A70196010E9431B5B90117
:10F0E000CE0101960E94A92E6FE476E0CE0109962A
:10F0F0000E942B8DBE016F5F7F4FCE0109960E944B
:10F10000B58BBC01CE0187960E94108CCE0109966A
:10F110000E948C8CCE0101960E948C8CC301B2019E
:10F12000A70196010E9431B5CE0101960E94A92E39
:10F130006FE476E0CE0109960E942B8DBE016F5FD1
:10F140007F4FCE0109960E94B58BBC01CE018796F8
:10F150000E94108CCE0109960E948C8CCE010196E3
:10F160000E948C8C64EB76E0CE0109960E942B8D78
:10F17000BE01695D7F4FCE0109960E94B58B67EB9A
:10F1800076E00E949F8BBC01CE0101960E94228DE9
:10F19000BE016F5F7F4FC8010E94408ECE01019675
:10F1A0000E948C8CCE0109960E948C8C65EC76E0D6
:10F1B000C8010E94388ECE0101960E949529B8019F
:10F1C000CE0101960E94D88D60EC76E0C8010E94C5
:10F1D000268E0E941E7629833A834B835C836D833F
:10F1E0007E838F83988749815A816B817C8121E05E
:10F1F000CE010F960E94948CBE01615F7F4FCE01BD
:10F2000009960E94228D6DEC76E0CE0109960E944F
:10F210009F8BBC018EE491E10E943C8CCE0109964B
:10F220000E948C8CCE010F960E948C8C64ED76E04F
:10F23000CE010F960E942B8D6EE471E1CE010F96E8
:10F240000E94B58BBC01CE0109960E94228DBE01A1
:10F25000675F7F4FC8010E94408ECE0109960E94D1
:10F260008C8CCE010F960E948C8C4D815E816F81BB
:10F27000788521E0CE0109960E94948CBE01675FDB
:10F280007F4F8EE491E10E94538CCE0109960E943B
:10F290008C8C66EE76E0CE010F960E942B8D6EE48C
:10F2A00071E1CE010F960E94B58B67EF76E00E9468
:10F2B0009F8BBC01CE0109960E94228DBE01675F23
:10F2C0007F4FC8010E94408ECE0109960E948C8C0F
:10F2D000CE010F960E948C8C4091DF0B5091E00B79
:10F2E0006091E10B7091E20B22E0CE010F960E943B
:10F2F000948C6EEF76E0CE0145960E942B8DBE0178
:10F30000615F7F4FCE0145960E94B58B60E177E04B
:10F310000E949F8BBC01CE0109960E94228DBE01E6
:10F32000675F7F4FC8010E94408ECE0109960E9400
:10F330008C8CCE0145960E948C8CCE010F960E943B
:10F340008C8C4091DB0B5091DC0B6091DD0B70914C
:10F35000DE0B22E0CE010F960E94948C69E177E0EB
:10F36000CE0145960E942B8DBE01615F7F4FCE017D
:10F3700045960E94B58B60E177E00E949F8BBC01AF
:10F38000CE0109960E94228DBE01675F7F4FC801A2
:10F390000E94408ECE0109960E948C8CCE0145962B
:10F3A0000E948C8CCE010F960E948C8CE6EF2E165C
:10F3B000EFEF3E062CF46DE07FE0C8010E943F2E87
:10F3C0006AEE7DE0C8010E943F2E94EBE92E91E1A8
:10F3D000F92E27EDA22E22E0B22ECC24C394D12CFC
:10F3E0004701F8E08F0E911C82E0A80EB11C8091BD
:10F3F000B4119091B5118C159D050CF464C0B60143
:10F40000CE010F960E94878A65E876E0CE01459688
:10F410000E942B8DBE01615F7F4FCE0145960E94F9
:10F42000B58B6AEB75E00E949F8BBC01CE010996FB
:10F430000E94228DBE01675F7F4FC8010E94408EEF
:10F44000B701645E7F4FCE014B960E942B8DBE01AB
:10F45000655E7F4FC8010E94408E67E277E0C80179
:10F460000E94388EF50160817181660F771F660FEB
:10F47000771F60547E4ECE0181960E942B8DBE0177
:10F480006F5D7F4FC8010E94408E6CE277E0C8013B
:10F490000E94388ECE0181960E948C8CCE014B96B4
:10F4A0000E948C8CCE0109960E948C8CCE014596D0
:10F4B0000E948C8CCE010F960E948C8CFFEFCF1A8D
:10F4C000DF0A74018DCFCE0187960E948C8C81E07B
:10F4D0008093520C6BEC7EE0C8010E943F2E10928C
:10F4E000F50BAC960FB6F894DEBF0FBECDBFDF9123
:10F4F000CF911F910F91FF90EF90DF90CF90BF9031
:10F50000AF909F908F907F906F905F904F903F90C3
:10F510002F9008956DE07FE0C8010E943F2EDACF62
:10F520008F929F92AF92BF92CF92DF92EF92FF9213
:10F530000F931F93CF93DF93CDB7DEB7A0970FB68E
:10F54000F894DEBF0FBECDBF6DE574E088E791E1B2
:10F550000E947D8A6DE574E08CE691E10E947D8ACF
:10F5600040E6842E42E0942E54EBC52E51E1D52E78
:10F5700061EDA62E62E0B62E77EDE72E72E0F72E53
:10F5800001E010E0F40181919191A191B1914F01BD
:10F59000892B8A2B8B2B89F5F70182819381F501C9
:10F5A000208131818217930741F10130110559F40F
:10F5B0002091E7123091E81237FF05C082309105A3
:10F5C0000CF409C30197880F991FFC01E55AF34F0A
:10F5D000D801AA0FBB1FAD5AB34F60818C910E9416
:10F5E000CC0DF70182819381F5019183808364E6DC
:10F5F00070E080E090E00E94500EF5016191719101
:10F600005F018091B4119091B511801791070CF4AE
:10F61000E7C2CE0145960E94878AB801CE010F96B7
:10F620000E94878AB601645E7F4FCE0109960E94D0
:10F630002B8D6AEB75E0CE0101960E942B8DBE01E9
:10F64000675F7F4FCE0101960E94B58B62E377E042
:10F650000E949F8BBE01615F7F4F0E94B58B6DEB57
:10F6600075E00E949F8BBE016B5E7F4F0E94B58B41
:10F67000BC0188E791E10E94108CCE0101960E94A6
:10F680008C8CCE0109960E948C8CCE010F960E9424
:10F690008C8CCE0145960E948C8C0F5F1F4FF8E03A
:10F6A000CF0ED11C22E0E20EF11C0430110509F04E
:10F6B00069CFE091CE12F091CF12EE0FFF1FE15310
:10F6C000FD4F60817181CE0101960E94878A46E0DC
:10F6D00050E0BE016F5F7F4FCE0109960E94253139
:10F6E000BE01675F7F4F8CE691E10E94108CCE01D6
:10F6F00009960E948C8CCE0101960E948C8CE09120
:10F70000D012F091D112EE0FFF1FE153FD4F608137
:10F710007181CE0101960E94878A46E050E0BE01C9
:10F720006F5F7F4FCE0109960E942531BE01675F52
:10F730007F4F8CE691E10E94108CCE0109960E94C9
:10F740008C8CCE0101960E948C8C6AEB75E0CE0108
:10F7500045960E942B8D0E94830E28EE33E040E0F8
:10F7600050E00E940FB569017A016DE574E0CE01A9
:10F770004B960E942B8D6DE574E08EE791E10E941F
:10F780007D8ACE0101960E94803044E150E0BE01A6
:10F790006F5F7F4FCE0109960E942531BE01675FE2
:10F7A0007F4F8EE791E10E94538CCE0109960E9413
:10F7B0008C8CCE0101960E948C8C2AE0B701A601A8
:10F7C000CE0109960E94CA8C48E050E0BE01675FF6
:10F7D0007F4FCE010F960E9425316EE771E1CE0179
:10F7E00001960E94228DBE01615F7F4FCE0101967E
:10F7F0000E94B58BBC0182E791E10E943C8CCE0156
:10F8000001960E948C8CCE010F960E948C8CCE01AA
:10F8100009960E948C8C2AE0B701A601CE010996B8
:10F820000E94CA8C65E377E0CE0101960E942B8D81
:10F83000BE01675F7F4FCE0101960E94B58BBE016E
:10F840006B5E7F4F0E94B58BBC018EE791E10E94F9
:10F85000108CCE0101960E948C8CCE0109960E94DC
:10F860008C8C4091DF0B5091E00B6091E10B70911B
:10F87000E20B21E0CE0101960E94948CBE016F5FE5
:10F880007F4FCE014B960E94538CCE0101960E9471
:10F890008C8C6CE377E0CE0101960E942B8DBE012B
:10F8A000655E7F4FCE0101960E94B58BBE016B5EF7
:10F8B0007F4F0E94B58BBC018EE791E10E94108CB6
:10F8C000CE0101960E948C8CBE01655E7F4FCE01F9
:10F8D00001960E94228D46E050E0BE016F5F7F4F8F
:10F8E000CE0109960E942531BE01675F7F4F82E7F6
:10F8F00091E10E94108CCE0109960E948C8CCE0161
:10F9000001960E948C8C4091DB0B5091DC0B609136
:10F91000DD0B7091DE0B21E0CE0101960E94948CEC
:10F92000BE016F5F7F4FCE014B960E94538CCE017C
:10F9300001960E948C8C6AE477E0CE0101960E94C9
:10F940002B8DBE01655E7F4FCE0101960E94B58B67
:10F95000BE016B5E7F4F0E94B58BBC018EE791E1CB
:10F960000E94108CCE0101960E948C8CBE01655EB7
:10F970007F4FCE0101960E94228D46E050E0BE01ED
:10F980006F5F7F4FCE0109960E942531BE01675FF0
:10F990007F4F82E791E10E94108CCE0109960E9470
:10F9A0008C8CCE0101960E948C8C609181027091AA
:10F9B000820280917F02909180020E94802A90931F
:10F9C000EC0B8093EB0B892B71F0609181027091AD
:10F9D000820280917F02909180020E94802A9093FF
:10F9E000EC0B8093EB0B8091EB0B9091EC0B8C3F2D
:10F9F0009F4F0CF415C10E941E7629833A834B83D6
:10FA00005C836D837E838F83988749815A816B8164
:10FA10007C8121E0CE0109960E94948CBE01675F33
:10FA20007F4FCE014B960E94538CCE0109960E94C7
:10FA30008C8C64E577E0CE0109960E942B8DBE0187
:10FA4000655E7F4FCE0109960E94B58BBE016B5E4D
:10FA50007F4F0E94B58BBC018EE791E10E94108C14
:10FA6000CE0109960E948C8CBE01655E7F4FCE014F
:10FA700009960E94228D46E050E0BE01675F7F4FED
:10FA8000CE010F960E942531BE01615F7F4F82E754
:10FA900091E10E94108CCE010F960E948C8CCE01B9
:10FAA00009960E948C8C4D815E816F81788521E062
:10FAB000CE0109960E94948CBE01675F7F4FCE01F4
:10FAC0004B960E94538CCE0109960E948C8C6FE558
:10FAD00077E0CE0109960E942B8DBE01655E7F4FB7
:10FAE000CE0109960E94B58BBE016B5E7F4F0E94CE
:10FAF000B58BBC018EE791E10E94108CCE01099676
:10FB00000E948C8CBE01655E7F4FCE0109960E94DB
:10FB1000228D46E050E0BE01675F7F4FCE010F9619
:10FB20000E942531BE01615F7F4F82E791E10E9413
:10FB3000108CCE010F960E948C8CCE0109960E94EB
:10FB40008C8C68E771E18EE791E10E94108C6AEB82
:10FB500075E0CE0101960E942B8D6CE671E1CE011D
:10FB600001960E94B58BBC0182E791E10E94108C46
:10FB7000CE0101960E948C8C62E771E1CE01019664
:10FB80000E94228DCE0101960E946C31CE01019619
:10FB90000E948C8C6AE070E080E090E00E94500E41
:10FBA000CE014B960E948C8CCE0145960E948C8C87
:10FBB000A0960FB6F894DEBF0FBECDBFDF91CF91F8
:10FBC0001F910F91FF90EF90DF90CF90BF90AF907B
:10FBD0009F908F9008959801281B390BC901F3CC91
:10FBE000CE0145960E94878AB801CE010F960E94E9
:10FBF000878AB6016C5E7F4FCE0109960E942B8DDD
:10FC00006AEB75E0CE0101960E942B8DBE01675F05
:10FC10007F4FCE0101960E94B58B61E377E018CD4E
:10FC200065E677E08EE791E10E94068C64E777E075
:10FC300082E791E10E94068C6BE777E08EE791E125
:10FC40000E94068C64E777E082E791E10E94068CCF
:10FC500078CFBF92CF92DF92EF92FF920F931F93D4
:10FC6000CF93DF93CDB7DEB7C455D1090FB6F89463
:10FC7000DEBF0FBECDBF6C018B0165965FAF4EAF8F
:10FC800065978091D90B9091DA0B01969093DA0BDE
:10FC90008093D90B8091F50B81113CC0BB24B394A8
:10FCA000B092F50B1092DA0B1092D90B6DE574E05F
:10FCB000CE01895B9F4F0E942B8D6DE574E0CE01D4
:10FCC000835B9F4F0E942B8D50E040E069E374E01E
:10FCD000C6010E94582E0130110509F0A6C06DE53D
:10FCE00074E08EE791E10E947D8A6596EEADFFADEE
:10FCF00065978081811124C00E94907AB092520C45
:10FD0000CE01835B9F4F0E948C8CCE01895B9F4FFD
:10FD10000E948C8C0FB6F894DEBF0FBECDBFCC5ABC
:10FD2000DF4F0FB6F894DEBF0FBECDBFDF91CF918E
:10FD30001F910F91FF90EF90DF90CF90BF900895AB
:10FD40006596EEADFFAD65978081882309F467C0A5
:10FD500000E210E09E012F5F3F4F40E250E0BE0105
:10FD60006F5D7F4FCE018D5A9F4F0E947E84049716
:10FD700039F3BE016F5D7F4FCE018F5B9F4F0E94B5
:10FD80002B8DBE016F5B7F4FCE01895B9F4F0E9421
:10FD9000538CCE018F5B9F4F0E948C8CBE016F5F96
:10FDA0007F4FCE018F5B9F4F0E942B8DBE016F5BFB
:10FDB0007F4FCE01835B9F4F0E94538CCE018F5BA0
:10FDC0009F4F0E948C8CBE01695B7F4F8EE791E153
:10FDD0000E94108C63968EAD9FAD6397892B09F4BA
:10FDE000AFCF6DEB75E0CE018F5B9F4F0E942B8DE7
:10FDF000BE01635B7F4FCE018F5B9F4F0E94B58B2F
:10FE00006AEB75E00E949F8BBC018EE791E10E9436
:10FE1000108CCE018F5B9F4F0E948C8C91CF6EE730
:10FE200071E18AE591E10E943C8C1092F50B68CF5C
:10FE30000895AF92BF92CF92DF92EF92FF920F930D
:10FE40001F93CF93DF936C017B018B01040F151F70
:10FE5000EB015E01AE18BF08C017D10759F06991D8
:10FE6000D601ED91FC910190F081E02DC60119952C
:10FE7000892B79F7C501DF91CF911F910F91FF90E9
:10FE8000EF90DF90CF90BF90AF900895FC01538D1D
:10FE9000448D252F30E0842F90E0821B930B541764
:10FEA00010F0CF9608950197089584EB9EE00E948C
:10FEB000C00921E0892B09F420E0822F089581E513
:10FEC0009FE00E94C00921E0892B09F420E0822FE5
:10FED0000895CF92DF92EF92FF92CF93DF938091BC
:10FEE0005F10883050F0CFEFDFEFCE01DF91CF9180
:10FEF000FF90EF90DF90CF900895E0918410E11192
:10FF000042C00E94830E6B017C0128EEC20E23E0EA
:10FF1000D21EE11CF11C83E590E10E94122588238A
:10FF200011F38091BA10882331F08091851090915F
:10FF30008610892BC1F283E590E10E947523EC01C4
:10FF4000CF3FDC0771F08091BA10882371F2809165
:10FF5000851090918610019790938610809385105C
:10FF6000C4CF0E94830EC616D706E806F90698F697
:10FF70001092841083E590E10E946D2583E590E165
:10FF80000E943425B2CFE150E0938410F0E0E75BAB
:10FF9000FF4EC38DD0E0A9CF0F931F93CF93DF9374
:10FFA000EC018C01F80181918F018823A1F10E945D
:10FFB000697FF8012291022E000C330B8217930700
:10FFC00089F38F3F980781F0A091841091E09A0FF8
:10FFD00090938410B0E0A75BBF4E5B968C939032F9
:10FFE00019F48FE1809384102FE1EC17FD07C9F01D
:10FFF00092919F3FD1F3A091841081E08A0F80936A
:020000021000EC
:100000008410B0E0A75BBF4E5B969C93803269F78B
:1000100020938410EACF81E0DF91CF911F910F915F
:10002000089580E0F9CF8F929F92AF92BF92CF92C6
:10003000DF92EF92FF92CF932AEF3FE03093450C8F
:100040002093440C882309F46DC040E060E070E028
:10005000CB010E94C81381110BC080E0CF91FF90AB
:10006000EF90DF90CF90BF90AF909F908F900895CA
:1000700080911D0E8F7789F78091290E90912A0E1D
:10008000A0912B0EB0912C0E84369105A105B105DF
:1000900020F3C090250ED090260EE090270EF09011
:1000A000280EC114D104E104F104B9F240E0C70103
:1000B000B6010E94C813882381F280916A0C909146
:1000C0006B0C8115924049F6A0916F0CAA2329F27E
:1000D00060916D0C70916E0C6115710509F4BDCFC6
:1000E00020916C0C222309F4B8CFA0931810209310
:1000F0000A1090E080E030E0E1E0F0E0C82FAF01CE
:10010000082E02C0440F551F0A94E2F72417350742
:1001100069F041E0480F01968930910579F74093E5
:1001200013109BCFC12CD12C7601C0CF809313101C
:100130002091750C3091760C50E040E0211531058E
:1001400041F42091830C3091840C4091850C5091A6
:10015000860C20930B1030930C1040930D1050938D
:100160000E1046015701860E971EA11CB11C8092ED
:10017000191090921A10A0921B10B0921C10E091CE
:10018000700CF091710CF0931F10E0931E10B0E012
:100190000E9450B5DC01CB01880D991DAA1DBB1D25
:1001A0008093201090932110A0932210B0932310DD
:1001B00025E0EE0FFF1F2A95E1F7E150FE4FEF2FEC
:1001C000FF27E6958E0F9F1FA11DB11D8093141070
:1001D00090931510A0931610B09317108090720C86
:1001E0009090730CB12CA12C8114910441F4809057
:1001F0007F0C9090800CA090810CB090820CC81A5B
:10020000D90AEA0AFB0AC80CD91CEA1CFB1C04C068
:10021000F694E794D794C794CA95D2F7C0920F107A
:10022000D0921010E0921110F092121085EFC816C3
:100230008FE0D806E104F10428F48CE080931D10CF
:1002400081E00CCF80E125EFC2162FEFD206E1044A
:10025000F104A0F380918B0C90918C0CA0918D0CEB
:10026000B0918E0C8093201090932110A0932210B7
:10027000B093231080E2E2CF5F926F927F928F92D1
:100280009F92AF92BF92CF92DF92EF92FF920F9325
:100290001F93CF93DF93CDB7DEB7C754D1090FB605
:1002A000F894DEBF0FBECDBF5C013B0119A218A2BE
:1002B00082E993E09F8F8E8F1BA21C821B829A8300
:1002C00089831E8210E000E06E018EE1C80ED11C11
:1002D00084E2E82E80E1F82EF501E00FF11F808125
:1002E0008F3211F40F5F1F4FD501A00FB11FFE0118
:1002F000FB9690E080E04F012D912F3249F02223B0
:1003000039F00F5F1F4F019621938C309105A1F7B3
:10031000880D991DFC011082F501E00FF11F80810D
:100320008F3211F40F5F1F4FF501E00FF11F508066
:1003300041E0511040E030E020E0B401C701F3019A
:100340001995811121C0F4E2EF16F0E1FF06C1F426
:1003500080E0C95BDF4F0FB6F894DEBF0FBECDBFA4
:10036000DF91CF911F910F91FF90EF90DF90CF9091
:10037000BF90AF909F908F907F906F905F90089507
:10038000C7010E941419E4CF552091F021E0A40187
:10039000B701C6010E942819982E84E2E81680E170
:1003A000F80681F0C7010E941419911010C0D0CF37
:1003B00094E2E91690E1F90619F0C7010E941419B8
:1003C00081E0C7CF992021F2FE0131967F019E2D59
:1003D0008F2D7601C92ED82E7FCF1092430C10920C
:1003E000420C1092900E1092B20E0E945E1088E89D
:1003F0009BE09093410C8093400C89E89BE09093A4
:100400003F0C80933E0C0895FB0101900020E9F71A
:100410003197AF01461B570BDC01ED91FC91028037
:10042000F381E02D19940E94CEB80F931F93CF93C0
:10043000DF93EC0188819981009759F02A813B81F3
:100440002617370730F081E0DF91CF911F910F9190
:1004500008958B016F5F7F4F0E94EDB7009759F0B1
:10046000998388831B830A832C813D81232B59F731
:10047000FC011082E8CF80E0E7CFEF92FF920F936C
:100480001F93CF93DF936115710541F480E0DF91F5
:10049000CF911F910F91FF90EF9008954115510555
:1004A000B1F07B01EC010C811D81040F151FB80117
:1004B0000E941582882351F3288139818C819D8186
:1004C000B701820F931F0E941EB91D830C8381E028
:1004D000DECFCF93DF93EC0188819981009711F0F3
:1004E0000E9464B7198218821D821C821B821A82A4
:1004F000DF91CF910895EF92FF920F931F93CF93C7
:10050000DF93EC017B018A01BA010E9415828111FF
:100510000BC0CE010E946982CE01DF91CF911F9165
:100520000F91FF90EF9008951D830C83B701888190
:1005300099810E941EB9F0CFEF92FF920F931F9303
:10054000CF93DF93EC0181E0888F9B8D8C8D981386
:100550001AC0E889F989808185FF15C09FB7F89492
:10056000EE89FF896083E889F989808183708064DE
:1005700080839FBF81E090E0DF91CF911F910F9129
:10058000FF90EF900895F62E0B8D10E00F5F1F4F38
:100590000F731127E02E8C8D8E110CC00FB607FC47
:1005A000FACFE889F989808185FFF5CFCE010E94D5
:1005B000810DF1CFEB8DEC0FFD2FF11DE35AFF4FB5
:1005C000F0829FB7F8940B8FEA89FB898081806263
:1005D000CFCFCF93DF93EC01888D8823B9F0AA8920
:1005E000BB89E889F9898C9185FD03C0808186FDEE
:1005F0000DC00FB607FCF7CF8C9185FFF2CF80813D
:1006000085FFEDCFCE010E94810DE9CFDF91CF9123
:1006100008958CBD9DBD08958F929F92AF92BF9219
:10062000CF92DF92EF92FF920F931F93CF93DF93BE
:10063000D091B20ED13208F0D7C0182FC091B10EB0
:100640000E942B0E6B017C018091890E81116BC081
:1006500082E08093890E1093880E8FEF8093870E2F
:100660001092860ED093850EA1E9BEE0E5E6FEE08D
:1006700080E0D81391C01092640E8091640ECC0F6C
:10068000C82BC093640E8091630E813009F088C03E
:100690001092630E0E942B0E6B017C018091640E00
:1006A0008093BB0080918B0E90918C0EA0918D0E4B
:1006B000B0918E0E892B8A2B8B2BA1F00E942B0ED2
:1006C00000918B0E10918C0E20918D0E30918E0E1C
:1006D0006C197D098E099F09061717072807390726
:1006E00008F442C08091BC0083FDD8CF85EC809394
:1006F000BC000E942B0E6B017C018091890E823020
:1007000009F450C08091870E8F3F09F46FC080912B
:10071000870E803209F46CC08091870E803309F413
:1007200069C084E026C080918B0E90918C0EA091C0
:100730008D0EB0918E0E892B8A2B8B2B09F484CFD2
:100740000E942B0E80908B0E90908C0EA0908D0EA0
:10075000B0908E0E6C197D098E099F09861697063A
:10076000A806B90608F070CF80918A0E0E947C100E
:1007700085E01092900E1092B20E10928F0EDF91C3
:10078000CF911F910F91FF90EF90DF90CF90BF908E
:10079000AF909F908F9008959D9191938F5F69CFB7
:1007A00085EEA5CF80918B0E90918C0EA0918D0E31
:1007B000B0918E0E892B8A2B8B2B09F49ECF0E9431
:1007C0002B0E00918B0E10918C0E20918D0E30917E
:1007D0008E0E6C197D098E099F09061717072807C9
:1007E000390708F08ACFC0CF81E0C3CF80E0C1CF06
:1007F00082E0BFCF83E0BDCFCF93C82F682F607F4B
:100800008DE693E10E94120F80E1C89FB001112490
:100810008DE693E1CF910C94120FCF93DF9300D02C
:1008200000D01F921F92CDB7DEB798E0E1E3F3E06E
:10083000DE01119601900D929A95E1F79091761351
:10084000961708F46FEF70E0660F771F21E030E035
:100850002C0F3D1F620F731FFB019081890F806871
:1008600028960FB6F894DEBF0FBECDBFDF91CF91B3
:100870000C94FC83CF93DF93EC019A01AB01E889E0
:10088000F98982E08083211581EE38074105510501
:1008900081F160E079E08DE390E00E940FB5215096
:1008A0003109410951095695479537952795EC85AA
:1008B000FD851082EE85FF852083188EEC89FD89E9
:1008C00086E08083EA89FB89808180618083EA8970
:1008D000FB89808188608083EA89FB8980818068C8
:1008E0008083EA89FB8980818F7D8083DF91CF912E
:1008F0000895E889F989108220E1D9CF2F923F929B
:100900004F925F926F927F928F929F92AF92BF921F
:10091000CF92DF92EF92FF920F931F93CF93DF93CB
:1009200000D0CDB7DEB71C013B014A0129015801B7
:10093000FC01C080D18070E060E0C3010E9403B977
:10094000A80170E060E0C2010E9403B9F601808155
:1009500010E000E0811162C004E010E004C0760104
:10096000F101F182E082C8010F900F900F90DF91AA
:10097000CF911F910F91FF90EF90DF90CF90BF909C
:10098000AF909F908F907F906F905F904F903F902F
:100990002F9008956B3209F482C06D3309F04EC078
:1009A00081818823E9F2F7018FEFE81AF80A608164
:1009B000653209F452C00CF048C0662309F456C0F1
:1009C00082E0A816B1040CF061C0012B09F46BC0E1
:1009D00003E010E0E8CF81818983882309F28281D6
:1009E0008A837601811104C0F2E0EF0EF11CB8CFCA
:1009F00083E0E80EF11C1B8240E150E070E060E013
:100A0000CE0101960E9488AB19C0F3016083F1E02A
:100A10008F1A9108C30101963C0167017601FFEF2F
:100A2000EF1AFF0AF6016081663209F499CF0CF0E3
:100A3000B1CF662309F493CF653269F2F2E08F16E5
:100A400091041CF701E010E0E8CF663209F488CF8A
:100A50006B3209F0B5CF60E2B3CF818189838823FF
:100A600001F182818A83811103C032967F0178CFA0
:100A70007F0193E0E90EF11C1B8240E150E070E041
:100A800060E0CE0101960E9488AB9ACFF2016083AC
:100A9000F1E0AF1AB108C20101962C0184CF60E2E7
:100AA000CDCFF701E3CF02E010E07DCFAF92BF9250
:100AB000CF92DF92EF92FF920F931F93CF93DF932A
:100AC000C82FD62F1092F1121092F2121092F31238
:100AD0001092F4121092F51261E00E94FA0D60E09B
:100AE0008C2F0E94CC0D6D2F70E090E080E00E9472
:100AF000500E60E08C2F0E94FA0D8BE990E0019778
:100B0000F1F700E911E08C2F0E94A30D892B81F4ED
:100B100001501109C1F78EEF9FEFDF91CF911F9127
:100B20000F91FF90EF90DF90CF90BF90AF9008951E
:100B300000E911E08C2F0E94A30D019721F40150D0
:100B40001109C1F7E8CF18E2D0E800E090E9E92EFA
:100B5000FF24F3948C2F0E94A30D892B29F481E0AC
:100B6000E81AF108B9F7D7CF0E942B0E6B017C0170
:100B700080E9A82EBB24B3948C2F0E94A30D01976B
:100B800029F481E0A81AB108B9F7C5CF0E942B0E4D
:100B90006C197D098E099F096932710581059105DE
:100BA00038F0E02FF0E0E751FD4E80858D2B8087F7
:100BB000D69511F40F5FD0E8115041F690E080E037
:100BC000ACCF0F931F93CF93DF93EC010E94830E62
:100BD0008B010E9422128F3F69F00E94830E601BDE
:100BE000710B6C177D07A8F380E0DF91CF911F9107
:100BF0000F91089581E0F9CFCF93DF93EC016E85DB
:100C00007F858889998941E00E94C813882351F023
:100C10008A8920E2829FC0011124815A934FDF917B
:100C2000CF91089590E080E0FACF8F929F92AF929B
:100C3000BF92CF92DF92EF92FF920F931F93CF93C9
:100C4000DF9300D01F92CDB7DEB7FC0185818130E4
:100C500091F080E00F900F900F900F90DF91CF9167
:100C60001F910F91FF90EF90DF90CF90BF90AF90CA
:100C70009F908F900895848181FFEBCF8389948921
:100C8000A589B689892B8A2B8B2B09F45EC07F013D
:100C900040E050E0BA01CF010E940B168823C9F250
:100CA000F701C38CD48C8788908CA18CB28C82E0A5
:100CB00090E0A0E0B0E0F60180839183A283B3834B
:100CC0009E012F5F3F4FB501A401C6010E94B314DE
:100CD000882309F4BECF00E010E09801B501A4011B
:100CE000C6010E941114882309F4B3CF89809A8029
:100CF000AB80BC80F6018789803111F188EF9FEFCE
:100D0000AFEFBFE088169906AA06BB06C8F2F70146
:100D1000178A108E118E128E138A148A158A168ADB
:100D2000848180688483C7010E94E518882309F4C0
:100D300090CF40E050E0BA01C7010E940B168ACF65
:100D400088EF9FEFA0E0B0E0DDCF81E083CF4F924E
:100D50005F926F927F928F929F92AF92BF92CF924B
:100D6000DF92EF92FF920F931F93CF93DF93CDB754
:100D7000DEB763970FB6F894DEBF0FBECDBF7C0120
:100D80006B013A01FB0120E090E080E06AE03191E4
:100D9000332309F461C040ED430F4A3008F04DC0E1
:100DA000689FA001699F500D1124CA01C097830F4D
:100DB000911D37FD9A958F3F910549F340F3F70157
:100DC000428153816481758180911C1490911D141E
:100DD000A0911E14B0911F14481759076A077B078A
:100DE00009F40DC28701085F1F4F0E94830E6F70C8
:100DF00077277C5FC8010E94C526813009F004C2B4
:100E000080E394E09A838983F70182819381A481AE
:100E1000B5818B839C83AD83BE8345E350E0BE01E7
:100E20006F5F7F4FC8010E944E27892BA9F5D12CF7
:100E3000C12CC8010E94F12317C03E3209F0BFCF78
:100E4000233009F4BCCFD301A20FB11D12968C93AD
:100E50002F5F90E080E09BCF233009F0B0CFF3010B
:100E60008583CC24C394D12CC60163960FB6F89425
:100E7000DEBF0FBECDBFDF91CF911F910F91FF90CD
:100E8000EF90DF90CF90BF90AF909F908F907F902A
:100E90006F905F904F9008950E94830EF7017783C3
:100EA000668342E050E0B7016A5F7F4FC8010E944D
:100EB000E32681E090E09A83898342E050E0BE011E
:100EC0006F5F7F4FC8010E94E32680E091E09A8324
:100ED000898342E050E0BE016F5F7F4FC8010E94EE
:100EE000E3261A82198242E050E0BE016F5F7F4F15
:100EF000C8010E94E32642E050E0BE016F5F7F4FD1
:100F0000C8010E94E32642E050E0BE016F5F7F4FC0
:100F1000C8010E94E3265601F6018081882301F171
:100F20006501F60181912F01882311F08E32B1F411
:100F300046018A189B081814190474F48D8641E040
:100F400050E0BE01635F7F4FC8010E94E326A40109
:100F5000B501C8010E94E3265201DECF6201E1CF54
:100F60001D8641E050E0BE01635F7F4FC8010E94D3
:100F7000E326C12CDD24D394DA82C98242E050E01A
:100F8000BE016F5F7F4FC8010E94E326DA82C982EB
:100F900042E050E0BE016F5F7F4FC8010E94E32630
:100FA000C8010E941D27892B09F441CFF3E0AF2E21
:100FB000B12C230122E0420E511CD4C0F701428122
:100FC000538164817581808D918DA28DB38D481779
:100FD00059076A077B0709F008C1848D958DC5976D
:100FE00009F003C181A192A15DEFC52EDD24DA9441
:100FF0000C970CF4ADC04CE050E0BE016F5F7F4F2A
:10100000C8010E94D0228B819C819827892798272C
:101010009A8B898BF7014681578129813A81421742
:10102000530709F0E7C097FFE5C08F7092703BEF60
:10103000C32EDD24DA94892B09F08AC06F8078846E
:101040007624672476242AEFC22EDD24DA946114F4
:10105000710409F47DC0D12CC12C8D819E8198270B
:1010600089279827C816D906F8F441E050E0BE0158
:10107000635F7F4FC8010E94D0224D85442331F029
:1010800050E070E060E0C8010E94D0228D8581119F
:10109000ECCF44E050E070E060E0C8010E94D02254
:1010A000FFEFCF1ADF0AD9CF912C812C41E050E01D
:1010B000BE016D5E7F4FC8010E94D0224B89842FF4
:1010C000807C09F06CC0442331F050E070E060E0B7
:1010D000C8010E94D0228B898111E8CF42E050E004
:1010E000BE01615F7F4FC8010E94D02242E050E004
:1010F000BE01635F7F4FC8010E94D02244E050E0F0
:1011000070E060E0C8010E94D02242E050E0BE01E1
:101110006F5E7F4FC8010E94D0228F8598894989D0
:101120005A898115914009F043C0CD84DE84DC24C6
:10113000CD24DC2481E0C816D104D1F541155440FA
:1011400009F04AC044E050E0B201C8010E94D02238
:1011500021E0A21AB10809F46CCEFFEFCF16DF062A
:1011600009F067CE0E94830E3B014C01C8010E942A
:101170001923181619060CF421CF0E94830E661944
:10118000770988099909693873418105910548F5FE
:1011900062E370E080E090E00E94500EE7CF41E013
:1011A00050E070E060E0C8010E94D0221B8A93CF1B
:1011B00054274527542770E060E0C8010E94D022E0
:1011C000FFEF8F1A9F0A6814790409F06FCF96EF2A
:1011D000C92EDD24DA94BCCFE7EFCE2EDD24DA94DD
:1011E000B7CFCC24CA94DC2CB3CF6EEFC62EDD244F
:1011F000DA94AECF4CEFC42EDD24DA94A9CF8EEF73
:10120000C82EDD24DA9430CED12CC12C2DCEEF9215
:10121000FF920F931F93CF93DF93EC010E94420F35
:101220007E01EE0CFF1CEE0CFF1CF701E152FD4F9E
:101230006083718382839383CC0FDD1FFE01E952AB
:10124000FD4F808191811816190644F4FE01E15387
:10125000FD4F808191811816190654F1FE01E95263
:10126000FD4F01E010E011830083FE01ED5AF34FC2
:1012700060915D0C80810E94CC0DC153DD4F1983BC
:101280000883F701E154FD4F88E097E0A0E0B0E06B
:1012900080839183A283B38364EF71E080E090E068
:1012A000DF91CF911F910F91FF90EF900C94500E12
:1012B000DF91CF911F910F91FF90EF9008950F93C1
:1012C0001F93CF93DF934115510541F0FC01048139
:1012D00015810115110539F4FB011082DF91CF91C1
:1012E0001F910F910895415051094017510708F47B
:1012F0008A01EB01FC0160817181A801CE010E948D
:1013000033B9C00FD11F1882E9CF20E3FC0120833D
:101310003296862F82958F706F706A3030F4605DE0
:101320006293682F8111F5CF0895695CF9CF8F9290
:101330009F92AF92BF92CF92DF92EF92FF920F9364
:101340001F93CF93DF93CDB7DEB760970FB6F894B6
:10135000DEBF0FBECDBF7C0190914A0C992351F1A5
:1013600008E0933309F404E06B0180E591E00E940A
:1013700009839E012F5F3F4F5901490110E0812FE2
:101380000E94311FF40181934F018823D9F01F5F20
:101390000113F5CF00E0F50181915F018D3161F01E
:1013A000883151F08A51823038F00F5F1013F3CF3B
:1013B0000E94AC2018E08AC060E170E0802F0E949B
:1013C0008F1F102FA12EB12CF501EE0FFF1FE25D34
:1013D000F34F1182108283EE93E00197F1F742E818
:1013E00070E060E0812F0E94721F4FEF62E070E0BA
:1013F000812F0E94721FB601C114D10491F4809113
:1014000090029091910201968115F0EC9F0708F4EB
:1014100071C09093910280939002609190027091BC
:101420009102812F0E945C1F86E0E9E3F3E0DE0178
:10143000199601900D928A95E1F7F70183818F77D4
:101440008C8784818D8785818E87A7014E5F5F4F52
:1014500024E030E06CE070E0812F0E94351FB6017F
:10146000812F0E94461F26E030E0AE01475F5F4FAC
:1014700066E070E0812F0E94351F61E070E0812FEF
:101480000E948F1F27E02A9DC0012B9D900D1124E3
:101490009C012A50344F7901F9011182108222E017
:1014A00030E0AE01415F5F4F68E270E0812F0E9443
:1014B0009F1F8F859889982789279827F7019383FD
:1014C00082831682158214820E94AC20812F60963E
:1014D0000FB6F894DEBF0FBECDBFDF91CF911F9145
:1014E0000F91FF90EF90DF90CF90BF90AF909F90C3
:1014F0008F90089580E090EC8CCFFB01019000204C
:10150000E9F73197AF01461B570B0C947B820F9381
:101510001F93CF93DF93CDB7DEB762970FB6F894E2
:10152000DEBF0FBECDBF8C01CB01F801118210824E
:1015300013821282158214824AE0BE016F5F7F4FD0
:101540000E94CFACBE016F5F7F4FC8010E947D8AB1
:1015500062960FB6F894DEBF0FBECDBFDF91CF917C
:101560001F910F9108950F931F93CF93DF93CDB7E2
:10157000DEB7A1970FB6F894DEBF0FBECDBF8C01CA
:10158000CB01BA01F80111821082138212821582F6
:1015900014822AE0AE014F5F5F4F0E9409ADBE0189
:1015A0006F5F7F4FC8010E947D8AA1960FB6F894A5
:1015B000DEBF0FBECDBFDF91CF911F910F91089578
:1015C000FC0180819181009711F00C948BAC60E05C
:1015D00070E0CB010895FC0180819181009711F0AA
:1015E0000C948FAC60E070E0CB010895AF92BF9295
:1015F000CF92DF92EF92FF920F931F93CF93DF93DF
:10160000DC01CD90DC901197C114D10439F014960F
:10161000CD91DC918C017601209761F4DF91CF911F
:101620001F910F91FF90EF90DF90CF90BF90AF9000
:10163000089575015701BFEFAB1ABB0AF70180810E
:10164000082E000C990B0E94B6AC892B91F72197BC
:10165000CC0DDD1D8881082E000C990B0E94B6ACC4
:10166000892B29F0CE15DF0510F02197F3CFAE01BD
:101670004F5F5F4F4E195F09D80115965C934E93EB
:101680001497CE14DF0420F4B701C6010E94E8B815
:10169000D801ED91FC91119714968D919C91E80FD2
:1016A000F91F1082BBCFFC012481358162177307BB
:1016B00048F480819181009729F0860F971FFC01E3
:1016C0008081089580E00895FC0124813581FB012B
:1016D0004481558124173507A0F0FC018081918158
:1016E000009779F0FB01608171816115710549F006
:1016F000241B350B820F931F0E9415B921E0892B03
:1017000009F020E0822F0895FB0144815581FC01FE
:10171000248135812417350778F0808191810097E5
:1017200059F0FB01608171816115710529F00E94FA
:1017300025B921E0892B09F020E0822F0895CF936D
:10174000DF93EC01FB0101900020E9F73197AF0135
:10175000461B570B0E943D82811103C0CE010E949F
:101760006982CE01DF91CF910895CF93DF93EC0191
:10177000FB0144815581608171810E943D8281110C
:1017800003C0CE010E946982CE01DF91CF910895FE
:10179000EF92FF920F931F93CF93DF93EC017B01A6
:1017A000CB010E94C6AC0097A9F00C811D81080FE7
:1017B000191FB801CE010E941582882361F028818B
:1017C00039818C819D81B701820F931F0E94BFAC2C
:1017D0001D830C8381E0DF91CF911F910F91FF90CA
:1017E000EF900895CF93DF931F921F92CDB7DEB78E
:1017F00069831A8241E050E0BE016F5F7F4F0E9413
:101800003D820F900F90DF91CF910895FB010190E1
:101810000020E9F73197AF01461B570B0C943D822E
:10182000FB0144815581608171810C943D82EF926E
:10183000FF920F931F93CF93DF93EC018B01CB01AA
:101840000E94C6AC7C01BC01CE010E9415828111B0
:101850000BC0CE010E946982CE01DF91CF911F9112
:101860000F91FF90EF900895FD82EC82B80188817E
:1018700099810E94BFACF0CFCF93DF93EC01FB01C5
:101880008617970749F0608171816115710541F0F4
:10189000448155810E947B82CE01DF91CF910895D2
:1018A0000E946982F9CF0F931F93CF93DF938C012E
:1018B000EB01FC01808191810097E1F068817981E1
:1018C00061157105A9F0428153812C813D81421738
:1018D000530770F00E941EB98C819D81F801958399
:1018E00084831D821C82DF91CF911F910F910895F7
:1018F0000E9464B788819981F801918380838A81ED
:101900009B81938382838C819D81958384831982BB
:1019100018821B821A82E5CFFC0180819181009799
:1019200011F00C9464B70895EF92FF920F931F93F8
:10193000CF93DF93CDB7DEB7A1970FB6F894DEBF94
:101940000FBECDBF7C01CB01BA01F701118210821D
:10195000138212821582148242E0420F8E010F5FC1
:101960001F4F0E94C6AA009789F0BC01C7010E94C0
:101970007D8AA1960FB6F894DEBF0FBECDBFDF9172
:10198000CF911F910F91FF90EF900895C7010E9492
:101990006982EFCF0F931F93CF93DF93CDB7DEB75D
:1019A000A2970FB6F894DEBF0FBECDBF8C01CB015E
:1019B000BA01F801118210821382128215821482F8
:1019C00030E0AE014F5F5F4F0E94DAACBE016F5F47
:1019D0007F4FC8010E947D8AA2960FB6F894DEBFA1
:1019E0000FBECDBFDF91CF911F910F910895CF937F
:1019F000DF931F921F92CDB7DEB7FC0111821082D8
:101A0000138212821582148269831A82BE016F5F6B
:101A10007F4F0E947D8A0F900F90DF91CF910895A4
:101A2000FC011182108213821282158214820C949E
:101A3000538CFC011182108213821282158214824F
:101A40000C94178CFC011182108213821282158271
:101A500014820C943C8CFC0111821082138212823D
:101A6000158214826115710551F0FB01019000206F
:101A7000E9F73197AF01461B570B0C947B82089511
:101A8000AF92BF92CF92DF92EF92FF920F931F938C
:101A9000CF93DF936C015B017A018901241735072D
:101AA00020F48F2D7901042F182F6DE574E0C60105
:101AB0000E942B8DD5011496CD91DC91EC16FD067C
:101AC000E0F40C171D0708F4E801D501ED91FC9135
:101AD0001197EC0FFD1F108110826D917C916E0D9E
:101AE0007F1DC60161157105A1F00E947D8AF50177
:101AF00080819181C80FD91F1883C601DF91CF91D2
:101B00001F910F91FF90EF90DF90CF90BF90AF901B
:101B100008950E946982EBCF8F929F92AF92BF92FD
:101B2000EF92FF920F931F93CF93DF93CDB7DEB762
:101B3000A1970FB6F894DEBF0FBECDBF7C01FA01AE
:101B4000CB0119A2223008F42AE08E010F5D1F4F4D
:101B5000822E912CB12CA12CBF01A50194010E94D1
:101B60000FB5F901CA016A300CF5605DD8016E93BA
:101B70008D01232B242B252B79F790E080E0109703
:101B800021F0BD01C7010E940482A1960FB6F8940E
:101B9000DEBF0FBECDBFDF91CF911F910F91FF90A0
:101BA000EF90BF90AF909F908F900895695CDECFCB
:101BB0008F929F92AF92BF92CF92DF92EF92FF925D
:101BC0000F931F93CF93DF937C01EB016C0182E0B5
:101BD000C80ED11C4701E5E08E0E911C10E000E01C
:101BE000F60141916F0150E070E060E02AE0CE0123
:101BF0000E948C8D5C01E881F9810190F081E02DDB
:101C00006EE2CE0119958A0D9B1D080F191FC8148D
